:1000000000800020BD010000C5D700007DD70000A2
:100010007DD700007DD700007DD700007DD7000090
:100020007DD700007DD700007DD70000C5D7000038
:10003000C5D700007DD7000045CE000049CF0000A5
:10004000C5D70000C5D70000C5D70000C5D7000040
:10005000C5D70000C5D70000C5D70000C5D7000030
:10006000C5D70000C5D70000C5D70000C5D7000020
:10007000C5D70000C5D70000C5D70000C5D7000010
:10008000C5D70000C5D70000C5D70000C5D7000000
:10009000C5D70000C5D70000C5D70000C5D70000F0
:1000A00081B300008DB30000C5D70000C5D70000A4
:1000B000C5D70000C5D70000C5D70000C5D70000D0
:1000C000C5D70000C5D70000C5D70000C5D70000C0
:1000D000C5D70000C5D70000C5D70000C5D70000B0
:1000E000C5D70000C5D70000C5D70000C5D70000A0
:1000F000C5D70000E1FB0000C5D70000B1E2000059
:10010000C5D700004DE50000C5D70000C5D70000E9
:10011000C5D70000C5D70000C5D70000C5D700006F
:10012000C5D70000C5D70000C5D70000C5D700005F
:10013000C5D70000C5D70000C5D70000C5D700004F
:10014000C5D70000C5D70000C5D70000C5D700003F
:1001500035D0000049D000005DD0000071D0000013
:10016000C5D7000069E80000C5D70000C5D700006A
:10017000C5D70000C5D70000C5D70000C5D700000F
:10018000C5D70000C5D70000C5D70000C5D70000FF
:10019000C5D70000C5D70000C5D70000C5D70000EF
:1001A000C5D70000C5D70000C5D70000C5D70000DF
:1001B000C5D70000C5D70000C5D70000564B4CF28C
:1001C000205210B51A804DF628121A8000BF00BFC9
:1001D0000DF0FCFA514B4FF010621A60504A9A60D1
:1001E000504ADA60504A136813F4807304D14F49BF
:1001F0000B604FF4A85313604D4B1A78110703D5C9
:100200001A7842F008021A704A4B4B492A221A7097
:100210004A4A4B4B8B4204D252F8040F43F8040B6A
:10022000F8E7484B484900228B4202D243F8042B9E
:10023000FAE74649464A002352F8230041F82300D2
:1002400001336F2BF8D1434B434A802103F8011B44
:100250009342FBD1414B3D4A1A60414B8A221A70AE
:10026000A3F5805324225A70A0221A709A7992071B
:10027000FCD59A79D406FCD43A4A937903F00C035E
:10028000082B384BF9D103221A7140225A719A79FE
:100290009006FCD5334A9179324B4906FBD5324A58
:1002A000324911600221516020221A709A7902F0BD
:1002B0000C020C2AFAD12E4B2E4A1A602E4B2F4AD2
:1002C0001A6000225A60072243F8042C2C4AC3F813
:1002D0000C2D62B60DF02AFE144B1B68DA0705D50B
:1002E00028480DF0F7FB284B284A1A60284B1B784A
:1002F0005B0609D5244C254B22689A4204D121483B
:100300000DF0E8FB0023236010F022FF0DF064FAEB
:100310000DF092F9FEE700BF0E200540308004404A
:10032000823F04000100002B10D0034014D0034092
:1003300002D0074000E00740549CFF1F244D0100FD
:100340004088FF1F549CFF1F7CA4FF1F0082FF1FDB
:100350000000000000E400E05FE400E008ED00E0E1
:100360000050064000400640448004400000030165
:1003700004800440C010050014E000E0FF76010096
:1003800000002020DADD50601CE00340A5C3945A31
:1003900000F00740FFFFFFFFFFFFFFFFFFFFFFFF32
:1003A000FFFFFFFFFFFFFFFFFFFFFFFFFFFFFFFF5D
:1003B000FFFFFFFFFFFFFFFFFFFFFFFFFFFFFFFF4D
:1003C000FFFFFFFFFFFFFFFFFFFFFFFFFFFFFFFF3D
:1003D000FFFFFFFFFFFFFFFFFFFFFFFFFFFFFFFF2D
:1003E000FFFFFFFFFFFFFFFFFFFFFFFFFFFFFFFF1D
:1003F000FFFFFFFFFFFFFFFFFFFFFFFFFFFFFFFF0D
:10040000FFFFFFFFFFFFFFFFFFFFFFFFDEF9FFFF23
:1004100010B5054C237833B9044B13B10448AFF33E
:1004200000800123237010BD549CFF1F00000000BA
:10043000284D0100084B10B51BB108490848AFF31F
:1004400000800848036803B910BD074B002BFBD0A0
:10045000BDE81040184700BF00000000589CFF1F77
:10046000284D0100549CFF1F0000000038B50446D1
:10047000104621700A491D4610F04CFC01464FF011
:100480007E5010F0FBFC074910F044FCE560606012
:10049000256165610DF0DAFCE061204638BD00BFE2
:1004A000DB0FC9400024744938B50446104621705A
:1004B00009491D4610F02EFC01464FF07E5010F009
:1004C000DDFC064910F026FCE56060602561656191
:1004D0000DF0BCFCE06138BDDB0FC940002474495D
:1004E00038B503780446032B20D8DFE803F01A1848
:1004F0001002C168406910F003FB0D4905466068B1
:1005000010F0BCFC0146284610F0B8FC38BD084984
:10051000406810F0B3FCE16810F0FCFB38BDC06827
:1005200038BDC168406910F0EBFA38BD002038BD15
:100530000024744970B504460E460DF087FC05464C
:10054000E069281A10F092FBE3682361E5616661B7
:10055000A0610146606810F091FC0146A06010485F
:1005600010F08CFC0FF062FF0FF002FC10F074FA38
:10057000054601464FF07E5010F0C2FA616910F056
:10058000C9FB21690646284610F0C4FB01463046E7
:1005900010F0B8FAE0602046BDE87040FFF7A0BF59
:1005A000000080BF08B50E200CF020FF114B1B8807
:1005B000012B19D0104B1B88984213DB40F6FF71BA
:1005C0008842D4BFC3EB0001C3EB0101C1EB013191
:1005D000C3F57F630F33282091FBF3F1BDE808409A
:1005E0000DF08ABA0021F3E70146BDE80840142067
:1005F0000DF082BAB09EFF1F449DFF1F10B5044648
:100600000CF0F6FC204610BD70B44C88A04220D9F6
:1006100001230133DBB21CB2660031F8144084427E
:100620001D46F6D3A04211D005F10045013D965B71
:1006300031F8151032F81530401AF21A00FB02F0AA
:10064000641A90FBF4F4E01870BC7047905B70BCC7
:10065000704702260125E5E700280CDA064A4342E6
:1006600082FB0320DA17C2EB600000EB4000A3EB33
:100670008000C0F10C007047ABAAAA2A38B5234B02
:100680001B78002B2CD015200CF0B0FE204B1860EE
:10069000204B1B88984203DA1F4C237863BB38BD7C
:1006A0001E4A1488A042A4EB0302A8BF20467F2A5A
:1006B0001CDDC01AC001541C90FBF4F4002CEBD0DC
:1006C000154B1A780AB901221A70154D2B689C42F5
:1006D00004D0144BE1B2187808F0FCFE2C6038BD51
:1006E00011200DF09FFF0A4B1860D1E7C01AC0EB34
:1006F000C01090FBF2F4E1E70A4B0021187808F0F3
:10070000E9FE0023064A2370136038BDC29EFF1F16
:10071000809CFF1FFE9CFF1F389FFF1FDC9EFF1F5A
:10072000349FFF1FD49CFF1F38B50F200DF07AFFB8
:100730001B4A1C4B12881860C0F53B600830904281
:1007400020DB194B1B889842A3EB0204A8BF184674
:10075000801A7F2CC6BFC0010134C0EBC01090FBD3
:10076000F4F47CB1114B1A780AB901221A70104DB9
:100770002B689C4204D00F4BE1B2187808F0AAFE17
:100780002C6038BD094C237803B938BD094B0021D2
:10079000187808F09FFE0023054A2370136038BDC7
:1007A000489DFF1F989CFF1FC89EFF1FEC9EFF1FC8
:1007B000089DFF1FF69CFF1FF0B40E8886420DD2E5
:1007C00003F10043013B31F81350854202D9F0BCDC
:1007D000FFF71ABF32F81300F0BC70471088F0BC66
:1007E000704700BF094B1B880C2B09D8084A80B200
:1007F00052F8232028B143F6FE73984203D9108C97
:100800007047108870470349FFF7FEBEAE9CFF1F7C
:1008100040270100DC2801004B4B4C4A2DE9F047F2
:100820001E8814684A4BB442B3F80080494B33DB4E
:100830004445A8BF4446A6421C60C8BF00202DDD29
:10084000C6EB0807B7F5804F33DB80037B1C90FBBA
:10085000F3F0FFF7C7FF404A404B15881B88C0F3F1
:10086000C61909FB05F57F2D8246A8BF7F252BB34E
:10087000A64253DC4445D4BFC6EB0404C6EB0804CF
:100880009F42CCBF03FB04445C43354BC8BF0137D8
:1008900094FBF7F71F6013E034461E60C6EB0807B1
:1008A000A045D4BFC6EB0800C6EB0400B7F5804FE7
:1008B000CBDAC0EB803090FBF7F0CAE7284A136030
:1008C000284C2368994508D0274B1B88002B34D12E
:1008D000264B1B886BBBC4F80090254C23689A45B7
:1008E00006D0214B1B885A1F032A19D9C4F800A02F
:1008F000204C23689D420FD01F4B188848B11A4BDB
:100900001E4A1B88D35C834203D0C0B2E9B208F010
:10091000E1FD2560BDE8F087BDE8F0870024AFE782
:10092000164AD05C2030C0B20AF07F0108F0D2FD38
:10093000DCE7484608F06EFECDE7104A4946D05C39
:1009400008F0C8FDC4E700BF449DFF1FAC9EFF1F19
:100950000E9FFF1F789CFF1F889CFF1F8A9CFF1F14
:10096000149FFF1FF09CFF1F929EFF1F3A9DFF1FC9
:10097000A89CFF1F3C9DFF1FA29EFF1F9C89FF1F7D
:100980002DE9F04F17208BB00DF04CFEDFF870B35F
:10099000DFF870A3CBF8000016200DF043FEBA4B31
:1009A000CAF800001B880C2B00F05E82B74EB84AD4
:1009B0003188B84B52F8214000221A70B64BB74A22
:1009C0001B88B7491288013B012A31F9133005937E
:1009D00000F0AE81B34B0193B34B0293B34FDFF8FA
:1009E000288300230093B24B1B88012B00F0F48175
:1009F000DFF81893AF4B0393D9F80050AE4B049334
:100A00000023AE4A1288013A032A00F24982DFE845
:100A100012F0A500ED000400C9002846059310F06F
:100A200025F9A74910F076F9059B0546184610F000
:100A30001DF9A44910F06EF90146284610F062F83D
:100A400010F02EFB0546C9F80050386810F00EF97A
:100A50009B4910F05FF98146009810F007F9994919
:100A600010F058F90146484610F04CF810F018FB09
:100A70003860954A954B17881988954BDBF800200C
:100A80001B88DFF88CE2C7EB050C3D44039FC7F8D9
:100A900000C0471A084404990D6001990F6002993B
:100AA000BEF8007008609A4280F2E7800025C3EB30
:100AB000070E7445DAF8000080F2D380611C98427A
:100AC00005FB01F50EF1010E95FBFEF5C0F25F830B
:100AD0008742A8BF0746FF1A01FB07F494FBFEF408
:100AE0009A4200F3A780984200F3A480794C2068D2
:100AF00010F0BCF8784910F00DF9784910F002F8C0
:100B000010F0CEFAA0F5FF531C3B082B98BF4FF412
:100B10000050D8F80030184400282060C0F29F80B0
:100B2000B0F5804F80F2F6806D4B1B781BB1B0F5AD
:100B3000005F40F0F7806B4D2B78002B40F0AB81CD
:100B4000694D20682B68634C984204D080B208F04D
:100B500091FC23682B600BB0BDE8F08F284605930D
:100B600010F084F8614910F0D5F8059B0546184649
:100B700010F07CF85E4910F0CDF8014628460FF0E1
:100B8000C1FF10F08DFA0546C9F80050386810F022
:100B90006DF8564910F0BEF88146009810F066F8DE
:100BA00053495DE72846059310F060F84A4910F074
:100BB000B1F8059B0546184610F058F84D4910F05D
:100BC000A9F8014628460FF09DFF10F069FA054686
:100BD000C9F80050386810F049F83F4910F09AF809
:100BE0008146009810F042F8424939E728460593BB
:100BF00010F03CF8404910F08DF8059B054618466A
:100C000010F034F83D4910F085F8014628460FF001
:100C100079FF10F045FA0546C9F80050386810F021
:100C200025F8354910F076F88146009810F01EF846
:100C3000324915E73388002B3FF458AF2B1B002BAC
:100C4000B8BF5B42092B00F32D81D8F80030214C4E
:100C50004FF40050184400282060BFF661AF002216
:100C60005AE0984205FB04F5B8BF002195FBFEF55C
:100C700080F2848291FBFEF432E7BA42D4BFC3EB28
:100C80000205C3EB070512E7DE9EFF1FE49CFF1F72
:100C90005889FF1F7E9CFF1F2089FF1FB29EFF1FE8
:100CA0006C2B0100D89CFF1F189DFF1F709CFF1F1D
:100CB000409EFF1FD09EFF1F449EFF1F2E89FF1FD7
:100CC000CDCC4C3FCDCC4C3EA889FF1F2C89FF1FBB
:100CD000A89EFF1F9089FF1F9A99193FCDCC4C45C4
:100CE000EA9FFF1F399DFF1F2489FF1F3333733F86
:100CF000CDCC4C3DCDCCCC3E6666663FCDCCCC3D1C
:100D0000E09CFF1FA49CFF1FE89EFF1FCC9EFF1FBF
:100D1000C09CFF1F43F6FF72C04B22601B78002B64
:100D20003FF409AF05F076FCBD4B01221A7007E7CE
:100D3000BC4BBD4A1B88BD491278013B31F91350A9
:100D4000002A40F0C78011200DF06CFC0090B84BD9
:100D50000193D3F80080009B984540F3C080B54BC9
:100D6000B54F1B88B54A012B3B68B2F80090B44AD6
:100D700002922046A3EB050500F0E2800FF076FF1B
:100D8000029A52F829100FF0C5FF014600200FF01B
:100D9000B7FE10F085F9009BC8EB05029D42B8BF75
:100DA0001D469042C8EB050580F2DE8000FB05552C
:100DB000013295FBF2F5A34BDFF8B4820293D8F829
:100DC00000302B4403EBD3735B10C8F800309E4B0C
:100DD0001B88012B7FF40CAE9C4B03931D460F2008
:100DE0000DF020FC2A6804929042034680F2CC80E9
:100DF000904A1288012A00F03F81904A0790128899
:100E00008F4D069220460FF031FF069ADFF864926C
:100E100055F82210D9F800500FF07CFF0146002051
:100E20000FF06EFE059BEA1A059210F039F9059A4B
:100E3000079B04999A42C1EB020EB8BF1A4670454F
:100E400080F24481521A00FB02220EF1010192FB52
:100E5000F1F2D8F800107E4804900A4402EBD272F6
:100E60005210C8F80020CCE57A4B1B78002B3FF4D9
:100E70009DAD794E794A3188794B52F82100012293
:100E80001A700FF0F3FE4FF07C510FF043FF10F09B
:100E900007F9044692E505F0B9FB00232B704FE6F5
:100EA0003868E6E505F500500130001B0FF0DEFE66
:100EB0006C496D4C0FF02EFF054620680FF0D6FEF2
:100EC0006A490FF027FF014628460FF01BFE10F07D
:100ED000E7F81EE615200CF089FA009037E7594B29
:100EE0000293D3F80080009B984542DA514B524F51
:100EF0001B88524A012B3B68B2F80090504A03927B
:100F000020461D4400F0E9800FF0B0FE039A52F82D
:100F100029100FF0FFFE10F0C3F8009B9D42C8EBB4
:100F20000502A8BF1D46C8EB05059042BABF00FBED
:100F300005550132454395FBF2F5DFF834813EE774
:100F40000FF094FE029A52F829100FF0E3FE10F011
:100F5000A7F8009BC8EB05029D42B8BF1D46824220
:100F6000C8EB05053FF722AF00FB05F595FBF2F551
:100F700021E7DFF8FC80304FD8F8003003EBD37363
:100F80005B10C8F800302EE5314A049212680692D0
:100F9000904237DD274A1288012A00F0BC80274A98
:100FA00009901188264A0891204607920FF05EFEAC
:100FB000079A0899DFF8BC9052F82110D9F8005030
:100FC0000FF0A8FE059B2B44059310F069F80599D6
:100FD000099B069A9942C2EB010EA8BF19467045BB
:100FE00080F2BE80891A00FB01110EF1010291FB13
:100FF000F2F2D8F800100A4402EBD2725210C8F88C
:101000000020FEE4D8F80020DFF8689002EBD272EE
:101010005210D9F80050C8F80020F2E4EA9FFF1FF0
:10102000399DFF1FAC89FF1FC29EFF1F942801003E
:10103000D89CFF1F1E9DFF1F709CFF1FC89CFF1F99
:10104000842B0100189DFF1F409EFF1FD09EFF1F95
:10105000449EFF1F909EFF1FE49CFF1F5889FF1FA7
:101060007E9CFF1FCDCCCC3E9089FF1F9A99193FE3
:10107000E89EFF1FCC9EFF1F464A08901188464AF3
:101080000791204606920FF0F1FD069A0799DFF8C6
:101090000C9152F82110D9F800500FF03BFE059B3F
:1010A000E91A05910FF0FCFF0599089B049A9942F3
:1010B000C2EB010EB8BF1946704558DA891A00FB19
:1010C00001110EF1010291FBF2F2C2E60499521AEB
:1010D00000FB02F292FBFEF2BBE60FF0C7FD039AA3
:1010E00052F829100FF016FE014600200FF008FDFF
:1010F0000FF0D6FF009A9542C8EB0503A8BF15462E
:10110000C8EB05059842BABF00FB055501334543BE
:1011100095FBF3F511E71F491F4A089020460D88FB
:1011200007920FF0A3FD079ADFF8709052F8251090
:10113000D9F800500FF0EEFD014600200FF0E0FC62
:10114000059B2B4405930FF0ABFF0599089B069A6E
:101150009942C2EB010EA8BF19467045FFF642AF97
:10116000069A891A00FB01F191FBFEF241E7049A0D
:10117000891A00FB01F191FBFEF26AE6B842D4BF86
:10118000C3EB0001C3EB070104FB01F172E51F464D
:10119000A1E400BFC89CFF1F842B0100CC9EFF1F51
:1011A00008B5244B1B88FBB1234B1B78FBB1234BA9
:1011B0001B78E3B1224B1B78CBB1224B1B78B3B128
:1011C000214B22481A78C2B9214A22490088128844
:1011D00009680244B1EB620F09DD01221A70642034
:1011E000BDE8084005F02ABA174A117801B908BDD0
:1011F0001370BDE8084008F0E1B9154A16490088A7
:10120000128809680244B1EB620FF0DD00221A7007
:1012100008F0D4F9642005F011FA642005F00EFA04
:10122000642005F00BFA4FF41670BDE808400CF08E
:101230002FBE00BF509EFF1F3C9FFF1F089FFF1F38
:10124000099FFF1F0A9FFF1FAC9CFF1FC09CFF1F31
:10125000A89EFF1FE09CFF1FA49CFF1F38B5114CE8
:10126000232025780CF0C2F80F4A42F82500131FFE
:1012700002F1C400002253F8041F83420A44FAD149
:1012800023780A4907480A4C0133DBB2322B81FB31
:10129000025108BF0023D217C2EB21120370226053
:1012A00038BD00BF8C9CFF1F549DFF1F1F85EB5155
:1012B000A49EFF1F2DE9F04FB84CB94D2068B94FDF
:1012C00083B00FF0D3FCB8490FF024FD0646102080
:1012D0000DF0A8F90FF0CAFCB4490FF01BFD314620
:1012E0000FF010FC0FF0DCFE2988206088423B885C
:1012F00043DA9E465B1A7F2B4FF0000247DDD20196
:101300005E1C92FBF6F2AA4EDFF8C882B6F800C067
:10131000C8F80020BCF1190F00F0DF80BCF11A0FF3
:1013200000F01881BCF11E0F00F021810126B146AA
:10133000A04A1288002A00F09D808842C0F20881ED
:101340007045D4BFC1EB0000C1EB0E009A42BABF9A
:1013500002FB00000133504390FBF3F3964A136005
:10136000964B1888C0B9964A1288AAB9954B197835
:1013700001B11A7003B0BDE8F08F9842D4BFC1EB41
:101380000002C1EB03029E465B1A7F2BB7DCC2EB67
:10139000C21292FBF3F2B6E72988D4F800E0DFF836
:1013A0000082DFF8F8A171456CDCDFF818C29CF808
:1013B0000020002A2ED14FF0010B04288CF800B039
:1013C00028D1002E40F095817D4B18880028D1D07F
:1013D000B9F1000FCED023682C883A88A34280F25E
:1013E00066810023141B7E2C774DD5BFC3EB83137E
:1013F000C3EBC3135B00013493FBF4F42B6801349B
:10140000A34203D0C0B2E1B208F064F82C6003B08C
:10141000BDE8F08F012800F0F780022800F0EC8092
:101420000328D1D1694B1B88092BCDD0002ECBD0FE
:1014300023682E883A88B34280F27C810023961B71
:101440007E2EDFF88CA1D5BFC3EB8313C3EBC31390
:101450005B00013693FBF6F6DAF800300136B34252
:1014600003D0F1B24A2008F035F8CAF80060ABE7C3
:1014700091460126BCF11E0F7FF472AF0022DFF807
:1014800058817FE04F4B1A78002A3FF473AF002455
:1014900001281C7000F0A480022840F00F81002E6B
:1014A00000F0A3804A4D2B68002B00F09E800420A2
:1014B000214608F00FF8424B2C60188800283FF4B2
:1014C00059AFB9F1000F3FF455AFC0B2002108F099
:1014D00001F83D4B00221A604CE7DFF8FC8098F8D9
:1014E0000020C2B1DFF8D890B9F800A0BAF1000F1F
:1014F00011D0DFF8E89099F800B0934578D05FFA02
:101500008AF07F2107F0E6FF98F80030B6F800C0B7
:1015100089F8003010E0DFF8C49099F800A09245F7
:1015200066D0274B0021187807F0D4FF98F80030D8
:10153000B6F800C089F800301E4B1A88002A97D0F0
:10154000BCF11E0F40F0078101264FF0000919E0A1
:101550000020FBE6DFF8808098F80020002A0BBF0F
:10156000012600264FF000094FF00109E0E6DFF800
:101570006880104B98F800601A88B6FA86F67609EB
:101580004FF0000998F80030002B3FF4E7AE2988AF
:10159000B7F800E02068C1EB0E03CEE6D09CFF1F39
:1015A000569EFF1F529EFF1F9A99193FCDCCCC3EED
:1015B000DE9EFF1F189FFF1F4C9DFF1FDE9CFF1F1D
:1015C000F09EFF1FE59EFF1FB49CFF1F929EFF1F12
:1015D000509DFF1FC49EFF1F909EFF1F929CFF1FE8
:1015E0001EB1624D2B68002B7CD1614B188865E7DA
:1015F00001264FF000099BE6002E3FF4E5AEDFF830
:101600006CA1DAF800202EE0002E3FF4DDAEB7F832
:101610000080F045D4BFC1EB0802C1EB0E02C1EB64
:101620000808B8F17E0FDFF844A1D5BFC2EB8212E3
:10163000C2EBC212520008F1010892FBF8F8DAF886
:10164000002008F10108424506D05FFA88F1012028
:10165000009307F03FFF009B1888CAF8008002281B
:101660007FF4DEAE42462168B5F8008038884145F7
:1016700059DA0021C8EB0008B8F17E0FD3BFC1EBE7
:101680008111C1EBC11108F10108490091FBF8F883
:1016900008F10108904506D05FFA88F10420009314
:1016A00007F018FF009B1888CAF80080B8E693423C
:1016B000D4BFC4EB0303C4EB020393E6032827D192
:1016C0002C4B1B88092B90D0002E8ED0274D2B68D9
:1016D000002B8AD04A20214607F0FCFE244B2C60C8
:1016E0001888EBE6214607F0F5FE214B2C601888A0
:1016F000E4E640207F218DE80C0007F0EBFE019B23
:10170000009A188858451CD002287FF489AE76E7E5
:1017100004287FF46AAF002E3FF467AF21464020D3
:1017200007F0D8FE61E78142D4BFC8EB0101C8EBE6
:1017300000019FE79342D4BFC6EB0303C6EB02034D
:101740007DE6B8F80010DAF800E0B7F800808E45C2
:10175000FFF665AF5DE72988B7F800E02068C1EBC8
:101760000E0301264FF00009E7E500BF509DFF1F63
:10177000F09EFF1F929EFF1F08B5114B1B88022B86
:1017800009D0052B07D0032B15D0042B0BD00D4B04
:1017900001221A7008BD7F21412007F09BFE094BF2
:1017A00001221A7008BD7F21092007F093FE054B26
:1017B00001221A7008BD4021092007F08BFEE6E7E0
:1017C0004A9DFF1F009DFF1F38B5074B074D1B8823
:1017D000052B044606D02B68834203D0C1B20520F6
:1017E00007F078FE2C6038BD4A9DFF1FF49EFF1F56
:1017F00038B5124D124C2B88052B12D022684AB9ED
:10180000022B0ED0033B012B13D90E4A0023137079
:10181000236038BD0021052007F05CFE2B88022BD9
:1018200004D10021412007F055FEEEE7052BE9D158
:10183000F7E70021092007F04DFEE6E74A9DFF1F6C
:10184000F49EFF1F009DFF1F464B1B881D2B70B58C
:1018500041D0454D0024454B1B88022B16D0444BEC
:101860001B88022B54D02888424B002C1B780ADBA3
:101870008442A8BF044634B1002B3AD02046BDE8CC
:101880007040FFF7A1BF002B2FD170BD3A4B1B78E2
:10189000002B37D015200BF0A9FD384B1860384AC3
:1018A0001288002ADBD0374A186811888142D6DCBA
:1018B000354B2A881B888342A3EB0106A8BF034649
:1018C0005B1AB242BABF02FB03330136534393FBA8
:1018D000F6F31C44C3E72A4B1C888CB12B4B224DDA
:1018E0001C78002CB7D02C88B5E7BDE87040FFF716
:1018F0007FBFFFF741FF2046BDE87040FFF764BFA0
:10190000194DA8E711200CF08DFE1C4B1860C6E79E
:101910000F200CF087FE1A4B1D4A1B881060002B0D
:10192000A1D01C4AC0F53B63118808338B429ADB77
:10193000194A288812889342A2EB0105A8BF1346D2
:10194000A842A3EB010306DA00FB0333013593FB46
:10195000F5F31C4488E700FB03F292FBF5F31C440B
:1019600082E700BFDE9EFF1FE29EFF1FB29EFF1FA9
:10197000409EFF1F009DFF1FC29EFF1F809CFF1FF8
:101980004A9DFF1FFE9CFF1FDC9EFF1F909EFF1FB6
:10199000989CFF1F489DFF1FC89EFF1F38B5102051
:1019A0000CF040FEC830B0F5FA7FC0F2EE80B0F522
:1019B0007A6F0146A8BF4FF47A6101F51673B3F54B
:1019C0007A6FA8BF4FF47A639BB289B28E4A8F4C6C
:1019D00011802220238007F0D7FE21888C4D8D4C6A
:1019E000242007F0D1FE0E200BF000FD40F6FF7121
:1019F000C8308842A8BF084620EAE07000F2DC52F6
:101A000083B28A42A8BF0A460220194622802B8050
:101A100007F0BAFE2188042007F0B6FE17200CF06C
:101A200001FE044616200CF0FDFDA042B8BF204682
:101A300000F1C801B1F5FA7FC0F2A280B1F57A6F6A
:101A4000A8BF4FF47A6101F54873B3F57A6FA8BF68
:101A50004FF47A639BB289B26F4A704C11800A20AE
:101A6000238007F091FE21880C2007F08DFE0F20C7
:101A70000CF0D8FDC0F53F610431B1F5AF6F7CDBF0
:101A8000B1F5FA6FA8BF4FF4FA6189B2644BC0F5A3
:101A90004360B0F5AF6F19806CDBB0F5FA6FA8BF8B
:101AA0004FF4FA6083B25F4CA420238007F06CFEF1
:101AB000A620218807F068FE0B200CF0B3F900285F
:101AC00068D011200CF0AEFD00F1C801B1F52F7FF8
:101AD0006EDA40F214534FF42F71534A1180534C75
:101AE0000620238007F050FE2188082007F04CFED6
:101AF00000244FF4AF75E1B24D4809F0B5FC013454
:101B00008542A8BF05460C2CF5D101200CF08AFDBA
:101B1000044600200CF086FD323CA0F1320345491A
:101B20006FF4957000FB03F300FB04F081FB0342AC
:101B300081FB0041DB17C017C3EB6223C0EB6120C0
:101B400003F5AF7200F5AF739342A8BF13469D42F1
:101B5000A8BF1D46A5F11401312938DC40F26C7391
:101B600032213548354A018013602A20BDE83840CB
:101B700007F00ABE4FF4AF6395E74FF4AF6185E716
:101B800040F214534FF4FA7166E740F24C434FF4BD
:101B9000FA711BE715200BF029FC00F59671B1F5E1
:101BA0002F7F96DB41F25C2399421FDD194694E7B3
:101BB00041F25C239942F9DC1B4A00F5487089B276
:101BC000B0F52F7F118019DA4FF42F7387E740F2B9
:101BD0003A72A5F5B9751A4B02FB05F583FB05238F
:101BE000ED17A5EB631389B23233BAE70E4A00F55D
:101BF000617089B2B0F52F7F1180E5DB8342A8BF09
:101C000003469BB26BE700BF569EFF1F529EFF1F0D
:101C1000449DFF1F0E9FFF1FA89EFF1FC09CFF1F1C
:101C2000489DFF1FC89EFF1FFE9CFF1FDC9EFF1FDD
:101C3000389DFF1F67BBCF46069FFF1F9889FF1F78
:101C4000B5814E1B2DE9F84F0C200BF09BFB0C20AF
:101C50000CF050F8C149DFF88CA314200CF05AF8AE
:101C6000BF49C04809F092F8022103200CF0E8F8BF
:101C7000022104200CF0E4F8022105200CF0E0F829
:101C8000022106200CF0DCF801210A200CF0D8F823
:101C9000012109200CF0D4F801210D200CF0D0F81E
:101CA000012128200CF0CCF8012114200CF0C8F8F8
:101CB00002210B200CF0C4F801210C200CF0C0F81C
:101CC00000210C200CF0A8F8012121200CF0B8F81C
:101CD00002211C200CF0B4F801211B200CF0B0F8FC
:101CE00000211B200CF098F81C200CF09BF8B0FA97
:101CF00080F35B091A208AF800300CF037FA1F20B5
:101D000000210CF0F9F904200CF08CF8002800F008
:101D1000EA8005200CF086F8002800F017810023E7
:101D2000914C062023700CF07DF8B0FA80F35B092B
:101D30004FF0000B8D4A137006F0A4F82378002BA7
:101D400040F0CD80584607F049FD894B894A1B88F1
:101D500089491488894D8A4840F23A72A3F5AF73D5
:101D600002FB03F381FB0312DB17A3EB6213323395
:101D70002B60844B5A211C7009F0B2FB002800F044
:101D80003781814A81481268DFF85C920023012183
:101D9000FEF78AFB0B200CF045F8011E0CBF012357
:101DA000002389F8003000F0B780794F794D7A4EE2
:101DB000DFF8388200233B602B60336004240F205F
:101DC0000CF030FC336803440E2033600BF00EFB44
:101DD0003B6899F8002018443860002A78D0152014
:101DE0000BF004FB2B681844286004F0010080F01D
:101DF000010004F013FCB8F80030002B14BF4B2096
:101E0000DC200CF045F8013CD9D133683968604AD0
:101E10002868624F002BB8BF03330029B8BF0331D5
:101E2000891011605E495F4A098814889B10002858
:101E30003360B8BF03305C4E8210581A19442A60D0
:101E400031603860594D5A485A49161B22442E6059
:101E500002600B60BBF1000F62D1B8F80030002BBC
:101E60004DD0554B012404201C600BF0DBFF18B94A
:101E7000524B444A1C701070514B1B881C2B56D07F
:101E8000504C04F1C80523200BF0B0FA44F8040FBD
:101E900001200BF0FDFFAC42F5D19AF800301BB1E8
:101EA000494B1B78002B4CD1002121200BF0B4FFB3
:101EB000464A474B1078187007F098FA04F0A6FBD2
:101EC00045F6BF5243494448BDE8F84F0BF046B8C9
:101ED00011200CF0A7FB2B681844286085E7BDE8AB
:101EE000F84F08F063BE06200BF09CFF00287FF43B
:101EF00010AF1D4C034620704FF0010B1AE74FF452
:101F0000FA7004F09BFB04F085FB06F00FFB4FF426
:101F1000AF600BF0BDFFA4E711200BF091FF44E789
:101F2000FFF73CFDB8F80030002B9AD1E7E72B4BC8
:101F300018880028A4D02A4BC0B2197807F0CAFA32
:101F40009EE7012121200BF067FFB1E703200BF092
:101F500069FFB0FA80F35B09E2E600BF001B374679
:101F600040420F005C91FF1FB29CFF1F489EFF1F65
:101F7000069FFF1FE09EFF1FB5814E1B9889FF1F24
:101F8000389DFF1F149DFF1F2889FF1F709EFF1F94
:101F9000849CFF1F709CFF1FCC9EFF1FD09EFF1FC5
:101FA000A889FF1F2C89FF1F449EFF1FD89CFF1F7D
:101FB000189DFF1F209FFF1FD89EFF1F9C9CFF1F87
:101FC000DE9EFF1F509DFF1F589EFF1F5A9EFF1F42
:101FD0003E9EFF1FA5050000FC9EFF1F1C9DFF1FCE
:101FE000CC9CFF1F429EFF1FC29EFF1F9E9EFF1F95
:101FF00003200BF017FF0028FAD104200BF012FF8A
:102000000028F5D105200BF00DFF0028F0D10620A7
:102010000BF008FF0028EBD10CF024FC2DE9F04F69
:1020200089B005ADA14F2C4608AE611BC9B2A048CE
:1020300009F01AFA3B88834294BF0020012004F87B
:10204000010BA642F1D19B489B4A9DF814E09B49A5
:1020500080F800E09DF81600994D10709DF818204A
:102060009DF81C30974E984C0A709DF81A102970F4
:1020700000253370257073B9002940F00F81934F0C
:102080001AB13B78002B40F01F82002800F0F2814B
:102090000222227005E0002A40F0B08005228B4F1A
:1020A00022708B4BDFF888929DF815109DF819006F
:1020B000DFF880A2DFF880B2864DDFF88082864E9E
:1020C0003A709DF81EE019709DF81F209DF81D10B4
:1020D0009DF817C09DF81B7089F80000012000933F
:1020E0008BF800E088F8001032708AF800C02F707A
:1020F0000CF098FA79497A4AD1F800E0009B7045D3
:10210000CCBF0121002111707CDD764A1288182A8B
:1021100078D875490F880C3A002F78D1734993F815
:1021200000C00B7899F800909AF800109BF80070A6
:1021300095F800B02478A3EB4C03A9EB890A5B1A4D
:102140005344C7EB877AC7EB8A07DFF8A8A11F447F
:1021500098F80030BAF800A007EB4B0796F800B0EB
:102160003B440BFB0A33624F4FF00C0A1AFB043A54
:10217000C7F800A0B9F1000F0BD033784BB15D4B1D
:102180001B88042B0CBF0AF1020A0AF1040AC7F8E3
:1021900000A0594B594CDFF8A8B11B882488DBF804
:1021A00000B0574F574E3F883688033BC4EBC404FA
:1021B0005C4403EB4303DFF88CB10AEB83033B443D
:1021C000DBF800B0504FC6EBC60657F824404F4F1F
:1021D0005E440C3B134457F826601A193244BCF194
:1021E000000F27D02B782BB300295BD1B9FA89F9DE
:1021F000474B4FEA591983F8009023E006222270DA
:10220000324F4EE738490F880022002F86D0012F29
:1022100000F0CF80022F00F0FB80032F00F09480AD
:10222000334F9AF8001093F800C099F80090D7F84F
:1022300000A09FE7364B00241C7011B198F80030C5
:1022400023BB0021334B70451970C8BF324B334953
:10225000C8BFC3F800A00B689A4213D0304B314C72
:1022600018680390039820601B6804932E4C049B0D
:1022700024880A601B1AA34284BF2C4B1A6009B041
:10228000BDE8F08F2748264B0068EDE7BCF1000F52
:10229000D7D1B9F1000FD4D10121D3E704222270A4
:1022A0000A4FFEE61A4B00211970CAE7069FFF1F6E
:1022B000389DFF1F089FFF1F099FFF1F0A9FFF1FD9
:1022C0000B9FFF1F0C9FFF1F4A9EFF1F549EFF1F67
:1022D000399FFF1F3D9FFF1FE49EFF1F9889FF1F2F
:1022E000909EFF1FDE9EFF1F7C9CFF1FAA89FF1F81
:1022F000989EFF1FEC9CFF1FB69EFF1FD49EFF1FE2
:102300008E9CFF1F029DFF1F482901000024010031
:102310001A9FFF1F1B9FFF1F249FFF1FF89CFF1F7B
:1023200028A0FF1FE89CFF1FEE9EFF1F2C9FFF1F92
:102330003B9FFF1F3A9FFF1F3C9FFF1F3E9FFF1FBA
:102340004C9DFF1F149FFF1F664993F800C00B7838
:1023500099F800909AF800109BF8007094F800A08B
:102360002C78A3EB4C03A9EB890B5B1A5B444FF071
:10237000050B1BFB0733009398F800300193009B7B
:10238000DFF86CB1C7EBC707BA440533019FBBF850
:1023900000B003EB440334783B4404FB0B33524C52
:1023A000524F54F82A400C3303EB040AC7F800A03C
:1023B000E0E64C4993F800C00B7899F800909AF841
:1023C00000109BF8007095F800A02478A3EB4C0354
:1023D000A9EB890B5B1A5B44C7EB877BC7EB8B07C9
:1023E000DFF80CB13B4498F80070BBF800B003EB89
:1023F0004A0A3378BA44C4F1060403FB0BA3E4B2DF
:102400004FF00C0A394F1AFB043AC7F800A0B1E6A6
:10241000344993F800C00B7801932B780093019B0B
:102420009AF8001099F800909BF800A02478A3EB8C
:102430004C03A9EB890B5B1A5B44A3F1020B2C4BF9
:10244000CAEBCA0A54441B88DFF8C8A00193BDF840
:1024500000305AF824A098F8004017FB03BB3778E7
:10246000019B5C4407FB03431833204F9A44C7F891
:1024700000A07FE6BEF1000F29D13A78012A2FD9BA
:102480001C4B22701B882BB31B4B1B88013B9BB240
:10249000062B1FD8194B1B78E3B1194B1B68012B76
:1024A0007FF4FFAD1749184B0968184D83FB0130C5
:1024B000CB17C3EB600303EB4303A1EB83032B8038
:1024C000134B03211970ECE503222270E9E5012288
:1024D0002270E6E50A4B1B68012B7FF4E2ADEFE7C3
:1024E0007246DEE5AA89FF1FCC2C0100989EFF1FD3
:1024F000EC9CFF1FC09EFF1F5C9EFF1F469DFF1FA1
:10250000D89EFF1F2C9FFF1FABAAAA2A9C9EFF1FCD
:102510008C89FF1F342B01002DE9F04F3A4B1B78BB
:102520008BB0002B6BD10E200AF060FF0EF09EFBEB
:1025300001463648364E374DFDF7FCFF3348FDF770
:10254000CFFF0EF0ADFD80F30C003060FFF766FDAD
:102550002C68012C7AD0022C00F0CB82032C00F0E6
:10256000DF832D4E2D4C33682D4A2E4E0993099B47
:10257000316812882360591A013A9142274F00F2BC
:10258000B382294E32689A1A0D2A00F29C82274E95
:1025900032689A1A132A00F29182254E32689A1AEA
:1025A000252A1AD9234B1B88002B40F06481224B2B
:1025B0001B78002B40F05F81FEF750FE1F4B1B88FD
:1025C0001B3B9BB2022B04D81D4B1B78002B40F009
:1025D000558104F045F8236833601A4D2A689B1A28
:1025E000502B00F21982184B1B88012B00F031820E
:1025F00006F0F4FE06F0D8FD0BB0BDE8F08F08F051
:102600005DF90BB0BDE8F08FB29CFF1F709EFF1FFD
:10261000AC9EFF1FD89EFF1F28A0FF1F6C9EFF1FB0
:102620009489FF1F409DFF1F2C9DFF1F0C9DFF1FC6
:10263000109DFF1F509EFF1FAC9CFF1FDE9EFF1FC3
:10264000909EFF1F609EFF1FB09EFF1FDFF8389314
:10265000A44AB9F800001378834204D0C3B21846E4
:10266000137006F0ADFEDFF81C839F4AB8F8003007
:102670001178994204D09D4F3978002940F03E8767
:102680009B4A336812889B4E9A42C0F201819A4A53
:102690001278002A40F0FC80DFF8F0A2BAF800308F
:1026A00023B9964B1B88002B00F05C85944A954B10
:1026B00011881B88944A0B4412685B109342934A1A
:1026C000126880F2FE8400219342B4BF01230B46BE
:1026D00004910093ACBF4FF0010B8B4605910E2087
:1026E0000AF084FE8A4B8B4A1B68176803930133F8
:1026F000A7F25232002B8446029240F31087802BBF
:10270000A8BF8023844A854912780191002A00F0ED
:10271000C9800978914200F0C580B8F80010DFF850
:1027200064E2994201F0F8807049AEF800307C4BC9
:102730004FF0010E81F800E01978DFF854E2019BB8
:102740008EF800101A70009B002B00F02381BAF85D
:102750000030002B00F01E81724B1B685A1C002AAF
:1027600040F3E886802A00F3E4866F4C6F49704896
:102770002488098800682144B0EB610FC1F25D83B1
:10278000A3F148020F2A02D8473BA9F800300E20D7
:102790000AF02CFE6FF454731F44874202DC654B31
:1027A00000221A7000200BF03DFF634A634B116852
:1027B000634C1B888842D4BF002201222270002B68
:1027C00000F075845F4B1C78944243D0884241DD11
:1027D0005D490C78002C00F09A875C4991F800C0A4
:1027E000BCF1000F40F09187594F0097594F5A485C
:1027F0000297574F007887F800C0564F4FF0010EF0
:1028000087F800C081F800E0002841F0F5805349C6
:102810000978002901F02980514903910C46097873
:10282000002941F01F804F484A4F0078397001213C
:102830000297217070B14648444900904A480327E6
:102840000770002008700099029F08700399012406
:102850003C7008701A70454B1B88A3F11B02012ABB
:1028600040F23A861D2B7FF47DAE3E4A404B1278F3
:102870001A70404C77E6FEF793FC9DE63E4B1B78C2
:10288000002B3FF4A6AE2B68012B7FF4A2AEA2E68C
:1028900031683A4A069106983949106002220B6065
:1028A0002A60F9E61E49DFF8E8E0097800293FF4DC
:1028B00046AF9EF8000081423FF441AF03984B2899
:1028C00040F3F1871833802BB8F80000A8BF8023AD
:1028D00098423FF434AF2B4803800448012303702F
:1028E0002DE700BF3E9EFF1F149DFF1F9C9CFF1FF6
:1028F000449DFF1F28A0FF1FAC9CFF1F329DFF1FA0
:10290000C09CFF1FA89EFF1FE09CFF1FA49CFF1FF1
:10291000249FFF1F849CFF1F1A9FFF1FF49CFF1F13
:102920001B9FFF1F989EFF1F569EFF1F529EFF1F5B
:10293000D09CFF1F499EFF1F9889FF1F5C9EFF1FB1
:10294000C69CFF1F749CFF1F3C9FFF1FA09EFF1F84
:10295000F29EFF1F469DFF1F3D9FFF1F399FFF1FD8
:10296000759CFF1F909EFF1F8C89FF1FDE9EFF1F1F
:10297000929CFF1F6C9EFF1FE49EFF1F049DFF1F84
:10298000689EFF1FE09EFF1F5A9EFF1FFC9CFF1FBB
:10299000F59CFF1F029B9C45BFF6F9AE924B1B882E
:1029A000002B3FF4F4AEBBF1000F7FF4D5AE8F4B9C
:1029B0001B881BB1059B002B7FF4CEAE049B002B24
:1029C0003FF4E5AE8A4B1A78002A7FF4E0AEDFF8D8
:1029D000A09299F8004001221A70002C40F08F83D9
:1029E000844B1B78002B02F0B880834B1B78002BA4
:1029F00002F08783814B1B78002B7FF4C8AE804B9D
:102A00001B78002B3FF4C3AEB8F800307D490A3B79
:102A1000A8F800300A70BAE605F07CFA7A4B1B7809
:102A200073B97A4B1B785BB9794B1B7843B9794BF7
:102A30001B782BB9784B1B7813B903F0E7FD01E045
:102A400003F0F0FD23682B60744B1B88012B7FF48F
:102A5000CFAD734B73491A680868734DA92303FB04
:102A600002F3002BB8BF03F57F53704AB8BF3F3362
:102A70009B131178543BA0F118022A2000FB02306E
:102A80002860002900F0C08269490A68904200F37A
:102A9000748310DA674D2B78002B40F04385664B2A
:102AA0001B68D3F17F0348BF03339B100133D21A55
:102AB000904242F3B08608600246A8E2FEF7C4FEE8
:102AC0002368336069E5FDF75BFFFEF7F3FB5B4BC3
:102AD0001B88032B00F04E85594B1B88032B00F0FD
:102AE00045852368336052E5FDF796FE3B68336009
:102AF00047E5544A34681288A24204DB464B1B78EF
:102B0000002B00F07383504E504833680793504BAE
:102B1000079900681B88091A994200F2AF80002BC0
:102B200000F0AC804B4B198800293FF41BAD4A4B99
:102B30004A481B680088A342B8BF23469A4241F323
:102B40006A81474B1A60DFF82C8188F80010354FF6
:102B5000FDF762FE38687F2840F3D385414B7F380C
:102B600083FB0032C317C3EB620303EB4303A0EB09
:102B7000830073303C4B01931B883860002B40F07E
:102B8000BD86234B00931B78002B00F02684374C26
:102B90002378002B00F02184DFF8DC90DFF8C4A05C
:102BA0004FF0000B0CE003F17300C0B298F8001076
:102BB00006F0C0FC23780BF1010B5B4540F30D845C
:102BC0003B6859F8040F1844A0F17F038AFB0321E6
:102BD000DA17C2EB610202EB42027F28A3EB820309
:102BE000E1DCFDF739FDE0E7329DFF1F649EFF1F2A
:102BF000499EFF1F399FFF1F3A9FFF1F3B9FFF1FEB
:102C00003C9FFF1F9C9CFF1F469DFF1FA09EFF1F18
:102C1000F29EFF1F759CFF1FAC9CFF1FB09EFF1F05
:102C20009089FF1F2C9FFF1F249DFF1F009DFF1FEA
:102C3000349DFF1FF89EFF1FF49EFF1FB29EFF1FD3
:102C4000409EFF1F449DFF1F28A0FF1F049DFF1FE4
:102C5000309DFF1F949CFF1F689EFF1F0E9FFF1F4C
:102C6000789CFF1FABAAAA2ADC9CFF1F5489FF1F78
:102C70004A9EFF1F209DFF1F2C89FF1FBD4BBE4991
:102C80001B680888BD49A342B8BF23469A4200F397
:102C90008A82BB4C09888342A8BF0346236000296F
:102CA0007FF451AF9A42C8BF0B4640F38382801A2B
:102CB000B0F5804FAABF9B03C3EB8333013093FB76
:102CC000F0F0FDF78FFDC0F3C6100DF0CFFFAD4B58
:102CD000044618880DF0CAFFAB49074620460EF09F
:102CE00019F8014638460EF015F821460DF00AFF96
:102CF0004FF07E5104460EF0ABF9002841F0708091
:102D0000A24920460EF0C2F9002840F06F86204606
:102D10000EF0ECF9C0B2DFF8A48288F8000016E7E4
:102D20009B4BD6F800801988414553DD994B1B78A1
:102D3000002B4FD1DFF8889299F800007F2840F3EC
:102D40004E86A3F155337F3803F1004383FB0032F5
:102D5000C317C3EB620303EB4303A0EB83007330A1
:102D60008D4B01931B88C0B289F80000002B41F005
:102D700033808A4B00931B78002B00F0F584884C3D
:102D80002378002B00F0F084864FDFF820824FF08C
:102D9000000A0AE003F17300C0B206F0EFFB2378EB
:102DA0000AF1010A534540F3DF8457F8043F99F8CC
:102DB00000001844A0F17F0388FB0321DA17C2EB5F
:102DC000610202EB42027F28A3EB8203E2DCFDF703
:102DD00043FCE1E7744F38687F2800F3F281FDF788
:102DE0003BFCDFF8DC9199F80040844200F050820F
:102DF000624B1B88002B43D1614A5F4812680088F0
:102E0000914205DC8242D4BFC1EB0203C1EB000357
:102E1000411AB1F5804FA6BF9B030131C3EB833349
:102E200093FBF1F0FDF7DEFCC0F3C6100DF01EFFC2
:102E3000544B804618880DF019FF5349824640468E
:102E40000DF068FF014650460DF064FF41460DF05D
:102E500059FE4FF07E5180460EF0FAF8002840F0FF
:102E6000AE874A4940460EF011F9002840F0BB8574
:102E700040460EF03BF9C0B2DFF8408188F8000010
:102E80007F2C40F32F8449487F3C80FB0430E317BC
:102E9000C3EB600000EB4000A4EB800073303F4BBD
:102EA00000931B78C0B289F80000002B40F06983C2
:102EB0003F4B03931B78002B40F074853D4B0293EE
:102EC0001B78002B40F0A087334B0193029B1B78AB
:102ED000FBB1394B1B88012B00F0C785022B00F09A
:102EE000DF87032B01F08681042B01F08783052BFC
:102EF00001F09B84062B01F00486072B01F0AF87BD
:102F0000082B02F06680092B02F08C810A2B02F05C
:102F10007483009B1B78002B00F0B784019B1E4C30
:102F20001988002900F0378538687F2840F3268308
:102F30001E4B7F3883FB0032C317C3EB620303EBE6
:102F40004303A0EB830073303860002940F0BC8459
:102F5000009B1B78002B00F0EF81114C2378002B95
:102F600000F0EA81DFF83CA0DFF850804FF0000B62
:102F700035E000BF689EFF1F0E9FFF1F949CFF1F40
:102F8000789CFF1F1C9FFF1FCDCCCC3D0000FE4254
:102F9000449DFF1FAC9CFF1FDC9CFF1FF29EFF1F88
:102FA0005489FF1F2C89FF1F2C9FFF1FABAAAA2A41
:102FB000759CFF1F469DFF1F5C9EFF1F209DFF1FEE
:102FC000949EFF1F03F17300C0B298F8001006F042
:102FD000B1FA23780BF1010B5B4540F3AD813B68FF
:102FE0005AF8040FB04A1844A0F17F0382FB032172
:102FF000DA17C2EB610202EB42027F28A3EB8203E5
:10300000E0DCFDF729FBDFE7A84902460860A84B92
:10301000188858B3A74B256853F82040B5FBF4F344
:10302000772C04FB135300F3A180C3EBC30303EB22
:10303000031393FBF4F3A048A04C50F8230024683A
:103040009F4BA0F2FF7004FB00F000F57D3000F50F
:10305000607000EB4004C0EBC40083FB00430344FA
:10306000C017C0EBA3400B3802440A609549964B49
:103070000888198800F27C704300B3F57C6FA1F1D9
:1030800064014FEA4100B5BF9049914903FB022218
:103090005A4381FB02311144D317C3EBE123C1181A
:1030A00081F30C0128200AF027FDFFF7A1BA894C13
:1030B00089488A498A4A237003700B701370FFF79E
:1030C000CABB93424FF0000B80F288800123CDF8F9
:1030D00000B0CDF814B00493FFF701BB814B1B780F
:1030E000002B7FF454AB039B7F4A243B83F34703BD
:1030F000D9B25B20136006F0EDF999F80040032C7B
:1031000030D1DFF8308298F80030002B42F0F181A6
:10311000764F3B78002B42F0DF81724C2378002BF6
:1031200042F0CD81724B1B78002B42F0BB81714A7B
:103130001380714B1B78002B42F0E7816F4B7F228D
:103140001A8098F800306BB93B785BB923784BB99B
:103150006B4A7F210720138006F0BCF97F210B20EA
:1031600006F0B8F9674B1F68FFF711BBC3EB0313F9
:10317000D800631C90FBF3F35DE7634D2B78002BC5
:1031800040F0D081614B1B68D3F17F0348BF03330C
:1031900002EBA302013290420A60444BBFF637AF04
:1031A0001860024633E75A4B09881A6000297FF4F9
:1031B000CAAC13469842D4BFC2EB0003C2EB030370
:1031C00075E5394B7F3883FB0032C317C3EB6203CD
:1031D00003EB4303A0EB8300733002E60123CDF839
:1031E00010B0CDF800B00593FFF779BA01232B603A
:1031F000FFF7B7B9029B1B78FBB1464B1B88012B2D
:1032000000F0B584022B00F0E586032B01F07480FA
:10321000042B01F01882052B01F0A282062B01F08D
:103220006884072B01F07685082B01F01987092B9C
:1032300002F019800A2B02F07581019B1B88002B7C
:1032400000F04B83009B1B783BB9039B1B7823B991
:10325000029B1B78002B00F0C3871F4B1B78002BB1
:1032600000F04A812C490B78082B00F245812B484D
:103270003A6800682A4C0133DBB25F1E101A44F82A
:1032800027000B70274BD6F80080198889F800209A
:103290008845254E7FF766A93268244B0892089A24
:1032A000234C1A60FFF75FB9ABAAAA2A349DFF1F0F
:1032B000909CFF1F00290100FC210100C49EFF1FFC
:1032C0004D261281309FFF1F049FFF1F81DFFF816A
:1032D00083200882469DFF1FA09EFF1FF29EFF1FB6
:1032E000759CFF1F3C9FFF1FBC9CFF1F3B9FFF1F48
:1032F0003A9FFF1F3A9DFF1F3D9FFF1F949CFF1F9A
:10330000929EFF1F849CFF1FF89EFF1FF49EFF1FCD
:10331000789CFF1F5C9EFF1F5489FF1FA09CFF1F0E
:103320003089FF1F449DFF1F28A0FF1FD49FFF1F50
:103330006C9EFF1F399FFF1F039B1B78002B3FF4E0
:1033400059AF3B68A3F10C007F2840F34283A648A5
:103350008B3B80FB0320DA17C2EB600000EB4000E0
:10336000A3EB800303F17300DFF8C082C0B298F8CA
:10337000001006F0DFF8009B1B78002B3FF43AAFFB
:103380009A4C2378002B3FF435AFDFF8A4A24FF01E
:10339000000B0CE003F17300C0B298F8001006F0C7
:1033A000C9F823780BF1010B5B457FF723AF3B682E
:1033B0005AF8040F8C4A1844A0F18B0382FB0321B6
:1033C000DA17C2EB61020C3802EB42027F28A3EB52
:1033D0008203DFDCFDF740F9DEE7854B1B78002B2D
:1033E00040F081823B68834A1278002A45D0A3F1DD
:1033F0000C007F2840F3F0827B4A8B3B82FB032149
:10340000DA17C2EB610202EB4202A3EB820303F183
:103410007300C0B298F8001006F08CF8009B1B787F
:1034200053B3724C23783BB3DFF80492DFF8B8A1B2
:103430004FF0000B0BE003F17300C0B298F80010DE
:1034400006F078F823780BF1010B5B4514DD3B683F
:1034500059F8040F1844A0F18B038AFB0321DA17F3
:10346000C2EB61020C3802EB42027F28A3EB82031D
:10347000E1DCFDF7F1F8E0E73B685F4A1278FAB16A
:103480005E4A1288012A00F01784022A00F023867F
:10349000032A00F0AE87042A01F00A81052A01F010
:1034A0002A82062A01F04B83072A01F07183082A39
:1034B00001F03A86092A01F00D870A2A02F0698094
:1034C000019A1288002A00F020824D4A4D4C137058
:1034D00003232B60FFF747B8DFF8408198F80030EE
:1034E000002B40F00481484F3B78002B40F09A8439
:1034F000444C3B70FFF737B83A68C3E6DBB2184676
:10350000137006F0A5F8414B39491A46394B184655
:1035100000230B703B7013700370FFF7B1B80123E9
:10352000FFF7F0B80133DBB2022B88BF00232B700A
:103530006DE580243649374B374A09881B88126865
:103540000B44B2EB630FBFF622A9344B1B78002B60
:1035500040F01282B8F80030314AA3423FF417A974
:10356000304B148001221A70FFF711B9FDF7DCF817
:10357000FFF7B7BAFDF782F8FFF7AEBAFDF76CF8C0
:10358000E2E4294B01931B88002B53D1194B039381
:10359000194B0293154C2378002B55D0DFF89080FF
:1035A000DFF844A04FF0000B09E003F17300C0B254
:1035B00005F0E4FF23780BF1010B5B4544DD58F87F
:1035C000043F99F800001844A0F17F038AFB03210F
:1035D000DA17C2EB610202EB42027F28A3EB8203FF
:1035E000E3DCFDF739F8E2E7ABAAAA2A5489FF1F0A
:1035F000A09EFF1F759CFF1F469DFF1F5C9EFF1F27
:10360000949EFF1F6C9EFF1F929CFF1FF29EFF1F48
:10361000529EFF1F569EFF1FD09CFF1F909EFF1FB4
:10362000E09EFF1F9C9CFF1FDC9CFF1F209DFF1F37
:103630002C89FF1FBB4B0393BB4B029305F09EFFEE
:10364000009B1B78002BA5D1039B1B78002B3FF41C
:103650003DAC99F80030A3F10C007F2840F3B6810F
:10366000B2488B3B80FB0320DA17C2EB600000EB13
:103670004000A3EB800303F17300C0B205F07EFFAE
:10368000009B1B78002B00F09681A94C2378002B1F
:1036900001F05C82DFF8BC82DFF890A24FF0000BF3
:1036A0000AE003F17300C0B205F068FF23780BF164
:1036B000010B5B457FF70AAC58F8043F99F800000E
:1036C0001844A0F18B038AFB0321DA17C2EB6102D5
:1036D0000C3802EB42027F28A3EB8203E1DCFCF70B
:1036E000BBFFE0E72046FCF7B7FFFFF7D8BB914AE6
:1036F0001278002A40F08D818F4F904C3B70FEF77E
:1037000032BFFCF7A9FFFFF735BA002008708C49DB
:10371000087840B18B4900910978002900F069814F
:10372000009F002139708849097800297FF474A826
:10373000002C40F09A80002840F09780834C814F05
:1037400094F800E0774C0394774C0294754C8049D0
:103750002070754C0097087038702070BEF1000F13
:103760007FF46CA8FFF776B86E4B1B78002B42D025
:1037700099F80030A3F10C007F2840F367836B4A6F
:103780008B3B82FB0321DA17C2EB610202EB4202A0
:10379000A3EB820303F17300C0B205F0EFFE009BC0
:1037A0001B7843B3624C23782BB36A4FDFF87C81DC
:1037B0004FF0000A09E003F17300C0B205F0DEFE2D
:1037C00023780AF1010A534515DD57F8043F99F8AB
:1037D00000001844A0F18B0388FB0321DA17C2EB29
:1037E00061020C3802EB42027F28A3EB8203E2DC89
:1037F000FCF732FFE1E74C4B1B78FBB1564B1B88C3
:10380000012B00F07486022B00F07D87032B01F062
:10381000F780042B01F08281052B01F0BF83062B7A
:1038200001F0DC84072B01F0A385082B01F0118740
:10383000092B01F0A9870A2B01F08787019B1B88C0
:10384000002B00F0C482424B1B78002B40F0BA8260
:10385000424B434A1988D6F80080002001231060AB
:103860002B6015E50398002101703849097800297B
:103870003EF4F0AF2C4902910978002900F06987E5
:10388000029800210170FEF7E5BF039B1B78002B17
:103890007FF444AB029B1B78002B7FF43FAB019B72
:1038A0001988FFF741BB243B002BB8F8000040F318
:1038B000918498423EF443AF9BB22A48A8F8003066
:1038C00001230370FEF73BBFDFF89C80C0B298F87D
:1038D000001005F02FFEFFF73BBB234B387819781B
:1038E00005F028FEAEE47F21402005F0F3FD1F49DE
:1038F0000F4A3B680B600021117074E5C0B298F864
:10390000001005F017FEFFF73CB9D8B298F8001088
:1039100005F010FE3B68D8E5154BDFF858E0197844
:10392000FEF70DBF759CFF1F469DFF1FABAAAA2A7D
:103930005489FF1FE49EFF1F929CFF1F6C9EFF1F78
:103940003D9FFF1FF29EFF1F399FFF1F909EFF1F8D
:10395000A09EFF1F2C89FF1F5C9EFF1F449DFF1F21
:10396000789CFF1F9C9CFF1F209DFF1FA09CFF1F9A
:103970001B9FFF1FF59CFF1F4B2C40F33482183414
:10398000802CB8F80030BD4AA8BF8024A3427FF441
:10399000E7ADFEF7FCBE99F8000005F0EFFD2188C9
:1039A000FFF7C2BAB64B01931B88002B41F02F875B
:1039B000B44B02934DE6029B1B78002B7FF489AA3F
:1039C000039B1B78002B7FF4A9AA68E7FCF744FE51
:1039D00053E6FCF741FEC7E4FCF73EFE19E5FCF7B1
:1039E0003BFEFFF7BDB97F20FFF746BA7F20FFF708
:1039F00092B9A44FA44902974FF0000C81F800C07F
:103A0000009F02994FF0010E87F800E081F800C096
:103A100089E69E4F387802F073FE9D4B1B78002B91
:103A200000F021823B887E2B00F21D82994CDFF84A
:103A300078922268D9F80010521A0F2A40F20A82AE
:103A4000954A0133108899B23980002800F0248209
:103A5000C9B2C0B205F03EFD904F226898F8003020
:103A6000C9F800203B70FEF77EBDDFF840A299F850
:103A70000000BAF800308A4A8A4CC31A82FB031E3F
:103A8000D917C1EB6E0101EB4101A3EB810303EBFD
:103A9000430354F8233018447F2840F321857F38AE
:103AA00082FB0032C317C3EB620303EB4303A0EBBB
:103AB00083007330DFF8F8B1C0B205F05FFDBBF8EA
:103AC0000030022B7FF625AA99F80010BAF80030D2
:103AD000734ACB1A82FB030ED817C0EB6E0000EBC3
:103AE0004000A3EB800303EB430304EB830358681C
:103AF00008447F2840F362877F3882FB0032C31777
:103B0000C3EB620202EB4202A0EB82007330C0B250
:103B100005F034FDBBF80030032B7FF6FAA999F8C5
:103B20000010BAF800305E4ACB1A82FB030ED81799
:103B3000C0EB6E0000EB4000A3EB800303EB4303FC
:103B400004EB8304A06808447F2840F379817F3820
:103B500082FB0032C317C3EB620202EB4202A0EB0E
:103B600082007330C0B205F009FDFFF7D2B9DFF86B
:103B70003CA13868BAF80030494A4A4CC31A82FB63
:103B8000031ED917C1EB6E0101EB4101A3EB8103C9
:103B900003EB430354F8233018447F2840F3258473
:103BA0007F3882FB0032C317C3EB620303EB43038E
:103BB000A0EB83007330DFF8FC80DFF8F4B098F8F6
:103BC0000010C0B205F0B6FCBBF80030022B7FF647
:103BD00034AB3968BAF80030314ACB1A82FB030E95
:103BE000D817C0EB6E0000EB4000A3EB800303EBA3
:103BF000430304EB8303586808447F2840F3778627
:103C00007F3882FB0032C317C3EB620202EB420231
:103C1000A0EB82007330C0B298F8001005F08AFC67
:103C2000BBF80030032B7FF608AB3968BAF80030D8
:103C30001B4ACB1A82FB030ED817C0EB6E0000EBB9
:103C40004000A3EB800303EB430304EB8304A06871
:103C500008447F2840F304817F3882FB0032C31779
:103C6000C3EB620202EB4202A0EB8200733098F8D1
:103C70000010C0B205F05EFCFFF7DFBAE09EFF1F48
:103C8000DC9CFF1F469DFF1FA09EFF1FCC9CFF1FBB
:103C90003E9FFF1F6C9EFF1F1C9DFF1F929CFF1FDE
:103CA000ABAAAA2A04280100289FFF1F9C9EFF1F81
:103CB000B09CFF1F209DFF1FDFF80CA3B749BAF887
:103CC0000020B74C9A1A81FB020ED017C0EB6E0091
:103CD00000EB4000A2EB800202EB420254F822000B
:103CE00018447F2840F30084A0F17F0381FB032167
:103CF000DA17C2EB610000EB4000A3EB80007330E9
:103D0000DFF8C8B298F80010C0B205F013FCBBF899
:103D10000030022B50D93968BAF800309F4ACB1ACC
:103D200082FB030ED817C0EB6E0000EB4000A3EB44
:103D3000800303EB430304EB8303586808447F28A4
:103D400040F346867F3882FB0032C317C3EB620222
:103D500002EB4202A0EB82007330C0B298F8001070
:103D600005F0E8FBBBF80030032B25D93868BAF81A
:103D700000308A4AC31A82FB031ED917C1EB6E01B9
:103D800001EB4101A3EB810303EB430304EB830449
:103D9000A36818447F2856DD7F3882FB0032C317A2
:103DA000C3EB620202EB4202A0EB82007330C0B2AE
:103DB00098F8001005F0BEFB3B68FFF781BB0120BF
:103DC000FFF75AB80021402005F084FB40E599F840
:103DD000000005F0D3FB36E505F0D0FBFEF7C9BFC8
:103DE0000120FEF798BF243C002CB8F8003040F3C7
:103DF000E985A3423EF4CBACA4B26A4BA8F80040DC
:103E000001221A70FEF7C3BC674B01931B88002B7D
:103E10003FF45CA812E4654A8342A8BF03461360DE
:103E2000FEF791BE624B634C19886A2005F0ACFC2A
:103E300098F800303B70FEF796BB1446FFF785BB41
:103E4000FCF70AFC8EE6FCF707FCB0E7FCF704FC85
:103E5000A2E4584C584F98F800303B70FEF783BBF3
:103E6000FCF7FAFB03E7554B1B78002BF1D03B889E
:103E70004F4F002BEDD04F4CDFF854912268D9F80A
:103E80000010521A0F2AE5D94D4A013B108899B209
:103E9000398000287FF4DCADC8B205F0BBFBDBE560
:103EA000DFF824A199F80000BAF800303B4A454CED
:103EB000C31A82FB031ED917C1EB6E0101EB41014E
:103EC000A3EB810303EB430354F8233018447F280A
:103ED00040F312847F3882FB0032C317C3EB6203C6
:103EE00003EB4303A0EB83007330DFF8E0B0C0B214
:103EF00005F044FBBBF80030022B7FF60AA899F8C6
:103F00000010BAF80030254ACB1A82FB030ED817EE
:103F1000C0EB6E0000EB4000A3EB800303EB430318
:103F200004EB8303586808447F2840F3F3857F3807
:103F300082FB0032C317C3EB620303EB4303A0EB26
:103F400083007330C0B205F019FBBBF80030032BBF
:103F50007EF6DFAF99F80010BAF800300F4ACB1A9E
:103F600082FB030ED817C0EB6E0000EB4000A3EB02
:103F7000800303EB430304EB8304A06808447F2819
:103F80007FF75EAF7F3882FB0032C317C3EB62035B
:103F900003EB4303A0EB83007330E3E5ABAAAA2A4B
:103FA000042801009C9CFF1FDC9CFF1F789CFF1FC6
:103FB000CC9CFF1F6C9EFF1F929CFF1F3D9FFF1F0D
:103FC0001C9DFF1FF02901009C9EFF1FB09CFF1F3E
:103FD000289FFF1FDFF814A33868BAF80030C04AE2
:103FE000C04CC31A82FB031ED917C1EB6E0101EB53
:103FF0004101A3EB810303EB430354F8233018443E
:104000007F2840F344837F3882FB0032C317C3EB21
:10401000620303EB4303A0EB83007330DFF8D0822D
:10402000DFF8D0B298F80010C0B205F083FABBF800
:104030000030022B7FF601A93968BAF80030A84A8F
:10404000CB1A82FB030ED817C0EB6E0000EB4000CA
:10405000A3EB800303EB430304EB8303586808449A
:104060007F2840F368857F3882FB0032C317C3EB9B
:10407000620303EB4303A0EB83007330C0B298F8F4
:10408000001005F057FABBF80030032B7FF6D5A8D7
:104090003868BAF80030924AC31A82FB031ED91757
:1040A000C1EB6E0101EB4101A3EB810303EB430381
:1040B00004EB8304A36818447F287FF7D1AE7F38D0
:1040C00082FB0032C317C3EB620303EB4303A0EB95
:1040D00083007330CBE5DFF814A28149BAF80020E1
:1040E000804C9A1A81FB020ED017C0EB6E0000EBD9
:1040F0004000A2EB800202EB420254F82200184476
:104100007F2840F3FD82A0F17F0381FB0321DA17B2
:10411000C2EB610000EB4000A3EB80007330DFF8DE
:10412000D4B198F80010C0B205F004FABBF8003022
:10413000022B7FF641AE3968BAF80030684ACB1AD4
:1041400082FB030ED817C0EB6E0000EB4000A3EB20
:10415000800303EB430304EB8303586808447F2880
:1041600040F3E5847F3882FB0032C317C3EB620360
:1041700003EB4303A0EB83007330C0B298F8001048
:1041800005F0D8F9BBF80030032B7FF615AE386880
:10419000BAF80030524AC31A82FB031ED917C1EB8A
:1041A0006E0101EB4101A3EB810303EB430304EB3D
:1041B0008304A36818447F287FF745AE7F3882FBCD
:1041C0000032C317C3EB620303EB4303A0EB83008E
:1041D0007330ECE501283EF4B2AA0123FFF76DBB72
:1041E0004FF47A43013BFDD199F8000005F0C6F980
:1041F000FFF733B8DFF8F4A099F80000BAF8003000
:10420000374A394CC31A82FB031ED917C1EB6E0122
:1042100001EB4101A3EB810303EB430354F823308B
:1042200018447F2840F3DB817F3882FB0032C317BC
:10423000C3EB620202EB4202A0EB82007330DFF8B4
:10424000B4B0C0B205F09AF9BBF80030022B7EF68C
:1042500060AE99F80000BAF80030214AC31A82FB18
:104260000321DA17C2EB610202EB4202A3EB8203E5
:1042700003EB430304EB83035B6818447F2840F39C
:1042800028847F380C2290FBF2F302FB130073307A
:10429000C0B205F073F9BBF80030032B7EF639AEDF
:1042A00099F80000BAF800300D4AC31A82FB0321C6
:1042B000DA17C2EB610202EB4202A3EB820303EBCB
:1042C000430304EB8304A36818447F287FF7B8AD49
:1042D0007F380C2290FBF2F302FB1300733041E4B1
:1042E000ABAAAA2AF0290100802A01009C9EFF1F88
:1042F000209DFF1FB09CFF1FDFF8A8A33868BAF805
:104300000030E44AE44CC31A82FB031ED917C1EB08
:104310006E0101EB4101A3EB810303EB430354F86E
:10432000233018447F2840F35D817F3882FB0032C0
:10433000C317C3EB620202EB4202A0EB82007330B0
:10434000DFF86483DFF864B398F80010C0B205F0BA
:10435000F1F8BBF80030022B7EF66FAF3868BAF880
:104360000030CC4AC31A82FB0321DA17C2EB610288
:1043700002EB4202A3EB820303EB430304EB830350
:104380005B6818447F2840F3A1837F380C2290FBA0
:10439000F2F302FB13007330C0B298F8001005F07E
:1043A000C9F8BBF80030032B7EF647AF3868BAF87F
:1043B0000030B84AC31A82FB0321DA17C2EB61024C
:1043C00002EB4202A3EB820303EB430304EB8304FF
:1043D000A36818447F287FF743AD7F380C2290FBF9
:1043E000F2F302FB1300733041E4FCF735F9FFF7F9
:1043F000E2BBDFF8B0A2A749BAF80020A64C9A1A8F
:1044000081FB020ED017C0EB6E0000EB4000A2EB68
:10441000800202EB420254F8220018447F2840F345
:10442000E480A0F17F0381FB0321DA17C2EB610175
:1044300001EB4101A3EB81007330DFF870B298F813
:104440000010C0B205F076F8BBF80030022B7FF602
:10445000B3AC3868BAF800308E4AC31A82FB032125
:10446000DA17C2EB610202EB4202A3EB820303EB19
:10447000430304EB83035B6818447F2840F33683CF
:104480007F380C2290FBF2F302FB13007330C0B2B2
:1044900098F8001005F04EF8BBF80030032B7FF6BB
:1044A0008BAC3868BAF800307A4AC31A82FB032111
:1044B000DA17C2EB610202EB4202A3EB820303EBC9
:1044C000430304EB8304A36818447F287FF7BBAC45
:1044D0007F380C2290FBF2F302FB1300733066E48A
:1044E000FCF7BAF8FFF7E6BAFCF7B6F808E4DFF82D
:1044F000B4A199F80000BAF80030664A674CC31AB4
:1045000082FB0317D917C1EB670101EB4101A3EB54
:10451000810303EB430354F8233018447F286ADDFA
:104520007F3882FB0032C317C3EB620202EB420208
:10453000A0EB82007330DFF874B1C0B205F01EF852
:10454000BBF80030022B7FF679A999F80000BAF881
:104550000030504AC31A82FB0321DA17C2EB610212
:1045600002EB4202A3EB820303EB430304EB83035E
:104570005B6818447F2840F3B6827F380C2290FB9A
:10458000F2F302FB13007330C0B204F0F7FFBBF884
:104590000030032B7FF652A999F80000BAF80030DA
:1045A0003C4AC31A82FB0321DA17C2EB610202EB19
:1045B0004202A3EB820303EB430304EB8304A368EF
:1045C00018447F2814DD7F380C2290FBF2F302FBA5
:1045D00013007330C0B204F0D1FFFFF72FB9FCF71E
:1045E0003BF82CE6FCF738F8AAE6FCF735F824E7A8
:1045F000FCF732F8EEE7FCF72FF89CE7DFF8A4A011
:1046000099F80000BAF80030224A254CC31A82FB00
:10461000031ED917C1EB6E0101EB4101A3EB81032E
:1046200003EB430354F8233018447F28D7DD7F3849
:1046300082FB0032C317C3EB620303EB4303A0EB1F
:1046400083007330FBE5DFF85CA03868BAF800300F
:10465000104A134CC31A82FB031ED917C1EB6E011B
:1046600001EB4101A3EB810303EB430354F8233037
:1046700018447F28B6DD7F3882FB0032C317C3EBB6
:10468000620303EB4303A0EB8300733058E6FBF7B0
:10469000E3FFC3E4ABAAAA2A802A01000428010090
:1046A000702401009C9EFF1F209DFF1FB09CFF1FD8
:1046B000DFF840A3C849BAF80020C84C9A1A81FB19
:1046C000020ED017C0EB6E0000EB4000A2EB8002A0
:1046D00002EB420254F8220018447F2885DDA0F145
:1046E0007F0381FB0321DA17C2EB610000EB40007E
:1046F000A3EB80007330A0E6FBF7AEFFFFF7F5BB3E
:10470000FBF7AAFF0BE5DFF8ECA299F80000BAF876
:104710000030B14AB24CC31A82FB0317D917C1EB60
:10472000670101EB4101A3EB810303EB430354F861
:10473000233018447F287FF75EAF7F3882FB00323A
:10474000C317C3EB620303EB4303A0EB8300733097
:10475000F1E6A4480090A448A4490390FEF76EB87F
:10476000DFF890A23868BAF800309B4AA04CC31A10
:1047700082FB0321DA17C2EB610202EB4202A3EBD8
:10478000820303EB430354F8233018447F2840F39B
:10479000A7817F380C2290FBF2F302FB13007330E9
:1047A000DFF85482DFF854B298F80010C0B204F079
:1047B000C1FEBBF80030022B1AD93868BAF80030B5
:1047C0000C22C11A91FBF2F302FB131302FB034309
:1047D0005B6818447F2840F390847F3890FBF2F3A5
:1047E00002FB13007330C0B298F8001004F0A2FE70
:1047F000BBF80030032B7EF620ADBAF800303868E5
:104800000C22C11A91FBF2F302FB131302FB0344C7
:10481000A36818447F287FF723AB7F3890FBF2F31F
:1048200002FB13007330FFF722BADFF8C8A199F832
:104830000000BAF80030684A6D4CC31A82FB0321AD
:10484000DA17C2EB610202EB4202A3EB820303EB35
:10485000430354F8233018447F2840F33E817F38C7
:104860000C2290FBF2F302FB13007330DFF88CB1E3
:10487000C0B204F083FEBBF80030022B19D999F8BE
:104880000000BAF800300C22C11A91FBF2F302FBCF
:10489000131302FB03435B6818447F2840F326840C
:1048A0007F3890FBF2F302FB13007330C0B204F0C8
:1048B00065FEBBF80030032B7EF62BABBAF8003058
:1048C00099F800000C22C11A91FBF2F302FB1313BA
:1048D00002FB0344A36818447F287FF7B1AA7F38FE
:1048E00090FBF2F302FB13007330FFF73BB9FBF7C9
:1048F000B3FEFFF790B9DFF8FCA03749BAF8002003
:104900003B4C9A1A81FB0210D117C1EB600101EBFD
:104910004101A2EB810202EB420254F8220018444A
:104920007F2840F3D080A0F17F030C2093FBF0F2AE
:1049300000FB12307330DFF8C4B098F80010C0B23A
:1049400004F0F8FDBBF80030022B1AD93868BAF829
:1049500000300C22C11A91FBF2F302FB131302FB8D
:1049600003435B6818447F2840F3C4837F3890FB7F
:10497000F2F302FB13007330C0B298F8001004F099
:10498000D9FDBBF80030032B7FF616AABAF8003029
:1049900038680C22C11A91FBF2F302FB131302FBDD
:1049A0000344A36818447F287FF74DAA7F3890FB03
:1049B000F2F302FB13007330FFF7F9B9FBF74CFE7B
:1049C000FFF7A5B8012B3DF4E2AE0124FFF715BABD
:1049D000FBF742FEFFF7C1B9ABAAAA2A7024010077
:1049E000F0290100F29EFF1F759CFF1FA09EFF1F74
:1049F000042D01009C9EFF1F209DFF1FB09CFF1FE8
:104A0000DFF800A399F80000BAF80030B34AB44CBC
:104A1000C31A82FB0321DA17C2EB610202EB4202E6
:104A2000A3EB820303EB430354F8233018447F289D
:104A300046DD7F380C2290FBF2F302FB130073304B
:104A4000DFF8CCB2C0B204F099FDBBF80030022B05
:104A500019D999F80000BAF800300C22C11A91FB5C
:104A6000F2F302FB131302FB03435B6818447F2835
:104A700040F38B807F3890FBF2F302FB130073301E
:104A8000C0B204F07BFDBBF80030032B7EF6D6AE3F
:104A9000BAF8003099F800000C22C11A91FBF2F329
:104AA00002FB131302FB0344A36818447F287FF71B
:104AB0009FAD7F3890FBF2F302FB1300733089E562
:104AC000FBF7CAFDBCE7FBF7C7FD34E7FBF7C4FD06
:104AD00062E4FBF7C1FDFFF7DBBBFBF7BDFDC5E6FD
:104AE000FBF7BAFD5CE6FBF7B7FD4DE5FBF7B4FD60
:104AF000CDE4DFF810A23868BAF80030774A794C74
:104B000035E6DFF800A299F80000BAF80030734AE1
:104B1000744C92E6FBF7A0FDFFF714BADFF8E4A1AE
:104B200099F80000BAF800306C4A6F4C70E7FBF758
:104B300093FDFFF722BBFBF78FFDFFF79FBADFF86E
:104B4000C4A16649BAF80020664CDAE6029B1B78DD
:104B5000002B7EF4BEA9FEF7E1B9644B1B78002B55
:104B600000F02983624B1B78002B7DF410AE614B63
:104B70001B78002B3DF40BAEB8F800305E490A33C9
:104B8000A8F800300A70FDF702BEFBF765FD77E775
:104B90005A4C2288002A00F02C835949DFF870B162
:104BA0000988BBF800000331884227DD5548564983
:104BB0000088B1F800E0DFF854C1181A0C2190FB0E
:104BC000F1F901FB19004FF0900909FB0EFE01FB02
:104BD00000E06FF00B0E5CF8000003440EFB0230A7
:104BE0007F2840F332857F3890FBF1F301FB1300FF
:104BF0007330C0B298F8001004F09CFCBBF80020A1
:104C000023881344022B23DD3E4B3F4A38681B8820
:104C1000B2F800C0DFF8F4E0C31A0C2193FBF1F204
:104C200001FB1232902303FB0CF301FB02337344AC
:104C30005B6818447F2840F362857F3890FBF1F36E
:104C400001FB13007330C0B298F8001004F072FC3E
:104C5000BBF8002023881344032B23DD294B2A4A69
:104C600038681B88B2F800C0DFF8A0E0C31A0C2136
:104C700093FBF1F201FB1232902303FB0CF301FBD7
:104C8000023373449B6818447F2840F353857F3870
:104C900090FBF1F301FB13007330C0B298F80010E1
:104CA00004F048FCBBF8002023881344042B7FF752
:104CB00083A8134B1B88012B7FF47EA83A68A2F1CE
:104CC0000C007F287FF7BFA88B3A0C2092FBF0F3F3
:104CD00000FB13207330FFF76AB800BFABAAAA2A03
:104CE000802A0100AC2B0100702401003A9FFF1FB5
:104CF0003B9FFF1F3C9FFF1F9C9CFF1F289DFF1F8A
:104D0000CA9CFF1F9C9EFF1F4C9EFF1F0025010099
:104D1000B09CFF1FC74C2388002B40F06D82DFF84A
:104D20003CB3C549C54A0988D7F80080B2F800E00D
:104D3000C348C1EB080C0C229CFBF2F102FB11C131
:104D40004FF0900C0CFB0EFE02FB01E16FF00B0E1E
:104D5000405880440EFB03807F2840F37284A0F10A
:104D60007F0393FBF2F002FB10307330B54BC0B2FF
:104D7000197804F0DFFBBBF8002023881344022BD2
:104D800023DDAD4AAD4B11883868B3F800C0DFF8B9
:104D9000B0E2411A0C2291FBF2F302FB13119023B3
:104DA00003FB0CF302FB013373445B6818447F2858
:104DB00040F30D857F3890FBF2F302FB1300733054
:104DC000A04BC0B2197804F0B5FBBBF800202388D3
:104DD0001344032B23DD984A984B11883868B3F8A5
:104DE00000C0DFF85CE2411A0C2291FBF2F302FBF7
:104DF0001311902303FB0CF302FB013373449B68F4
:104E000018447F2840F39D847F3890FBF2F302FB27
:104E1000130073308B4BC0B2197804F08BFBBBF8D6
:104E2000002023881344042B7EF707AA864B1B8897
:104E3000012B7EF402AA3A68A2F10C007F2840F30D
:104E4000D5818B3A0C2092FBF0F300FB13207330DA
:104E50007C4BC0B2197804F06DFBFEF7EEB9754CCF
:104E60002388002B40F0D381DFF8F0B17249734AF8
:104E7000098899F80000B2F800E0DFF8C481C1EBBE
:104E8000000C0C229CFBF2F102FB11C14FF0900CC4
:104E90000CFB0EFE02FB01E16FF00B0E58F8011047
:104EA00008440EFB03007F2840F3C883A0F17F0372
:104EB00093FBF2F002FB10307330C0B204F05EFBE3
:104EC000BBF8002023881344022B22DD5A4A5B4B97
:104ED000118899F80000B3F800C0DFF864E1411AC6
:104EE0000C2291FBF2F302FB1311902303FB0CF352
:104EF00002FB013373445B6818447F2840F36B84E2
:104F00007F3890FBF2F302FB13007330C0B204F061
:104F100035FBBBF8002023881344032B22DD464ACF
:104F2000464B118899F80000B3F800C0DFF810E193
:104F3000411A0C2291FBF2F302FB1311902303FBA5
:104F40000CF302FB013373449B6818447F2840F341
:104F5000F5837F3890FBF2F302FB13007330C0B28D
:104F600004F00CFBBBF8002023881344042B7DF7CE
:104F7000D0AF354B1B88012B7DF4CBAF99F80020C7
:104F8000A2F10C007F287EF75BAF8B3A0C2092FBDE
:104F9000F0F300FB13207330FEF7E4BDDFF898A0B8
:104FA00099F80000BAF80030284CC11A0C2291FB85
:104FB000F2F302FB131302FB03F3E35818447F28B8
:104FC0007FF77EAD7F3890FBF2F302FB1300733066
:104FD00036E51F4B1B88182B12D099F8002013447C
:104FE000A3F118007F2840F3A2830C20973B93FB8A
:104FF000F0F200FB123303F17300C0B204F0BEFA0A
:10500000144A154B127833F81230182B3DF481AF47
:1050100099F800201344A3F118007F287EF710AF01
:105020000C20973B93FBF0F200FB123303F173006B
:10503000FEF798BD289DFF1F9C9EFF1F4C9EFF1FE3
:1050400000250100209DFF1FCA9CFF1F042D0100A9
:10505000B89CFF1F8C89FF1FB89EFF1FB09CFF1FCD
:10506000B64B1A88182A13D03B681344A3F11800D2
:105070007F2840F34B830C20973B93FBF0F200FB1F
:10508000123303F17300AE4BC0B2197804F052FA38
:10509000AC4BAD491A78022A94BF013200221A7033
:1050A0001A7831F81200182810D10424022A02F1CB
:1050B0000100C2B288BF002231F81200182804D1C2
:1050C000013CF3D11A70FEF7B8B81A703B6803447C
:1050D000A3F118007F2840F389800C20973B93FBB5
:1050E000F0F200FB123303F17300B1E6FBF7B4FA00
:1050F000FFF7DCBBFBF7B0FA3EE4FBF7ADFAFFF7D6
:1051000072BB924B1B78002B7DF441AB904B1B780C
:10511000002B3DF43CABB8F800308E49013BA8F8B9
:1051200000300A70FDF733BB844A1288182A12D067
:105130001344A3F118007F2840F3E5820C20973B2D
:1051400093FBF0F200FB123303F17300C0B298F846
:10515000001004F0EFF97B4B7B491A78022A94BFC8
:10516000013200221A701A7831F81200182811D171
:105170000424022A02F10100C2B288BF002231F8E1
:105180001200182805D1013CF3D11A703B68FEF7D4
:1051900097B91A703B680344A3F118007F287EF783
:1051A00052AE0C20973B93FBF0F200FB123303F15D
:1051B0007300FEF7FCBD654B1B78002B7DF48EAFB2
:1051C000634B1B78002B3DF4E2AAB8F8003061492C
:1051D0000133A8F800300A70FDF7D9BADFF888A1CA
:1051E00099F80000BAF800305B4CDEE6FBF734FAC1
:1051F0002EE6DFF878B1D9E4584ADFF870B11288AA
:10520000BBF80010033291427FF7B5AD89E5534AF0
:10521000DFF858B11288BBF80010033291427FF7D3
:105220004FAE23E64E4B1B88182B12D099F8002066
:105230001344A3F118007F2840F3C6820C20973B4B
:1052400093FBF0F200FB123303F17300C0B204F0E1
:1052500095F93C4A434B127833F81230182B7FF4FF
:10526000D7AEFDF756BE3E4B1A88182A13D03B68BE
:105270001344A3F118007F2840F33E820C20973B93
:1052800093FBF0F200FB123303F173002C4BC0B21E
:10529000197804F04FF92B4B32491A78022A94BF3F
:1052A000013200221A701A7831F8120018287FF49F
:1052B0000DAF0424022A02F1010294BFD2B20022EF
:1052C00031F8120018287FF400AF013CF2D11A70B7
:1052D000FDF7B3BF224A1288182A12D01344A3F153
:1052E00018007F2840F3E6810C20973B93FBF0F2F7
:1052F00000FB123303F17300C0B298F8001004F001
:1053000019F9104B17491A78022A94BF013200226A
:105310001A701A7831F8120018287FF43BAF042471
:10532000022A02F1010294BFD2B2002231F8120027
:1053300018287FF42EAF013CF2D126E7B89CFF1F5E
:10534000209DFF1F8C89FF1FB89EFF1F3B9FFF1FE3
:105350003C9FFF1F9C9CFF1FAC2B0100CA9CFF1FA2
:10536000C29CFF1F2C9EFF1F9C9EFF1FB09CFF1F17
:10537000D24C2388002B40F0CF81DFF878B3D0499E
:1053800099F80000CF4A09881788DFF83CE3411AF2
:105390000C2291FBF2FC02FB1C114FF0900C0CFB59
:1053A00007F702FB01716FF00B075EF80110014473
:1053B00007FB03107F2840F3AC817F3890FBF2F3AA
:1053C00002FB13007330C0B204F0D8F8BBF8002021
:1053D00023881344022B21DDB94BBA4A99F8000007
:1053E0001B88B2F800E0B84FC31A0C2193FBF1F20E
:1053F00001FB1232902303FB0EF301FB02333B440B
:105400005B6818447F2840F3F3817F3890FBF1F309
:1054100001FB13007330C0B204F0B0F8BBF80020F9
:1054200023881344032B21DDA54BA64A99F80000DD
:105430001B88B2F800E0A44FC31A0C2193FBF1F2D1
:1054400001FB1232902303FB0EF301FB02333B44BA
:105450009B6818447F2840F3D7817F3890FBF1F395
:1054600001FB13007330C0B204F088F8BBF80020D1
:1054700023881344042B7EF7E1A9944B1B88012B4E
:105480007EF4DCA999F80020A2F10C007F287FF7B8
:10549000AFA88B3A0C2092FBF0F300FB1320733083
:1054A000FFF798B88A4B01227F2107201A8004F069
:1054B00011F87F210B2004F00DF8FDF73ABE854B63
:1054C00004227F2107201A8004F004F800210B2019
:1054D00004F000F8FDF726BE7E4B02227F21072054
:1054E0001A8003F0F7FF7F210B2003F0F3FFFDF795
:1054F00014BE784B002107201C8003F0EBFF7F21B6
:105500000B2003F0E7FFFDF703BE734B00227F2162
:1055100007201A8003F0DEFF7F210B2003F0DAFF63
:10552000FDF70FBE6D4B1A88182A13D03B68134441
:10553000A3F118007F2840F364810C20973B93FB74
:10554000F0F200FB123303F17300654BC0B219781F
:1055500003F0F0FF634B64491A78022A94BF0132CA
:1055600000221A701A7831F8120018287FF4AEADB4
:105570000424022A02F1010294BFD2B2002231F8BF
:10558000120018287FF4A1AD013CF2D11A70FDF78A
:1055900054BE524A1288182A12D01344A3F118009C
:1055A0007F2840F322810C20973B93FBF0F200FB15
:1055B000123303F17300C0B298F8001003F0BAFF81
:1055C000484B49491A78022A94BF013200221A70C6
:1055D0001A7831F8120018287FF4DCAD0424022A6E
:1055E00002F1010294BFD2B2002231F81200182851
:1055F0007FF4CFAD013CF2D1C7E5384B1B88182BA7
:1056000012D099F800201344A3F118007F2840F32A
:10561000E9800C20973B93FBF0F200FB123303F17F
:105620007300C0B203F0AAFF2E4A2F4B127833F852
:105630001230182B7FF4ECACFDF76BBCFBF70CF8C9
:105640003BE4FBF709F8FFF791BBFBF705F8FFF721
:10565000D0BA264B1B88182B12D099F8002013447F
:10566000A3F118007F2840F3C6800C20973B93FBE2
:10567000F0F200FB123303F17300C0B203F07EFFBF
:10568000184A1B4B127833F81230182B3EF4D6A868
:1056900099F800201344A3F118007F287EF7A8AFE3
:1056A0000C20973B93FBF0F200FB123303F17300E5
:1056B000FEF790BFFAF7D0FF1EE600BF289DFF1F40
:1056C0009C9EFF1F4C9EFF1F00250100CA9CFF1FD0
:1056D0003A9DFF1F929EFF1F949CFF1FC49CFF1FBB
:1056E000209DFF1F8C89FF1F349EFF1FB89CFF1F4A
:1056F000B89EFF1FB09CFF1FFAF7AEFFC6E5FAF792
:10570000ABFFFFF7A0BAFAF7A7FF1FE5FAF7A4FF70
:10571000B9E4FAF7A1FF56E6404ADFF81CB1128857
:10572000BBF80010033291427FF750AE27E6FAF73C
:1057300093FF62E4FAF790FFFFF7AFBAFAF78CFF36
:105740000DE4FAF789FFFFF765BB354B1B88182B73
:1057500011D099F800201344A3F118007F284DDDE3
:105760000C20973B93FBF0F200FB123303F1730024
:10577000C0B203F003FF2B4A2B4B127833F81230E0
:10578000182B85D1FEF75AB8284B1B88182B11D03F
:1057900099F800201344A3F118007F281FDD0C2086
:1057A000973B93FBF0F200FB123303F17300C0B29E
:1057B00003F0E4FE1B4A1E4B127833F81230182B0C
:1057C0007FF466AFFEF73AB8FAF746FF3EE5FAF720
:1057D00043FFFFF7F5BAFAF73FFFFFF797BBFAF77A
:1057E0003BFFE4E7FAF738FF1BE7FAF735FFE2E69D
:1057F000FAF732FF0FE6FAF72FFF3EE7FAF72CFF32
:10580000B6E7FAF729FFA0E6FAF726FF2BE6094BE1
:105810000293FDF713BF0A60FDF7F9BBCA9CFF1F97
:10582000C49CFF1F8C89FF1F349EFF1FC29CFF1F5B
:105830002C9EFF1F469DFF1FB09CFF1F38B507F031
:1058400071FE0B4805F0A8FD00234FF07E520121A8
:105850000848FAF70BFE084B084A0949802400253E
:105860001C7118461D60BDE838400BF05FBC00BFDE
:10587000389DFF1F709EFF1FFC9EFF1F1C89FF1F8E
:10588000FD05000010B50446A4206368198803F0E4
:105890007BFFE368A6201988BDE8104003F074BFC1
:1058A00043682A20198803F06FBF00BF10B5044673
:1058B00022206368198803F067FFE36824201988B1
:1058C000BDE8104003F060BF10B504460A206368CD
:1058D000198803F059FFE3680C201988BDE81040CF
:1058E00003F052BF10B5044606206368198803F020
:1058F0004BFFE36808201988BDE8104003F044BF5F
:1059000010B5044602206368198803F03DFFE36880
:1059100004201988BDE8104003F036BF70B50E4C66
:1059200084B01225042201230646039002932046E8
:105930008DE824001423102106F032FF06220923EB
:10594000029303960195204600921423102106F03D
:1059500027FF04B070BD00BF709FFF1F70B5AE4C35
:10596000B4F90030032B00F0E880002B4DD0022B5F
:105970006CD0052B00F09880012B00F0C080042B28
:1059800000D070BD00244FF4AF75E1B2A34805F01C
:105990006BFD01348542A8BF05460C2CF5D10120D2
:1059A00008F040FE0446002008F03CFE323CA0F126
:1059B00032039B496FF4957000FB03F300FB04F086
:1059C00081FB034281FB0041DB17C017C3EB62235D
:1059D000C0EB612003F5AF7200F5AF739342A8BF2F
:1059E00013469D42A8BF1D46A5F11401312900F3BD
:1059F000E28040F26C7332218A488B4A0180BDE814
:105A000070402A20136003F0BFBE0E2007F0EEFCAA
:105A100040F6FF71C8308842A8BF084620EAE0700F
:105A200000F2DC5283B28A42804D814EA8BF0A4602
:105A30000220194633802A8003F0A6FE298804201C
:105A400003F0A2FEB4F90030022B92D1172008F027
:105A5000E9FD0546162008F0E5FDA842B8BF284636
:105A600000F1C801B1F5FA7FC0F2BF80B1F57A6FDD
:105A7000A8BF4FF47A6101F54873B3F57A6FA8BFF8
:105A80004FF47A639BB289B26A4A6B4D11800A2047
:105A90002B8003F079FE29880C2003F075FEB4F901
:105AA0000030052B7FF468AF0F2008F0BBFDC0F578
:105AB0003F630433B3F5AF6FC0F28F80B3F5FA6F75
:105AC000A8BF4FF4FA6399B25C4BC0F54360B0F5E0
:105AD000AF6F19807EDBB0F5FA6FA8BF4FF4FA60A4
:105AE00083B2574DA4202B8003F04EFE2988A620B8
:105AF00003F04AFEB4F90030012B7FF440AF0B20D5
:105B000008F090F900283CD0112008F08BFD00F13E
:105B1000C801B1F52F7F3CDB41F25C23994278DC70
:105B2000484A00F5487089B2B0F52F7F11806DDBCF
:105B30008342A8BF03469BB231E0102008F072FDFB
:105B4000C830B0F5FA7F4BDBB0F57A6F0146A8BFDD
:105B50004FF47A6101F51673B3F57A6FA8BF4FF46D
:105B60007A639BB289B2384A384D118022202B804B
:105B700003F00AFE2988242003F006FEB4F9003061
:105B8000F3E6152007F032FC00F59671B1F52F7F92
:105B900030DA40F214534FF42F712A4A11802C4D01
:105BA00006202B8003F0F0FD2988082003F0ECFD8F
:105BB000B4F90030E3E640F23A72A5F5B975254B29
:105BC00002FB05F583FB0523ED17A5EB631389B2F3
:105BD000323311E74FF4AF6383E74FF4AF6173E7FC
:105BE00040F24C434FF4FA71BDE740F214534FF4C6
:105BF000FA7149E741F25C2399420ADC114A00F547
:105C0000617089B2B0F52F7F118091DA4FF42F7354
:105C1000C5E71946C1E700BF489FFF1F389DFF1F1A
:105C200067BBCF46069FFF1F9889FF1F0E9FFF1F70
:105C3000449DFF1FA89EFF1FC09CFF1F489DFF1F84
:105C4000C89EFF1FFE9CFF1F569EFF1F529EFF1FF8
:105C5000DC9EFF1FB5814E1B2DE9F041224D82B025
:105C6000012602B284B200922846019678231921B7
:105C700006F0DCFC04F10C0212B28DE84400284668
:105C8000A7197823192104F1020806F0CFFC3FB2CE
:105C90000FFA88F819233A46284619460196CDF896
:105CA000008006F0C3FC78233A4628461946CDF812
:105CB0000080019604F10A070B3406F0B7FC3FB2EE
:105CC00024B278233A46284619468DE8500006F05B
:105CD000ADFC192300943A4601962846194606F071
:105CE000A5FC02B0BDE8F081709FFF1F30B583B006
:105CF00000230C4605B2009326225B231C210C488E
:105D000006F0E4F9294601232622094805F0EEFCB5
:105D1000002C24B205DB214601232622044805F08D
:105D2000E5FC044A044B15801C8003B030BD00BF65
:105D3000709FFF1FAE89FF1FB089FF1F70B5A54C74
:105D4000237882B01BB1A44B4FF6FF721A80A34B8D
:105D5000B3F90030C3B9A24A9F4B1068B3F90020D1
:105D600080F30C005B2303FB00F000131C30824225
:105D70004AD04FF0FF31FFF7B9FF9A4806F00AFA10
:105D80000023237002B070BD012B1BD0022B5AD010
:105D9000032B3FD0042B00F09A80052BF0D10F206D
:105DA00008F040FCC0F53B600830B0F5AF6F48DB51
:105DB000B0F5FA6FA8BF4FF4FA60A0F5AF625B23AD
:105DC000894835E0894B1B78002B70D0152007F0EF
:105DD0000DFB874B1860B0F52F7F32DB41F25C235F
:105DE0009842A8BF1846A0F52F735B22814802FB9A
:105DF00003F380FB0320DB17C3EBA0201C30764BA2
:105E0000B3F900308342B4D17B4BB3F90030013396
:105E1000AFD1B5E7794B1B68B3F5FA7F11DBB3F56A
:105E20007A6FA8BF4FF47A637548A3F5FA725B23C3
:105E300003FB02F380FB0320DB17C3EB20201C30A5
:105E4000DDE71C20DBE76F4B1B68B3F5FA7F36DB21
:105E5000B3F57A6FA8BF4FF47A63A3F5FA72684876
:105E60005B2303FB02F380FB0320DB17C3EB202043
:105E70001C30654B1B68B3F5FA7F1EDBB3F57A6FF8
:105E8000A8BF4FF47A63A3F5FA725D495B2303FB65
:105E900002F381FB0321DB17C3EB21211C314E4BA5
:105EA000B3F9003083420CD0FFF720FF65E71120E3
:105EB00008F0B8FB4E4B18608DE71C21EFE71C2063
:105EC000D7E74D4BB3F900308B42EDD158E727228D
:105ED00000258DE8240076231C2142484B4E06F015
:105EE000A5FB16E0B0F5AF7FA8BF4FF4AF70323816
:105EF00003FB00F386FB0321DB17C3EB61111C31AD
:105F000009B201231D442722364805F0EFFB0C2D72
:105F100009D0E9B23E4805F0A7FA31284FF05B03FB
:105F2000E0DC1C21EDE7012008F07CFB6FF49573A9
:105F30003238384A03FB00F082FB0023C017C0EB65
:105F4000632303F5AF73312B42DDB3F5AF7FA8BFF9
:105F50004FF4AF735B22323B2C4D02FB03F385FB06
:105F60000325DB17C3EB65151C35002008F05AFB31
:105F70006FF495733238274A03FB00F082FB00234D
:105F8000C017C0EB632303F5AF73312B1EDDB3F5F0
:105F9000AF7FA8BF4FF4AF735B22323B1B4902FBBC
:105FA00003F381FB0321DB17C3EB61111C310A4BA7
:105FB000B3F90030AB4201D0284675E70E4BB3F978
:105FC00000308B423FF4D9AE28466DE71C21EEE746
:105FD0001C25CAE7429FFF1FAE89FF1F489FFF1F76
:105FE000AC9EFF1F709FFF1F37800B6DC29EFF1F6F
:105FF000809CFF1FD3058541B089FF1FD09CFF1FE8
:10600000011FB812E09CFF1FA49CFF1F4B48371BC9
:10601000389DFF1F67BBCF462DE9F041044682B093
:1060200071482768E56805F0A9FF1120FFF714FE05
:10603000012619234FF02808194624226A480196A0
:10604000CDF8008006F0F2FA78231946242266483B
:106050000196CDF8008006F0E9FA3146624806F074
:106060007BFE02221921604806F072FE38460BF0D2
:1060700027FE394602465C4807F004F85A4807F004
:1060800017F814220021584806F062FE03225749EF
:10609000554806F0F7FF544807F00AF8232200217C
:1060A000514806F055FE032251494F4806F0EAFFD9
:1060B0004D4806F0FDFF7DB12F20FFF7CDFD3222C8
:1060C0000021494806F044FE03224A49464806F0AA
:1060D000D9FF454806F0ECFF0123474A18461370E4
:1060E000FFF71CFC2189638962685B1A5C2B1288AC
:1060F00054DD521A02EB4202C2EB4212013392FB10
:10610000F3F31B333D4A3848138001261A221BB291
:106110008DE844001946142206F088FA002D4FD06D
:10612000218A638AE2685B1A5C2B12883EDC511A72
:106130005C2202FB01F292FBF3F31B33304A2A4844
:10614000138001251BB2382219468DE82400322223
:1061500006F06CFA4023002209218DE8060022484F
:10616000194606F031FA29461F4806F0F5FD0222CD
:1061700044211D4806F0ECFD63681B48198806F0B1
:10618000E7FF2A461F49184806F07CFFE3681648D7
:10619000198802B0BDE8F04106F0DABF511A5C225E
:1061A00002FB01F292FBF3F31B33ABE7521A02EB53
:1061B0004202C2EB4212334492FBF3F31B33BDE7BE
:1061C000402309212A46009107480195194606F007
:1061D000FBF93146044806F0BFFD0222682102485F
:1061E00006F0B6FD6368D2E7709FFF1FDC2D01004B
:1061F000E02D0100E42D0100E99FFF1F449FFF1FD8
:10620000469FFF1FE82D01002DE9F0471F4682B091
:106210001446002A4ED0052A0646D0F80C8000F01D
:10622000AB800B9B894A00EBC305012CB5F80AE053
:1062300029896868C1EB0E0382FB03C21A444FEA46
:10624000E373C3EBA213028851D0042C00F08D80BD
:106250000022402309218DE806007D48194606F0FA
:10626000B3F901217A4806F077FD0222B8F1000F58
:1062700000F0E1804421764806F06AFD73687448B6
:10628000198806F065FF73497148012206F0FAFE8D
:10629000F3686F48198806F05BFF6F4B022CB3F967
:1062A000001000F0A680082C00F0C280012002B08F
:1062B000BDE8F087694E6A4A33681268CB1A934288
:1062C0000D4655D9674A3B8811786148012918BFA6
:1062D000012414700A9A06321BB212B28DE814001F
:1062E0001946BDF9282006F0A1F93560DEE79BB21A
:1062F000D31A994203DC9E457146A8BF19460A9AF3
:106300000180B7F90030BDF928A0514802F1060913
:106310004FF0000E0FFA89F919465246CDF8009059
:10632000CDF804E006F082F929896A896868521A72
:1063300003885C2AA3EB010373DD03EB4303013203
:10634000C3EB431393FBF2F303F11B0213B20120DF
:106350003A80194652460190CDF800903C4806F02C
:1063600065F9404B00221A7072E712FA83F3C0E716
:10637000204602B0BDE8F08707254FF000095A23F8
:1063800023228DE820021A21314806F01DF901214F
:106390002F4806F0E1FC01212D4806F0E3FC232202
:1063A00035212B4806F0D4FC2A462F49284806F010
:1063B00069FE274806F07CFE254805F0EBFE4FF409
:1063C000FA6007F065FDFFF7C9FA5A2323221A2164
:1063D0008DE820021E4806F0F7F81D4805F0DAFEA9
:1063E0003046FFF719FE214B01221A70FFF7A6FC79
:1063F0002EE74A1C12B21A8091423FF457AF0A9A14
:10640000B7F9003012480632012412B20092194640
:106410000194BDF9282006F009F9204602B0BDE834
:10642000F0875C2101FB03F393FBF2F21B328DE753
:1064300000221A80E0E76821054806F089FC7368AD
:106440000348198806F084FE27E700BFC94216B248
:10645000709FFF1FE82D01004C9FFF1FD49FFF1F5F
:10646000E43D0100E99FFF1FEC2D0100429FFF1F4B
:106470002DE9F04F5A4E5B4DB6F900704C7855F847
:10648000277085B08146984604B10C78DFF874A176
:106490001AB99AF80030002B39D0534D00233846F2
:1064A0002B808AF80030FFF7B7FD504A504BB5F902
:1064B0000000012111704FF6FF721A8060B30128AD
:1064C0005ED0012032232246019000934946494B79
:1064D0003846FFF799FE00240346B5F90020022A4A
:1064E00039DD00222A80B6F900203D49002A3BDB35
:1064F000052AC4BF00220A80B8F1000F39D1002C50
:106500000CBF18464FF0FF3005B0BDE8F08F364D98
:10651000B5F900000028D2D1DFF8ECB0364ADBF83C
:1065200000301268C3EB0903934227D9334B1A7822
:10653000012A18BF01201870FFF7F0F90123CBF8EA
:106540000090012C2AD0042C35D0022C3AD0082CF3
:106550003ED00024C1E7C6D1FA68002AC1D0B6F9FE
:1065600000201F49002AC3DA05220A80B8F1000F73
:10657000C5D00393FFF7E2FB039BC0E70346E0E7C8
:106580004FF0000E142322468DE8084049461C4B6C
:1065900038467446FFF738FE03469EE732888AF88D
:1065A0000040013232807A6982B100243846039378
:1065B0009047039B91E732880121013A32808AF8A3
:1065C0000010F0E701222A8000248CE7144684E7BB
:1065D0007A69002129804FF0FF34002AE6D182E752
:1065E000489FFF1FB489FF1F4C9FFF1F429FFF1F43
:1065F000AE89FF1F469FFF1FE43D0100E99FFF1F7B
:10660000449FFF1F4A9FFF1FD49FFF1F01210D20A2
:1066100007F002BC00210D2007F0FEBB01460D2053
:1066200007F0FABB08B50D2007F0FCFBB0FA80F1CB
:1066300049090D20BDE8084007F0EEBB10B5002168
:1066400044080D2007F0E8FB204607F021FC0D2050
:10665000012107F0E1FB2046BDE8104007F018BC1F
:10666000214A224B10881B68984210B535DA204A1F
:106670001288141A9A42A8BF1A46B4F5157F22DA76
:10668000121A40F2532303FB02F393FBF4F105319A
:106690000A2007F031FA174B197801B3164B174946
:1066A0001B6840F2271283F3070302FB03F381FB0D
:1066B00003211944DB17C3EBA11105310920BDE803
:1066C000104007F019BA131A4FF41572611C02FB3F
:1066D00003F393FBF1F10531DAE70021D8E7092054
:1066E000BDE8104007F008BA449DFF1F789CFF1FCB
:1066F0000E9FFF1F009DFF1FF49EFF1F09040281D4
:106700007F2838B5A8BF7F200F4C4FF4167202FBCC
:1067100000F284FB02311144D2170546C2EBA111ED
:106720000A2007F0E9F97F3D4FF4967303FB05F368
:1067300084FB03211944DB17A3EBA1110920BDE859
:10674000384007F0D9B900BF09040281C368B3F922
:10675000003030B583EAE374A4EBE374002BA0B2FD
:1067600018DB012300E0134603EB8302520094423E
:10677000F9DA0A4D90FBF3F285FB03E403FB120008
:10678000DB173032D3EBA40380B201F8012BF1D137
:106790000B7030BD2D230B700131E2E76766666632
:1067A00038B5094D8224204603F008F835F8021B5D
:1067B00000B28842204601D002F0E6FF0234A4B2C3
:1067C0008A2CF0D138BD00BF349EFF1F024B8020C1
:1067D000198802F0D9BF00BFC49CFF1F38B5094D0E
:1067E0007824204602F0EAFF35F8021B00B2884206
:1067F000204601D002F0C8FF0234A4B2802CF0D1B0
:1068000038BD00BF2C9EFF1F024B7620198802F076
:10681000BBBF00BFC29CFF1F38B5094D46242046B0
:1068200002F0CCFF35F8021B00B28842204601D0AE
:1068300002F0AAFF0234A4B24E2CF0D138BD00BF42
:10684000B89EFF1F024B4420198802F09DBF00BF75
:10685000B89CFF1F024B4E20198802F095BF00BF65
:10686000DC9CFF1F024B9A20198802F08DBF00BFED
:10687000289DFF1F024B9820198802F085BF00BF9A
:10688000CA9CFF1F024B8C20198802F07DBF00BFFD
:106890004C9EFF1F024B9C20198802F075BF00BF61
:1068A000B09CFF1F024BA020198802F06DBF00BFF3
:1068B000C09EFF1F024B9620198802F065BF00BFE3
:1068C0009C9EFF1F024B8A20198802F05DBF00BF0B
:1068D0005C9EFF1F024B1020198802F055BF00BFBD
:1068E0005A9EFF1F024B2C20198802F04DBF00BF9B
:1068F000AE9CFF1F024B1E20198802F045BF00BF4F
:10690000C89CFF1FC3680E20198802F03DBF00BF5E
:10691000024B2820198802F037BF00BFB69EFF1F28
:10692000024B6220198802F02FBF00BFEC9CFF1FB2
:10693000024B6420198802F027BF00BFB09EFF1FE2
:10694000024BB420198802F01FBF00BF049FFF1F35
:10695000024BB620198802F017BF00BF309FFF1FFF
:10696000024B5A20198802F00FBF00BF889CFF1FFE
:10697000024B1620198802F007BF00BF949CFF1F2E
:10698000024B2E20198802F0FFBE00BF309DFF1F72
:10699000024B3020198802F0F7BE00BF1C9FFF1F7A
:1069A000024B9E20198802F0EFBE00BF9489FF1FA2
:1069B000024BAC20198802F0E7BE00BFB29EFF1F59
:1069C000024BAE20198802F0DFBE00BFD49CFF1F2F
:1069D000024BB020198802F0D7BE00BF409EFF1FB7
:1069E000024BB220198802F0CFBE00BFF69CFF1FF9
:1069F000024B1820198802F0C7BE00BF4A9DFF1F36
:106A0000024BA220198802F0BFBE00BFE29EFF1F0A
:106A1000024B1A20198802F0B7BE00BFE49CFF1F8A
:106A2000024B1C20198802F0AFBE00BFDE9CFF1F86
:106A3000024B6620198802F0A7BE00BFF09EFF1F20
:106A4000024B7220198802F09FBE00BF189FFF1FE3
:106A5000024B2020198802F097BE00BFEE9EFF1F58
:106A6000024B3220198802F08FBE00BFDE9EFF1F4E
:106A7000024B6820198802F087BE00BF1C9DFF1FD3
:106A8000024B6C20198802F07FBE00BF7C9CFF1F68
:106A9000024B5220198802F077BE00BF2E89FF1FDB
:106AA000024B5020198802F06FBE00BF2089FF1FE3
:106AB000024B5420198802F067BE00BFA889FF1F4F
:106AC000024B5C20198802F05FBE00BFAC89FF1F3B
:106AD000024B5E20198802F057BE00BF2C89FF1FB1
:106AE000024B5620198802F04FBE00BF1E9DFF1FAB
:106AF000244B1B880B2B43D8DFE803F00B10151A2F
:106B00001F24292E33383D06084604221E490BF067
:106B100095B9084604221D490BF090B90846042295
:106B20001B490BF08BB9084604221A490BF086B9B1
:106B30000846042218490BF081B908460422174977
:106B40000BF07CB90846042215490BF077B90846CA
:106B5000042214490BF072B90846042212490BF0C2
:106B60006DB90846042211490BF068B908460422A1
:106B70000F490BF063B9084604220E490BF05EB9C9
:106B8000704700BF9C9EFF1F48360100B4330100D0
:106B90001C32010034370100203201001C37010093
:106BA0002432010028320100DC3401002C320100C3
:106BB0005436010030320100064B074A10B41C88DD
:106BC000064B0846002C14BF11461946042210BC7F
:106BD0000BF034B9FC9CFF1F343201003832010045
:106BE000064B074A10B41C88064B0846002C14BFFD
:106BF00011461946042210BC0BF020B9329DFF1F2C
:106C00003432010038320100064B074A10B41C88A8
:106C1000064B0846002C14BF11461946042210BC2E
:106C20000BF00CB9509EFF1F3432010038320100C6
:106C3000064B074A10B41C88064B0846002C14BFAC
:106C400011461946042210BC0BF0F8B8649EFF1FD1
:106C50003432010038320100064B074A10B41C8858
:106C6000064B0846002C14BF11461946042210BCDE
:106C70000BF0E4B89E9EFF1F343201003832010051
:106C8000064B074A10B41C88064B0846002C14BF5C
:106C900011461946042210BC0BF0D0B83A9DFF1FD4
:106CA00034320100383201001B4B1B880A2B0AD8F2
:106CB000DFE803F00A0E12161A1E22262A2E0600FC
:106CC000164B186808607047154B186808607047C5
:106CD000144B186808607047134B186808607047B9
:106CE000124B186808607047114B186808607047AD
:106CF000104B1868086070470F4B186808607047A1
:106D00000E4B1868086070470D4B18680860704794
:106D10000C4B1868086070475C9EFF1F60320100D2
:106D2000383201003C32010040320100443201009F
:106D3000483201004C32010050320100543201004F
:106D4000583201005C320100F0B52B4E2B4FDFF8BA
:106D5000C4E005460FCE87B06C460FC496E803002A
:106D60003B68274A274F44F8040B40F6CC30834257
:106D7000C8BF3A46BEF800602180012E1188927883
:106D8000ADF80D108DF80F202AD032D340F6CA028C
:106D9000022E18BF00229A4226DAA3F698031A4957
:106DA0001A4AC3EB031381FB03011944DB17C3EB3E
:106DB0006123243382FB0321DA17C2EBA10202EB29
:106DC0008201A3EB4103303330328DF813308DF85C
:106DD00011206946284616220BF030F807B0F0BDA6
:106DE00040F698029A42D8DB094B1868CDF811009A
:106DF000EFE740F6FC02CEE774320100A49EFF1FCD
:106E000068320100643201003B773B986766666632
:106E10006C3201003C9EFF1FF8B5174C174E2278CC
:106E2000174D33782F888E46003218BF0122014655
:106E30007046FFF71DFB002398423370237015DB6B
:106E400014BF012000202B889F420ED040F23A72DE
:106E5000A3F5AF730B490C4C02FB03F381FB031248
:106E6000DB17A3EB621332332360F8BD074901221D
:106E700018460A702270E6E7808AFF1F5D9FFF1F99
:106E8000069FFF1FB5814E1B9889FF1FE89FFF1FBC
:106E9000014B187802F010BCD09FFF1F014B1878EF
:106EA00002F024BC8890FF1F134BB3F9003030B5BB
:106EB00083EAE374A4EBE374002BA0B218DB012394
:106EC00000E0134603EB830252009442F9DA0B4DC3
:106ED00090FBF3F285FB03E403FB1200DB17303277
:106EE000D3EBA40380B201F8012BF1D10B7030BDBC
:106EF0002D230B700131E2E78890FF1F67666666FD
:106F0000144BB3F9003070B583EAE375A5EBE37574
:106F1000002BACB21ADB012300E0034603EB830035
:106F200040008542F9DA0C4E94FBF3F086FB03E552
:106F300003FB1044DB173030D3EBA503A4B201F8F8
:106F4000010BF1D105480B70106070BD2D230B7043
:106F50000131E0E7889CFF1F676666668C3201009E
:106F6000134BB3F9003030B583EAE374A4EBE37458
:106F7000002BA0B218DB012300E0134603EB8302D1
:106F800052009442F9DA0B4D90FBF3F285FB03E4D7
:106F900003FB1200DB173032D3EBA40380B201F8FD
:106FA000012BF1D10B7030BD2D230B700131E2E7C5
:106FB0009489FF1F67666666134BB3F9003030B5DE
:106FC00083EAE374A4EBE374002BA0B218DB012383
:106FD00000E0134603EB830252009442F9DA0B4DB2
:106FE00090FBF3F285FB03E403FB1200DB17303266
:106FF000D3EBA40380B201F8012BF1D10B7030BDAB
:107000002D230B700131E2E7D49CFF1F6766666693
:10701000134BB3F9003030B583EAE374A4EBE374A7
:10702000002BA0B218DB012300E0134603EB830220
:1070300052009442F9DA0B4D90FBF3F285FB03E426
:1070400003FB1200DB173032D3EBA40380B201F84C
:10705000012BF1D10B7030BD2D230B700131E2E714
:10706000F69CFF1F67666666134BB3F9003030B5B8
:1070700083EAE374A4EBE374002BA0B218DB0123D2
:1070800000E0134603EB830252009442F9DA0B4D01
:1070900090FBF3F285FB03E403FB1200DB173032B5
:1070A000D3EBA40380B201F8012BF1D10B7030BDFA
:1070B0002D230B700131E2E7E29EFF1F67666666D3
:1070C000134BB3F9003030B583EAE374A4EBE374F7
:1070D000002BA0B218DB012300E0134603EB830270
:1070E00052009442F9DA0B4D90FBF3F285FB03E476
:1070F00003FB1200DB173032D3EBA40380B201F89C
:10710000012BF1D10B7030BD2D230B700131E2E763
:107110002E89FF1F67666666134BB3F9003030B5E2
:1071200083EAE374A4EBE374002BA0B218DB012321
:1071300000E0134603EB830252009442F9DA0B4D50
:1071400090FBF3F285FB03E403FB1200DB17303204
:10715000D3EBA40380B201F8012BF1D10B7030BD49
:107160002D230B700131E2E72089FF1F67666666F9
:10717000134BB3F9003030B583EAE374A4EBE37446
:10718000002BA0B218DB012300E0134603EB8302BF
:1071900052009442F9DA0B4D90FBF3F285FB03E4C5
:1071A00003FB1200DB173032D3EBA40380B201F8EB
:1071B000012BF1D10B7030BD2D230B700131E2E7B3
:1071C000A889FF1F67666666134BB3F9003030B5B8
:1071D00083EAE374A4EBE374002BA0B218DB012371
:1071E00000E0134603EB830252009442F9DA0B4DA0
:1071F00090FBF3F285FB03E403FB1200DB17303254
:10720000D3EBA40380B201F8012BF1D10B7030BD98
:107210002D230B700131E2E7AC89FF1F67666666BC
:10722000134BB3F9003030B583EAE374A4EBE37495
:10723000002BA0B218DB012300E0134603EB83020E
:1072400052009442F9DA0B4D90FBF3F285FB03E414
:1072500003FB1200DB173032D3EBA40380B201F83A
:10726000012BF1D10B7030BD2D230B700131E2E702
:107270002C89FF1F6766666608B5B82002F09EFA83
:10728000044B1988884204D0B820BDE8084002F0B9
:107290007BBA08BD909CFF1F08B5702002F08EFAE3
:1072A000044B1988884204D07020BDE8084002F0E1
:1072B0006BBA08BD3C9EFF1F08B5742002F07EFA31
:1072C000044B1988884204D07420BDE8084002F0BD
:1072D0005BBA08BDD49EFF1F054B1B8808460422DD
:1072E00013B904490AF0AABD03490AF0A7BD00BFBB
:1072F000DC9CFF1F94320100903201000E4B1B8872
:10730000032B17D8DFE803F0110C0702084604220C
:107310000A490AF093BD0846042209490AF08EBDC5
:107320000846042207490AF089BD08460422064996
:107330000AF084BD704700BF4C9EFF1FA0320100C1
:10734000383301009C3201009832010010B40A4B1E
:107350000A4C0A4693E8030083B0238802AC04E990
:10736000030004EB8303104653F8081C052203B006
:1073700010BC0AF063BD00BF6C2E0100B09EFF1F61
:1073800030B40A4B0A4D0C4693E8070084B02B88B2
:1073900004AD05E9070005EB8303204653F80C1CF8
:1073A000042204B030BC0AF049BD00BF742E0100B5
:1073B0003C9EFF1FF0B40C4D0C4F0E460FCD8CB011
:1073C00001AC0FC40FCD0FC495E807003B8884E8DB
:1073D00007000CAA02EB8303304653F82C1C04224E
:1073E0000CB0F0BC0AF02ABD802E0100929EFF1F57
:1073F00030B50A4B0A4D0C460FCB85B00DF1100E7F
:107400000EE90F002B880EEB8303204653F8101C67
:10741000042205B0BDE830400AF010BDBC2E0100CA
:10742000B29EFF1F30B50A4B0A4D0C460FCB85B0FC
:107430000DF1100E0EE90F002B880EEB8303204692
:1074400053F8101C042205B0BDE830400AF0F6BC29
:10745000BC2E0100409EFF1FF0B40B4D0B4F0E469B
:107460000FCD86B06C460FC495E803003B8884E8D6
:10747000030006AA02EB8303304653F8181C0422CB
:1074800006B0F0BC0AF0DABCCC2E01004A9DFF1F0A
:10749000F0B40A4D0A4F0E460FCD86B001AC0FC4B2
:1074A0002A683B88226006AA02EB8303304653F821
:1074B000141C0C2206B0F0BC0AF0C0BCE42E010083
:1074C000DE9CFF1FF0B40B4D0B4F0E460FCD86B068
:1074D0006C460FC495E803003B8884E8030006AAC5
:1074E00002EB8303304653F8181C042206B0F0BCAC
:1074F0000AF0A4BCF82E0100D49EFF1F164B1B8877
:107500000BB31BB283EAE370A0EBE370002B30B542
:1075100084B21DDB012300E0134603EB830252001B
:107520009042F9DA0D4894FBF3F280FB03E503FB8C
:107530001244DB173032D3EBA503A4B201F8012BC0
:10754000F1D10B7030BD0846042205490AF076BC23
:107550002D230B700131DDE71C9DFF1F67666666FA
:10756000A432010030B50A4B0A4D0C460FCB85B052
:107570000DF1100E0EE90F002B880EEB8303204651
:1075800053F8101C042205B0BDE830400AF056BC88
:10759000102F01007C9CFF1F054B1B881BB9054B5E
:1075A0001868086070470846042203490AF046BC80
:1075B000289DFF1F3832010034320100164B1B8812
:1075C0000BB31BB230B583EAE374A4EBE374002B76
:1075D000A0B21CDB012300E0134603EB8302520040
:1075E0009442F9DA0D4D90FBF3F285FB03E403FBC3
:1075F0001200DB173032D3EBA40380B201F8012B69
:10760000F1D10B7030BD064B1868086070472D2310
:107610000B700131DEE700BFC89CFF1F676666661E
:1076200038320100164B1B880BB31BB230B583EA0E
:10763000E374A4EBE374002BA0B21CDB012300E095
:10764000134603EB830252009442F9DA0D4D90FB8E
:10765000F3F285FB03E403FB1200DB173032D3EBBC
:10766000A40380B201F8012BF1D10B7030BD064BA1
:107670001868086070472D230B700131DEE700BFEA
:10768000909CFF1F6766666638320100164B1B88A8
:107690000BB31BB230B583EAE374A4EBE374002BA5
:1076A000A0B21CDB012300E0134603EB830252006F
:1076B0009442F9DA0D4D90FBF3F285FB03E403FBF2
:1076C0001200DB173032D3EBA40380B201F8012B98
:1076D000F1D10B7030BD064B1868086070472D2340
:1076E0000B700131DEE700BFA29EFF1F6766666672
:1076F00038320100164B1B880BB31BB230B583EA3E
:10770000E374A4EBE374002BA0B21CDB012300E0C4
:10771000134603EB830252009442F9DA0D4D90FBBD
:10772000F3F285FB03E403FB1200DB173032D3EBEB
:10773000A40380B201F8012BF1D10B7030BD064BD0
:107740001868086070472D230B700131DEE700BF19
:10775000949CFF1F67666666A8320100174B1B8862
:107760001BB31BB270B583EAE375A5EBE375002B81
:10777000ACB21EDB012300E0034603EB83004000B4
:107780008542F9DA0E4E94FBF3F086FB03E503FB2A
:107790001044DB173030D3EBA503A4B201F8010B82
:1077A000F1D108480B70106070BD074B1868086075
:1077B00070472D230B700131DCE700BF309DFF1FA8
:1077C00067666666AC32010038320100164B1B88D2
:1077D0000BB31BB230B583EAE374A4EBE374002B64
:1077E000A0B21CDB012300E0134603EB830252002E
:1077F0009442F9DA0D4D90FBF3F285FB03E403FBB1
:107800001200DB173032D3EBA40380B201F8012B56
:10781000F1D10B7030BD064B1868086070472D23FE
:107820000B700131DEE700BF1C9FFF1F67666666B5
:1078300038320100164B1B880BB31BB230B583EAFC
:10784000E374A4EBE374002BA0B21CDB012300E083
:10785000134603EB830252009442F9DA0D4D90FB7C
:10786000F3F285FB03E403FB1200DB173032D3EBAA
:10787000A40380B201F8012BF1D10B7030BD064B8F
:107880001868086070472D230B700131DEE700BFD8
:10789000F09EFF1F6766666638320100164B1B8834
:1078A0000BB31BB230B583EAE374A4EBE374002B93
:1078B000A0B21CDB012300E0134603EB830252005D
:1078C0009442F9DA0D4D90FBF3F285FB03E403FBE0
:1078D0001200DB173032D3EBA40380B201F8012B86
:1078E000F1D10B7030BD064B1868086070472D232E
:1078F0000B700131DEE700BF189FFF1F67666666E9
:1079000038320100174B1B881BB31BB270B583EADA
:10791000E375A5EBE375002BACB21EDB012300E0A1
:10792000034603EB830040008542F9DA0E4E94FBD8
:10793000F3F086FB03E503FB1044DB173030D3EB99
:10794000A503A4B201F8010BF1D108480B70106037
:1079500070BD074B1868086070472D230B7001310C
:10796000DCE700BFEE9EFF1F67666666AC32010073
:1079700038320100054B1B881BB1054B18680860A5
:107980007047044B18680860704700BF1E9DFF1FBA
:10799000C0320100BC32010070B5FAF73FFB164B54
:1079A0001B7813B1154C237833B9154B1020198867
:1079B00001F0EAFE012070BD124D134E2B78328883
:1079C000B3FA83F382F008025B09114642202B7060
:1079D000328001F0D9FE23780BB12B782BB900212E
:1079E000212006F019FA002070BD0121212006F0A7
:1079F00013FA002070BD00BF909EFF1F429EFF1F24
:107A00005A9EFF1F589EFF1F109FFF1F184B1A887A
:107A100052B3184A128830B50A80B3F90030002BEF
:107A200083EAE374A4EBE374BCBF2D238B70A0B294
:107A3000ACBF02310331012300E0134603EB8302A4
:107A400052009442F9DA0C4D90FBF3F285FB03E40B
:107A500003FB1200DB173032D3EBA40380B201F832
:107A6000012BF1D10B7030BD044B186808607047D2
:107A7000E49CFF1FC432010067666666383201006D
:107A800070B53C4D2B780646002B35D11C467378DB
:107A90000BB9204670BDFAF7C1FA374A374B384860
:107AA000127831781B78007802EB43034A1E03EB0F
:107AB00080030E2AEDD801A050F822F0257B0000AB
:107AC000477B0000937A0000257B0000937A00003A
:107AD000937A0000937A0000137B0000937A0000F1
:107AE000937A0000937A0000937A0000937A000062
:107AF000937A00000F7B0000AE21224803F0EEFFD6
:107B0000204804F03BFA00232B700124BFE706F065
:107B1000A9FEAF211B4803F0E1FF1B4A01231370AC
:107B20002B70B6E783B91948038804294FF6FF7113
:107B300003F1FF320CBF01230B46134403F07F0314
:107B4000013303800FE073B1013B114A32F8133067
:107B50004BB10E4E0F481049104A338001230026C6
:107B600006700B701370084A0221012311702B70EC
:107B7000204670BD808AFF1F3D9FFF1F3E9FFF1F55
:107B8000E49EFF1F709FFF1FE89FFF1FE09EFF1FE7
:107B90001C9EFF1F149DFF1F9C9CFF1FEB9FFF1F40
:107BA00010B5064B064C1A882046012101F0DAFD7B
:107BB00021884220BDE8104001F0E6BDFC9CFF1F7B
:107BC000109FFF1F10B5064B064C1A882046022155
:107BD00001F0C8FD21884220BDE8104001F0D4BD6D
:107BE000329DFF1F109FFF1F10B5064B064C1A88D1
:107BF0002046042101F0B6FD21884220BDE8104056
:107C000001F0C2BD509EFF1F109FFF1F10B5064B15
:107C1000064C1A882046062101F0A4FD2188422046
:107C2000BDE8104001F0B0BD649EFF1F109FFF1F14
:107C300010B5064B064C1A882046002101F092FD33
:107C400021884220BDE8104001F09EBD9E9EFF1F8E
:107C5000109FFF1F08B5122001F0B0FD054B1988D9
:107C6000884206D0122001F08FFDBDE8084001F0E7
:107C700055BC08BD929EFF1F08B5582001F09EFD1F
:107C8000054B1988884206D0582001F07DFDBDE8DB
:107C9000084001F043BC08BDA29EFF1F08B5142098
:107CA00001F08CFD054B1988884206D0142001F0A4
:107CB0006BFDBDE8084001F031BC08BD3A9DFF1FD7
:107CC000F0B480EAE075A5EBE0750028ACB21FDBEC
:107CD0001DBF2B230B704E1C0E46012300E01346E4
:107CE00003EB830252009542F9DA0B4F94FBF3F257
:107CF00087FB030503FB1244DB173032D3EBA503EC
:107D0000A4B206F8012BF1D133700846F0BC7047DD
:107D10002D230B704E1CE0E767666666174B1888CC
:107D20000C2813D0192815D01A2817D01B2819D0C1
:107D30001C281BD01D281DD01E2803D00C3800B2D3
:107D4000FFF7BEBF0E4A1068086070470D4A106802
:107D5000086070470C4A1068086070470B4A10684A
:107D6000086070470A4A106808607047094A10683E
:107D700008607047084A106808607047DE9EFF1F61
:107D8000E4320100CC320100D0320100D4320100D3
:107D9000D8320100DC320100E0320100034B1888C8
:107DA000A0EB8000400000B2FFF78ABFD09FFF1F0A
:107DB000024B1888643800B2FFF782BF309FFF1F64
:107DC000024B1888643800B2FFF77ABF049FFF1F88
:107DD000024BB3F90000FFF773BF00BFEC9CFF1F1D
:107DE000024B1888033800B2FFF76ABFB69EFF1F28
:107DF000024B18880C3800B2FFF762BF8E9CFF1F41
:107E0000024B1888183800B2FFF75ABFC49CFF1FF6
:107E1000024B1888183800B2FFF752BFC29CFF1FF0
:107E2000024B1888183800B2FFF74ABFB89CFF1FF2
:107E3000C3681888183800B2FFF742BF054B1B888B
:107E40001BB9054B186808607047084604220349AF
:107E500009F0F4BFC09EFF1F383201003432010028
:107E6000054B1B881BB9054B18680860704708460E
:107E70000422034909F0E2BFCA9CFF1F3832010007
:107E80003432010030B5134C85B001252B463C221D
:107E900002212046009503F097FE204604F06EF87C
:107EA00000224021802320460191009311460A4B75
:107EB000029504F011FD204604F06CF907480849CA
:107EC000084A0023036083800B608B8013609380DB
:107ED00005B030BD709FFF1F78390100509FFF1F14
:107EE000689FFF1FD89FFF1F10B500EBC00000F177
:107EF0000F02D2B293B284B09C1E981C3D23039112
:107F00008DE819003921024804F04AFC04B010BD84
:107F1000709FFF1F014B01221A7070475D9FFF1F6A
:107F2000F0B57A4B7A4C7B4F7B4E7C4D85B004226A
:107F30008DE80C0002932046794B4022802103F00B
:107F40004BFC2046774A7849784C09F0EFF8784A9C
:107F5000784B9761784FD761784F9F61784FDF6199
:107F6000784FB761784FF761784FAF61784FEF6125
:107F7000784FA7617848794FE761794F87617949F0
:107F8000794FC761794F8F61794A7A4FCF617A4FC4
:107F900097617A4B7A4FD7617A4F9F617A4E7B4FC8
:107FA000DF617B4F7B4DB7617B4FF7617B4F7C4C33
:107FB000AF617C4FEF617C4F7C48A7617C4FE761EC
:107FC0007C4F7D4987617D4FC7617D4F7D4A8F61C1
:107FD0007D4FCF617D4F7E4B97617E4FD7617E4F46
:107FE0007E4E9F617E4FDF617E4FB7617E4D7F4F3A
:107FF000F7617F4FAF617F4C7F4FEF617F4FA7618C
:108000007F48804FE761804F87618049804FC7611B
:10801000804F8F61804A814FCF61814F9761814B43
:10802000814FD761814F9F61814E824FDF61824FC7
:10803000B761824D824FF761824FAF61824C834FAF
:10804000EF61834FA7618348834FE761834F844982
:108050008761844FC761844F844A8F61844FCF61A9
:10806000844F854B9761854FD761854F854E9F61C2
:10807000854FDF61854F864DB761864FF761864F2B
:10808000864CAF61864FEF61864F8748A761874F67
:10809000E761874F87618749874FC761874F8F6146
:1080A000874A884FCF61884F9761884B884FD76147
:1080B000884F9F61884E894FDF61894F894DB76135
:1080C000894FF761894F8A4CAF618A4F8A488B4943
:1080D000EF618B4F8B4DA761E5618B4F8B4D8C4CC6
:1080E000DFF850E28B4A8C4B8761C5618C618B4E07
:1080F0008B4F8C4D8C4CC1F81CE08C488C4997619F
:10810000D5619C61D861B16005B0F0BD40420F00FF
:10811000709FFF1FF17D00006C8EFF1FF88FFF1F07
:108120005C91FF1F1C89FF1F31B80000448FFF1FA7
:10813000F089FF1F208FFF1F05690000E17D00000F
:1081400011690000B96B0000A17B0000E16B000029
:10815000C57B0000096C0000148AFF1FE97B00004A
:10816000D17D0000748CFF1F21690000316C00007C
:10817000288DFF1F0D7C00004D730000508CFF1FE9
:1081800031690000596C00004C8DFF1F317C0000EC
:10819000C17D0000F090FF1F41690000B17D00002B
:1081A000CC90FF1F5169000025760000048DFF1F51
:1081B000797200009D7D0000E08CFF1F916E000031
:1081C000A96E0000FC8EFF1F9D6E000081730000F1
:1081D0009C8BFF1F99720000B5730000B08FFF1FCA
:1081E000557C00008D7600002C8CFF1F797C0000F0
:1081F000016F00005C8BFF1F61690000816C000053
:108200006490FF1F9D7C0000F5760000088CFF1F26
:10821000716900005D770000948DFF1F8169000087
:10822000CD770000E48BFF1F91690000616F0000B3
:10823000148BFF1FA1690000F17300001C90FF1F49
:10824000B1690000B96F0000B48EFF1FC169000062
:1082500025740000F08AFF1FD16900001170000032
:10826000708DFF1FE169000059740000388AFF1FFC
:10827000F169000069700000988CFF1F016A00001E
:108280000D7A0000D88EFF1F116A00009174000063
:108290002091FF1F216A000035780000488EFF1FE3
:1082A000316A00009D780000CC8AFF1F416A0000FF
:1082B000C5740000D48FFF1FB9720000057900005B
:1082C000908EFF1F516A00001D7D0000A88AFF1FCD
:1082D000616A0000FD740000848AFF1F716A00005B
:1082E00065750000BC8CFF1F816A0000C170000032
:1082F000C08BFF1F916A00005C8AFF1F388BFF1F35
:1083000019710000A16A000071710000B16A0000DB
:10831000C9710000688FFF1FCC89FF1F1491FF1FD8
:1083200021720000D16A000075790000E16A000046
:10833000F9880000C16A0000F0B5461C83B00D4604
:108340000127032336B22AB2044631468DE888005D
:108350002348ADB204F0BAF90C23AA1C12B2009360
:108360000197052321B21E4804F0B0F91D4A1E4BA7
:1083700012881B68BA422AD023D3022A10D11B4C80
:10838000A3F6CA0384FB03241C44DB17C3EB2414A9
:108390000A2CA8BF0A2424EAE474A2B223B202E0A1
:1083A00000231A461C460D35AA1A0120009301909D
:1083B00012B2314603230A4804F006F9204603B0FE
:1083C000F0BD0B4CA3F6FC0384FB0324DDE7094C52
:1083D000A3F6980384FB0324DB17C3EBA404D7E7BD
:1083E000709FFF1F3C9EFF1FA49EFF1F09CB3D8D6A
:1083F0001F85EB51398EE3382DE9F0438FB283B0FE
:10840000DFF84C80BD1D461D2DB204B236B24FF0D0
:1084100001090AB22346314640460095CDF8049042
:1084200004F004F92A463346214640468DE82002EE
:1084300004F0FCF807F10C020095334612B2214615
:10844000CDF80490404604F0F1F803B0BDE8F083A5
:10845000709FFF1F2DE9F043804685B0002956D15B
:108460000121304804F078FC2F4998F8062098F84C
:10847000083011F80290994522DA4FEA89064D46F4
:108480000C24D8F80C3027489B595F6822B2002191
:1084900004F05EFC384609F013FC394602462148D8
:1084A00004F0F0FD1F4804F003FE98F80830013591
:1084B0000934AB42A4B206F1040601DD422CE0D13E
:1084C000B9F1000F13D109F1060999450CDA3C23E3
:1084D00001213B22039102930093019239233F2211
:1084E0003A21104804F05CF905B0BDE8F0830F2391
:1084F00001213B22039102930093019239230C2224
:108500003A21084804F04CF998F80830DBE70021DC
:108510003423009301913F230C22024804F054F8C5
:108520009EE700BF709FFF1F689FFF1F10B5104C94
:108530000121204604F016FC2046012104F00CFC29
:1085400020463422552104F003FC2046022209492A
:1085500004F098FD20460522074904F093FD2046CB
:1085600004F0A6FD2046BDE8104003F013BE00BF96
:10857000709FFF1F303301003433010070B50D468A
:10858000064609F09DFB00EB40008400002D36D02C
:10859000284609F095FB00EB4000400023185B10D3
:1085A00003F16001091A282209B21748C3F16004D7
:1085B00004F0CEFB0121144804F0CEFB284609F05C
:1085C0007FFB29460246104804F05CFD0E4804F08B
:1085D0006FFD02210C4804F0BFFB21B221220A48A2
:1085E00004F0B6FB304609F06BFB31460246064804
:1085F00004F048FD0448BDE8704004F059BD641023
:10860000C4F16004E5E700BF709FFF1F10B50D4B7C
:108610001B5C51F82340237884B013B1012004B0CF
:1086200010BD04AA01A942F8103D2046A36998474D
:10863000A38A9B07F2D401A80099FFF79FFF0120AE
:1086400004B010BD509FFF1F2DE9F04F2F4DDFF8F4
:10865000CCB0DFF8C4A0DFF8C8900FCD91B003AC68
:108660000FC40FCD0FC40FCD0FC42B68236000259E
:10867000A8462F462E4600E09846BAF80030244916
:108680005BF8232028461123F8F796F800EBC00486
:1086900000EB840089FB00340444C017C0EB643451
:1086A000C4F13C00C6F13C0207F14101012600B2D1
:1086B00008F1410300901BB2019612B209B21548AD
:1086C00003F0B4FF08EB060305F211153C2B264618
:1086D000ADB24746D0D134226B210E4804F038FBAE
:1086E00000210C4804F038FB0B4B1B8810AA02EB4E
:1086F000830353F8344C204609F0E2FA0246054859
:10870000214611B0BDE8F04F04F0BCBC202F0100A1
:10871000DC280100709FFF1FAE9CFF1F4027010057
:1087200009000280234B70B5B3F9003083EAE3748B
:10873000A4EBE374002B82B0A1B234DB68466D4633
:10874000012300E0134603EB830252009442F9DA5E
:10875000194E91FBF3F286FB03E403FB1211DB17C6
:108760003032D3EBA40389B205F8012BF1D11946BD
:108770002B70FFF703FF114B1B7813B1104B1B78C5
:108780000BB902B070BD01210E4804F0E5FA3322A6
:1087900064210C4804F0DCFA04220B49094804F077
:1087A00071FC02B070BD2D238DF800300DF1010574
:1087B0006846C5E75A9EFF1F67666666429EFF1FB2
:1087C000589EFF1F709FFF1F3C33010010B5424CA5
:1087D000424882B003F0D2FB2378C3B906213F4858
:1087E00004F0BAFA2378012B37D90A22022B11465A
:1087F0003A486BD004F0ACFA39490322374804F008
:1088000041FC364802B0BDE8104004F051BC354B85
:108810001A7801210523002A35D1019100931146D0
:108820002E4803F053FF304B1A78002A36D0052328
:1088300001220192009300220A21284803F0C4FE7D
:108840002A4B1A78002A35D1012105230191009382
:108850001421224803F03AFFC0E7254C2388092B56
:1088600032D9632B8CBF0A211F210A221B4804F036
:108870006FFA2188194804F06BFC184802B0BDE873
:10888000104004F015BC00220191009311461348DA
:1088900003F09AFE144B1A78002AC8D1052301214F
:1088A000019100930A210D4803F010FF0F4B1A7835
:1088B000002AC9D00122052301920093002214212D
:1088C000064803F081FE89E73021CEE704F040FA44
:1088D0000322084992E700BFEB9FFF1F709FFF1F15
:1088E000483301003D9FFF1F3E9FFF1FE49EFF1F77
:1088F000E09EFF1F44330100F8B56D4D287840B964
:108900006C4B1B6899425CD36B4A012313702B702C
:10891000F8BD0C4600266948664F03F02FFB04F6AD
:10892000AC53324665483B6031212E7004F010FA9A
:1089300001216248624D04F015FA31465F4804F0A7
:108940000BFA05225F495D4804F09CFB5B4804F08C
:10895000AFFB0C221021594804F0FAF90B225A49B6
:10896000564804F08FFB05225849544804F08AFB0E
:10897000524804F09DFB564B50481C68A4F69803DF
:10898000C3EB031385FB03251D441021DB172022B5
:10899000C3EB652504F0DCF940F6CC339C4205F1CD
:1089A00024054FF022014FF004000BDCFFF7C4FC5C
:1089B000484B1C88064674B3012C46D0022C41D08B
:1089C0000120F8BDFFF718FD092243493B4804F098
:1089D00059FB2A221021394804F0BAF93F4C374894
:1089E00084FB0534EB17C3EBA404214604F0B0FB71
:1089F00001223B49314804F045FB04EB8401A5EB1F
:108A000041012E4804F0A4FB012236492B4804F012
:108A100039FB0120F8BD34491022284804F032FB0C
:108A2000264804F045FB2A221021244804F090F93E
:108A30003146224804F08CFB07222C491F4804F0E1
:108A400021FBCBE70C222A49E7E70C2229491B48E6
:108A500004F018FB194804F02BFB2A2210211748B8
:108A600004F076F9314615481C4E04F071FB0722DC
:108A70001E49124804F006FB86FB0536EB17C3EBD4
:108A8000A60631460D4804F063FB224614490B4804
:108A900004F0F8FA06EB8601A5EB4101074804F063
:108AA00057FB22460F49054804F0ECFA2046F8BD72
:108AB000808AFF1F649FFF1FE89FFF1F709FFF1F9B
:108AC0003B773B984C3301005433010034330100B1
:108AD000A49EFF1F3C9EFF1F603301006766666611
:108AE000603F0100D83E01006C330100803301007B
:108AF00098330100883301002DE9F041754C22784C
:108B0000002A05460F4614BF4FF001084FF0000839
:108B10004ED1714E3368CB1AB3F5FA6F04D86B7827
:108B2000A3B94046BDE8F0816C4B6D486D49DFF854
:108B3000D0E11A70012303700988237026208EF873
:108B4000002000F021FE6B78002BEAD03760F9F7A7
:108B500065FA654A654B6649127828781B7809786A
:108B600002EB4303421E03EB81030E2AD9D801A175
:108B700051F822F0658C0000318C0000238B00003E
:108B8000658C0000238B0000238B0000238B0000EA
:108B9000198C0000238B0000CB8B0000238B00007E
:108BA000238B0000238B0000238B0000C78B000069
:108BB000AF215048484E02F091FFFFF707FE002317
:108BC00037602370ABE705F04DFE4A4803F0D6F955
:108BD0000221484804F0C0F80F222321454804F040
:108BE000B7F805224449434804F04CFA414804F0E0
:108BF0005FFA1E2223213F4804F0AAF805223F49CC
:108C00003C4804F03FFA3B4804F052FA394803F07C
:108C1000C1FA00F0D3FC84E7394D2B78012B50D9F1
:108C2000304B2620198800F0AFFD00232B7078E729
:108C3000002B3FF476AF013B324A32F81330002B61
:108C40003FF46FAF274C304825492D4A23804FF021
:108C500001080023037081F8008082F80080FFF78C
:108C6000B5FD5EE793B1013B264A32F8131019B304
:108C70001C4B254D1A4C224A198000260123262020
:108C80002E702370137000F07FFD15E0154C1E4907
:108C900022880B7004284FF6FF7002F1FF310CBFE1
:108CA000012202460A440E4E154D02F07F020132A7
:108CB0000121228031702B70FFF788FD4FF00108F1
:108CC0002FE70649064A012300200870137023701D
:108CD000A6E700BF808AFF1FE49FFF1FE89FFF1FDA
:108CE0009C9CFF1FE09EFF1F3D9FFF1F3E9FFF1F9D
:108CF000E49EFF1F709FFF1FA8330100B0330100E7
:108D0000EB9FFF1F1C9EFF1F149DFF1F2DE9F04FBF
:108D100005468BB00F46AD480121164604F022F8F7
:108D2000AA8812F0010440F0B080DFF8CC8298F8F5
:108D30000030002B7DD1AB79A54AD15CA1B9DFF819
:108D4000BCA279781AF8039041B339780139072920
:108D500000F2B780DFE811F0F1005401B5006C01BA
:108D6000B500B500B500E9007C78002C00F0CA80A1
:108D70000139EC68387854F82170FC68411EB4F869
:108D80000080072900F2A780DFE811F07401590183
:108D9000A5006C01A500A500A5009F00DFF854A266
:108DA000DAF80020B21AB2F5967F75D9894A1078A0
:108DB00001281ABF012010701170874A18BF0146A0
:108DC000D05CC0EB0900C0B2FFF78EF80124CAF8EE
:108DD0000060AB889B0770D57B78002B6DD0F9F7CE
:108DE0001DF97E4B7E4A7F481B78127839780078CF
:108DF000022515FB02330A2903EB800300F04E81A4
:108E00000C295AD1002B58D003F11900764E774A1D
:108E1000013B0021400080B226F813100123157099
:108E200088F8003000F0B0FC714B032220461A7025
:108E30002FE0664803F0A2F80121644803F08CFF9C
:108E400062482246214603F083FFAB88580725D4A9
:108E50002C68204608F034FF214602465B4804F0A7
:108E600011F95A4804F024F9092201238DE80C0075
:108E700000217F23554803F0D9FB00212846FFF746
:108E8000E9FA002388F8003055E7AB6831463846E8
:108E900098470BB0BDE8F08F0846FAE72B6804A8A6
:108EA000984704A808F00CFF04A90246474804F0BC
:108EB000E9F8464804F0FCF8D6E720460BB0BDE8D8
:108EC000F08F00240AF8039083E70021D15438463C
:108ED000FB699847FC68A4F80080002725223C2302
:108EE0008DE8840041211822384803F06DFBE968C1
:108EF000A879FFF78BFB374A3E4B17701E600BB00B
:108F0000BDE8F08F3B490A68B21AB2F5967FD4D912
:108F1000304F0E603E78012E00F0B480E9681846AC
:108F200001233B70FFF772FBB3E7304AE979117018
:108F3000012288F800200024C4E72A7A013A4A4531
:108F4000BFDD09F10104E4B2A145BAD0224E16F802
:108F500003B0CBEB0900C0B20021FEF7C5FF2B7AAE
:108F6000052BD9461BD9CBEB0402042A40F3AE8073
:108F7000A4F1040BBBF1000FC0F2B080063B5B45CF
:108F8000A8BF5B465FFA83F9AA791348B15C99429E
:108F900005D000F8029001212846FFF75BFAC9EBE3
:108FA0000400C0B201210B4EFEF79EFF00213423C6
:108FB000019100930548317040230B223F21A146C7
:108FC00003F002FB0124AB797CE700BF709FFF1F19
:108FD000D89FFF1FE99FFF1F689FFF1F3D9FFF1F37
:108FE0003E9FFF1FE49EFF1F1C9EFF1FE89FFF1F69
:108FF000EB9FFF1FD49FFF1F808AFF1F509FFF1F03
:109000000FFA89F1E868604C50F8216021680491FA
:1090100034785E4904980860002C71D0012C7FF4EC
:1090200050AF5B4A317A88F800401170002449E75C
:10903000B9F1000F50D009F1FF34E4B284E7B98AE6
:1090400001F0040189B200293FF440AF3B6A03926A
:109050009847039A00283FF43DAFAB79FC680021A4
:10906000D15438E77B8A43453CD908F101081FFAFF
:1090700088F830E73B8A43453BD208F1FF381FFAB6
:1090800088F828E725238DE8180042483C703C23E7
:109090001822412103F098FA3046FAE6002B3FF4FB
:1090A0000CAF3D4A3D4E1188394A03F11900013B8E
:1090B000400080B226F81310012388F800301570A4
:1090C00000F062FB364B20461D70E2E6002A3FF7B7
:1090D00055AF04F1FF3B4DE74C46F3E64FF0000976
:1090E0004B4651E7BB8ADA077FF5F5AEB7F810803B
:1090F000F1E6BB8AD9077FF5EEAEB7F81280EAE653
:109100002849C85CC0EB090009F1010EC0B2012179
:109110004FF0340B02F803E0FEF7E6FEB6681D4898
:10912000019440230B223F210124CDF800B003F02D
:109130004BFA40230B223F211648CDF800B0019492
:1091400003F0C4FA2146134803F006FE304608F047
:10915000B7FDA0EB800000F15F0109B20F220D48BE
:1091600003F0F6FD304608F0ABFD314602460948F3
:1091700003F088FF074803F09BFFE968A879FFF731
:1091800045FAAB799EE600BF28A0FF1FD49FFF1FC2
:10919000E89FFF1F709FFF1FE09EFF1F1C9EFF1F89
:1091A000EB9FFF1F689FFF1F2DE9F047DFF8089234
:1091B0006D4B99F800601B68DFF800A282B00036A2
:1091C00001934FF0030018BF0126019F9AF8008019
:1091D00004F028FE0546042004F024FE0446052081
:1091E00004F020FE800040EA4404062004F01AFE49
:1091F0002C4364B25D4944EAC0000A7880F00F0352
:10920000DBB29A425A4A3CD01760002259480B7090
:1092100003788DF800808DF8012053B3564A126808
:109220004EF66021BA1A8A4219D8022B59D0012B66
:109230005FD0062B48D0032B63D0042B69D0052BBD
:1092400077D0072B7DD0082B00F08380092B68D0C6
:1092500016B14A4802F09EFF02B0BDE8F087484AC6
:10926000484C00230121237003701360938089F818
:1092700000103A4669464448FFF748FD3043C6B2FD
:10928000E6E71268BA1A1E2A6BD99AF800209342B0
:1092900022D0394C3D488AF80030012B276082EA01
:1092A000030207609846B1D0042BAFD1374800685D
:1092B000381AB0F5C87FA9D9354C2068381A322839
:1092C000A4D927601A46A1E73A4669463148FFF714
:1092D0001DFD3043C6B2BBE7012B4FF00002E3D1C6
:1092E000E4E73A4669462C48FFF710FD3043C6B222
:1092F000AEE73A4669462948FFF708FD3043C6B253
:10930000A6E73A4669462648FFF700FD3043C6B255
:109310009EE73A4669462348FFF7F8FC3043C6B259
:1093200096E73A4669462048FFF7F0FC3043C6B25C
:109330008EE73A4669461D48FFF7E8FC3043C6B25F
:1093400086E73A4669461A48FFF7E0FC3043C6B262
:109350007EE73A4669461748FFF7D8FC3043C6B265
:1093600076E7002252E700BF28A0FF1FEC9FFF1FF7
:10937000589FFF1FE89FFF1FE09FFF1F709FFF1F69
:10938000D89FFF1FEA9FFF1F70310100F09FFF1F52
:10939000609FFF1FA0310100C8300100DC2F0100D9
:1093A0001C3E01000C3E0100CC2F010034300100B6
:1093B000583E01001491FF1F808AFF1F5C9FFF1F12
:1093C00028B11028044BA8BF102018607047024B2A
:1093D00001201860704700BFF49FFF1F08B50020F0
:1093E00006F02AF90028FAD108BD00BF10B50446DE
:1093F0004FF4406005F034F805F08CF80A4B1B7808
:1094000033B96CB1102C094BA8BF10241C6010BDDF
:109410004FF4C05004F0FAFD04F02EFF002CF1D1FF
:10942000024B01241C6010BD429EFF1FF49FFF1FD2
:1094300070B50D461446064605F062F8284605F05C
:109440005FF8204605F05CF8084B1B7813B1084B19
:109450001B7803B970BD304604F0B6FE284604F010
:10946000B3FE2046BDE8704004F0AEBE429EFF1F32
:10947000589EFF1F38B5164D2B78044641F6FF72F3
:10948000A0F50050824203F1FF33A8BF02461B0241
:1094900002F5005203F47063100443F4604343F098
:1094A0000E0300F4FE005204184302F0FE42104383
:1094B00005F0F8FF2868013860F01F00C4F3C612F9
:1094C00004F07F01C0B2BDE83840FFF7B1BF00BF74
:1094D000F49FFF1F70B5104E3378013B1B0203F45D
:1094E0007063044643F430430806220400F0FE4053
:1094F00043F00B03034302F4FE0018430D4605F04E
:10950000D1FF3068013860F04F002A462146C0B2D2
:10951000BDE87040FFF78CBFF49FFF1F08B56421C2
:109520000720FFF7D7FF7F210B20BDE80840FFF79A
:10953000D1BF00BF70B5104E3378013B1B0203F45E
:109540007063044643F410430806220400F0FE4012
:1095500043F00903034302F4FE0018430D4605F0EF
:10956000A1FF3068013860F06F002A462146C0B282
:10957000BDE87040FFF75CBFF49FFF1F38B50E4D8C
:109580002B78013B1B0203F47063044643F4104341
:10959000000443F0090300F4FE00184305F082FFC5
:1095A0002868013860F06F002146C0B20022BDE893
:1095B0003840FFF73DBF00BFF49FFF1F10B50021EB
:1095C0007B20FFF787FF0024E0B2FFF7D7FF0134CD
:1095D000022004F05DFC802CF6D110BD38B50C469D
:1095E000054604F08DFF204604F08AFF074B1B78E8
:1095F00013B1074B1B7803B938BD284604F0E4FDCE
:109600002046BDE8384004F0DFBD00BF429EFF1F8A
:10961000589EFF1F38B50D4D2B78013B1B0203F4FC
:109620007063044643F45043000443F00D0300F418
:10963000FE00184305F036FF2868013860F02F005F
:109640002146C0B2BDE83840FFF7C8BFF49FFF1FF6
:1096500038B50E4D2B78013B01381B02C4B203F420
:109660007063200443F4404343F00C0300F4FE0015
:10967000184305F017FF2868013860F03F002146C5
:10968000C0B2BDE83840FFF7A9BF00BFF49FFF1F7D
:1096900038B504460D46F02004F032FF35B12544BC
:1096A00014F8010B04F02CFFAC42F9D1F720BDE80F
:1096B000384004F025BF00BF00B50B4B83B0024615
:1096C000998818680090032AADF8041002D903B0F5
:1096D0005DF804FB684606218DF80520FFF7D8FFEA
:1096E00003B05DF804FB00BF983E010000B50B4BD2
:1096F000024683B0186899880090131F4C2BADF870
:10970000041002D903B05DF804FB684606218DF809
:109710000520FFF7BDFF03B05DF804FBA03E01008C
:10972000030203F4FE43C0F3C6101843704700BFA2
:1097300003784078DB0103F47E5300F07F00184388
:10974000704700BF82B002AA114642F8040D002003
:1097500012F8013B03F07F03914243EA0020F7D166
:1097600002B07047003210B403884FF0010404FACD
:1097700001F418BF012202FA01F123EA04020A43AC
:10978000028010BC704700BF70B5CEB20C460546D3
:1097900003F010FF864203D03146284603F024FF31
:1097A0000135284603F006FF240A844205D02146ED
:1097B0002846BDE8704003F017BF70BD38B50546B8
:1097C00003F0F8FE4FF0000460F30704681C03F098
:1097D000F1FE60F30F24A0B238BD00BFF8B5044617
:1097E0000020FFF7EBFF002C00F083814FF4AF6106
:1097F0000220FFF7C9FF04204FF47A61FFF7C4FF8E
:109800000B2004F00FFB002840F079874FF496619D
:109810000620FFF7B9FF4FF4FA610820FFF7B4FF05
:109820004FF4FA610A20FFF7AFFF40F6B8310C2081
:10983000FFF7AAFF4FF42F612220FFF7A5FF40F6A4
:10984000AC512420FFF7A0FF7D212A20FFF79CFFC9
:109850000C210E20FFF798FF01211020FFF794FF45
:1098600002211220FFF790FF00211420FFF78CFF48
:1098700000211620FFF788FF02211820FFF784FF40
:1098800001211A20FFF780FF01211C20FFF77CFF38
:1098900004211E20FFF778FF14212020FFF774FF1A
:1098A00001212620FFF770FF03212820FFF76CFF1E
:1098B00004212C20FFF768FF14212E20FFF764FFFE
:1098C00000213020FFF760FF0C213220FFF75CFF02
:1098D00000213420FFF758FF00213620FFF754FF06
:1098E00000213820FFF750FF00213A20FFF74CFFFE
:1098F00000213C20FFF748FF00213E20FFF744FFF6
:1099000000214020FFF740FF00214220FFF73CFFED
:109910001F214420FFF738FF13214620FFF734FFB3
:109920000E214820FFF730FF11214A20FFF72CFFBE
:109930000A214C20FFF728FF00214E20FFF724FFCB
:1099400006215020FFF720FF02215220FFF71CFFC5
:109950000C215420FFF718FF00215620FFF714FFB9
:1099600000215820FFF710FF01215A20FFF70CFFBC
:1099700008215C20FFF708FF0A215E20FFF704FFA3
:1099800000216020FFF700FF04216220FFF7FCFEAA
:1099900001216420FFF7F8FE00216620FFF7F4FEA6
:1099A0000B216820FFF7F0FE7F216A20FFF7ECFE15
:1099B00000216C20FFF7E8FE00216E20FFF7E4FE97
:1099C00000217020FFF7E0FE00217220FFF7DCFE8F
:1099D00000217420FFF7D8FE1F217620FFF7D4FE68
:1099E00013217820FFF7D0FE0E217A20FFF7CCFE5E
:1099F00011217C20FFF7C8FE0A217E20FFF7C4FE5C
:109A00001F218020FFF7C0FE13218220FFF7BCFE3C
:109A10000E218420FFF7B8FE11218620FFF7B4FE47
:109A20000A218820FFF7B0FE00218A20FFF7ACFE54
:109A300000218C20FFF7A8FE00219620FFF7A4FE4E
:109A400000219820FFF7A0FE00219A20FFF79CFE3E
:109A500005219C20FFF798FE06219E20FFF794FE2B
:109A60000021A020FFF790FE7F21A220FFF78CFEAF
:109A700040F2A461A420FFF787FE4FF4E161A62025
:109A8000FFF782FE0021A820FFF77EFE0021AA201A
:109A9000FFF77AFE0221AC20FFF776FE0121AE200F
:109AA000FFF772FE0121B020FFF76EFE0B21B220FE
:109AB000FFF76AFE6421B420FFF766FE6421B6203A
:109AC000FFF762FE0321B820FFF75EFE2C21002085
:109AD000FFF75AFE0220FFF771FEB0F5805F0346E4
:109AE00016D34FF4AF610220FFF74EFE4FF4AF6381
:109AF0000EE04FF6FF7398423FF478AE2C2840F00A
:109B00000A860220FFF75AFEB0F5805F0346E8D2CE
:109B1000D24A04201380FFF751FEB0F5805F034660
:109B200080F05684CE4A06201380FFF747FEA0F54A
:109B30002F739BB2B3F57A6F024606D940F62821FF
:109B40000620FFF721FE40F62822C64B08201A8087
:109B5000FFF734FEA0F52F739BB2B3F57A6F024680
:109B600006D940F6E4410820FFF70EFE40F6E44235
:109B7000BD4B0A201A80FFF721FEA0F5FA739BB2B5
:109B800040F6AC518B42024606D94FF4FA610A20E6
:109B9000FFF7FAFD4FF4FA62B44B0C201A80FFF77E
:109BA0000DFEA0F5FA739BB240F6AC518B42024613
:109BB00006D940F6B8310C20FFF7E6FD40F6B83282
:109BC000AB4B0E201A80FFF7F9FD1828034600F270
:109BD000C584A84A10201380FFF7F0FD431E9BB2F6
:109BE0000F2B024604D901211020FFF7CDFD0122E1
:109BF000A14B12201A80FFF7E1FD0A28034600F26C
:109C0000A6849E4A14201380FFF7D8FD012803463E
:109C100004D900211420FFF7B7FD0023984A16202D
:109C20001380FFF7CBFD7F28034600F28984954A15
:109C300018201380FFF7C2FD0528034600F279843F
:109C4000914A1A201380FFF7B9FD0C28034600F251
:109C5000BD848E4A1C201380FFF7B0FD0428034604
:109C600000F2AD848A4A1E201380FFF7A7FD092861
:109C7000034600F29D84874A20201380FFF79EFD53
:109C80004628034600F28D84834A22201380FFF782
:109C900095FDA0F5FA739BB240F6AC518B4202469B
:109CA00006D94FF42F612220FFF76EFD4FF42F628B
:109CB0007A4B24201A80FFF781FDA0F5FA739BB23E
:109CC00040F6AC54A342024604D921462420FFF7B3
:109CD0005BFD2246724B26201A80FFF76FFD7F281E
:109CE000034600F257846F4A28201380FFF766FD71
:109CF0000628034600F247846B4A2A201380FFF7A8
:109D00005DFDA0F132039BB2B3F5967F024604D904
:109D10007D212A20FFF738FD7D22644B2C201A80FC
:109D2000FFF74CFD0C28034600F22684604A2E20E3
:109D30001380FFF743FD1E28034600F216845D4A98
:109D400030201380FFF73AFD0928034600F2D08443
:109D5000594A32201380FFF731FD1E28034600F2D6
:109D6000C084564A34201380FFF728FD7F2803461D
:109D700000F2B084524C36202380FFF71FFD7F286D
:109D8000034600F2A08438206380FFF717FD7F2888
:109D9000034600F291843A20A380FFF70FFD7F284D
:109DA000034600F282843C20E380FFF707FD7F2812
:109DB000034600F273843E202381FFF7FFFC7F28D7
:109DC000034600F2648440206381FFF7F7FC7F289C
:109DD000034600F255844220A381FFF7EFFC394D82
:109DE00028804420FFF7EAFC3028034600F2418433
:109DF000354A46201380FFF7E1FC3028034600F285
:109E00003184324C48202380FFF7D8FC30280346A9
:109E100000F221844A206380FFF7D0FC30280346FB
:109E200000F212844C20A380FFF7C8FC30280346C0
:109E300000F2DF834E20E380FFF7C0FC01280346D9
:109E400004D900214E20FFF79FFC0023204A502018
:109E50001380FFF7B3FC431E3CE000BF449DFF1F8F
:109E60000E9FFF1FFE9CFF1FDC9EFF1FA89EFF1F73
:109E7000C09CFF1F8E9CFF1F5A9EFF1F929EFF1FBC
:109E80003A9DFF1F949CFF1F4A9DFF1FE49CFF1FEC
:109E9000DE9CFF1FC89CFF1FEE9EFF1F569EFF1FEC
:109EA000529EFF1FE09EFF1FB69EFF1F069FFF1FD3
:109EB000AE9CFF1F309DFF1F1C9FFF1FDE9EFF1FDC
:109EC0001C9EFF1F109FFF1FB89CFF1FB89EFF1F07
:109ED000DC9CFF1F9BB20B2B024604D906215020AD
:109EE000FFF752FC0622CF4B52201A80FFF766FC88
:109EF0000428034600F27783CB4A54201380FFF7EF
:109F00005DFC431E9BB21D2B024604D90C2154203C
:109F1000FFF73AFC0C22C54B56201A80FFF74EFC87
:109F20000128034604D900215620FFF72DFC002309
:109F3000BF4A58201380FFF741FC7F28034600F2F8
:109F40004C83BC4A5A201380FFF738FC431E9BB257
:109F5000092B024604D901215A20FFF715FC0122E2
:109F6000B54B5C201A80FFF729FC431E9BB2102BD7
:109F7000024604D908215C20FFF706FC0822AF4BFB
:109F80005E201A80FFF71AFC431E9BB21D2B02466F
:109F900004D90A215E20FFF7F7FB0A22A84B6020B4
:109FA0001A80FFF70BFC0228034600F2A482A54AA0
:109FB00064201380FFF702FC0128034604D9012125
:109FC0006420FFF7E1FB01239F4A62201380FFF723
:109FD000F5FBC31E9BB2012B024604D9042162206B
:109FE000FFF7D2FB0422994B66201A80FFF7E6FBAD
:109FF0007F28034600F27982954A68201380FFF794
:10A00000DDFB7F28034600F26A82924A6A201380B1
:10A01000FFF7D4FB7F28034600F25B828E4A6C2058
:10A020001380FFF7CBFB0328034600F24C828B4AD8
:10A030006E201380FFF7C2FB1928034600F23D8211
:10A04000874A70201380FFF7B9FB0228034600F20D
:10A050002E82844A72201380FFF7B0FB0628034645
:10A0600000F21F82804A74201380FFF7A7FB0528A7
:10A07000034600F210827D4A8A201380FFF79EFB80
:10A080000A28034600F20182794A8C201380FFF7E8
:10A0900095FB0428034600F2F281764A982013804B
:10A0A000FFF78CFB0128034604D900219820FFF715
:10A0B0006BFB0023704A9A201380FFF77FFB012877
:10A0C000034604D900219A20FFF75EFB00236B4A68
:10A0D00096201380FFF772FB0B28034600F2C9811C
:10A0E000674A9C201380FFF769FB831E9BB2032BFA
:10A0F000024604D905219C20FFF746FB0522614B4F
:10A1000076201A80FFF75AFB3028034600F2AB8115
:10A110005D4A78201380FFF751FB3028034600F298
:10A120009C815A4C7A202380FFF748FB3028034655
:10A1300000F28D817C206380FFF740FB30280346CE
:10A1400000F27F817E20A380FFF738FB3028034692
:10A1500000F271818020E380FFF730FB3028034656
:10A1600000F263814A4A82201380FFF727FB3028E0
:10A17000034600F25481474C84202380FFF71EFBE6
:10A180003028034600F2458186206380FFF716FBE6
:10A190003028034600F237818820A380FFF70EFBAA
:10A1A0003028034600F22981A020E380FFF706FB58
:10A1B0000128034604D90021A020FFF7E5FA002377
:10A1C000354A9E201380FFF7F9FAC31E9BB20C2B71
:10A1D000024604D906219E20FFF7D6FA06222F4B0D
:10A1E000A2201A80FFF7EAFA431E9BB27E2B02469A
:10A1F00004D97F21A220FFF7C7FA7F22284BA42091
:10A200001A80FFF7DBFAA0F5AF639BB2B3F5167FB8
:10A21000024647D940F2A461A420FFF7B5FA40F204
:10A22000A4623FE02089FF1F2E89FF1FA889FF1F1E
:10A230001E9DFF1FA29EFF1F889CFF1FAC89FF1F52
:10A240002C89FF1F4E9EFF1FB09EFF1FEC9CFF1F1F
:10A25000F09EFF1F1C9DFF1FCC9CFF1F7C9CFF1FBF
:10A26000409FFF1F3C9EFF1F189FFF1FD49EFF1F94
:10A270005C9EFF1F4C9EFF1FCA9CFF1F289DFF1F57
:10A280009C9EFF1FB09CFF1FC29CFF1F2C9EFF1FA8
:10A29000C49CFF1F349EFF1FC09EFF1F9489FF1F99
:10A2A000E29EFF1FD64BA6201A80FFF787FAA0F583
:10A2B000AF639BB2B3F5167F024606D94FF4E16156
:10A2C000A620FFF761FA4FF4E162CE4BA8201A8076
:10A2D000FFF774FA0628034600F28980CA4AAA20CA
:10A2E0001380FFF76BFA032803467AD8C74AAC20DD
:10A2F0001380FFF763FA0328034600F21481C44A6F
:10A30000B0201380FFF75AFA0328034600F20581B4
:10A31000C04AAE201380FFF751FA7F28034600F2AF
:10A32000F680BD4AB2201380FFF748FA7F28034623
:10A3300000F2E780B94AB4201380FFF73FFA431ECA
:10A340009BB2C62B024604D96421B420FFF71CFA45
:10A350006422B34BB6201A80FFF730FA431E9BB23B
:10A36000C62B024604D96421B620FFF70DFA6422F9
:10A37000AC4BB8201A80FFF721FA082822D82B8886
:10A38000DFF8C0E2A84FA94AA94DAA4EAA4CAB4992
:10A3900003F0010CAEF800C0C3F3400EA7F800E0D4
:10A3A000C3F380071780C3F3C007A54A2F70C3F318
:10A3B0000017C3F34015C3F38013378025800B804B
:10A3C0001080F8BDB8200321FFF7DEF90320D6E79F
:10A3D0004FF47A610420FFF7D7F94FF47A63FFF75F
:10A3E000A1BB0021AA20FFF7CFF900237EE70021BF
:10A3F000A820FFF7C9F9002370E70A218820FFF79A
:10A40000C3F90A23D0E611218620FFF7BDF91123F5
:10A41000C2E60E218420FFF7B7F90E23B4E613211C
:10A420008220FFF7B1F91323A5E61F218020FFF753
:10A43000ABF91F2396E60A217E20FFF7A5F90A2330
:10A4400088E611217C20FFF79FF911237AE60E217F
:10A450007A20FFF799F90E236CE613217820FFF795
:10A4600093F913235DE61F217620FFF78DF91F2353
:10A470004EE600219620FFF787F9002330E6002101
:10A480008C20FFF781F9002307E600218A20FFF7DF
:10A490007BF90023F8E500217420FFF775F900230C
:10A4A000E9E500217220FFF76FF90023DAE50021CA
:10A4B0007020FFF769F90023CBE500216E20FFF73C
:10A4C00063F90023BCE500216C20FFF75DF9002350
:10A4D000ADE57F216A20FFF757F97F239EE50B2129
:10A4E0006820FFF751F90B238FE500216620FFF765
:10A4F0004BF9002380E500216020FFF745F9002398
:10A5000055E50B21B220FFF73FF90B2312E701219C
:10A51000AE20FFF739F9012303E70121B020FFF74F
:10A5200033F90123F4E60221AC20FFF72DF90223D1
:10A53000E5E602211820FFF727F90223FFF780BB89
:10A5400000211620FFF720F90023FFF770BB02213E
:10A550001220FFF719F90223FFF753BB0C210E203D
:10A56000FFF712F90C23FFF734BB14212E20FFF75D
:10A570000BF91423FFF7E3BB04212C20FFF704F9A8
:10A580000423FFF7D3BB03212820FFF7FDF80323A3
:10A59000FFF7B2BB01212620FFF7F6F80123FFF7F2
:10A5A000A2BB14212020FFF7EFF81423FFF76CBBA8
:10A5B00004211E20FFF7E8F80423FFF75CBB01210C
:10A5C0001C20FFF7E1F80123FFF74CBB01211A2003
:10A5D000FFF7DAF80123FFF73CBB00215820FFF713
:10A5E000D3F80023ADE402215220FFF7CDF8022377
:10A5F00082E40A214C20FFF7C7F80A231AE400BFBF
:10A60000489DFF1FC89EFF1F8A9CFF1F029DFF1FC2
:10A61000B29EFF1F409EFF1FD49CFF1FF69CFF1F92
:10A62000049FFF1F309FFF1FFC9CFF1F329DFF1FD9
:10A63000589EFF1F509EFF1FB49EFF1F649EFF1F6A
:10A64000909CFF1F9E9EFF1F11214A20FFF79CF840
:10A650001123FFF7E7BB0E214820FFF795F80E23E3
:10A66000FFF7D8BB13214620FFF78EF81323FFF71F
:10A67000C8BB1F214420FFF787F81F23FFF7B8BB93
:10A6800000214020FFF780F80023FFF7A4BB002142
:10A690003E20FFF779F80023FFF795BB00213C200F
:10A6A000FFF772F80023FFF786BB00213A20FFF77F
:10A6B0006BF80023FFF777BB00213820FFF764F821
:10A6C0000023FFF768BB00213620FFF75DF8002369
:10A6D000FFF759BB00213420FFF756F80023FFF79E
:10A6E00049BB0C213220FFF74FF80C23FFF739BB91
:10A6F00000213020FFF748F80023FFF729BB40F680
:10A7000028210620FFF740F840F6E4410820FFF733
:10A710003BF8FFF785B817287FF668A819287FF659
:10A72000D7A81B287FF6F4A81C283FF409A91E28E7
:10A730007FF60EA91F283FF413A920283FF42CA967
:10A7400021283FF435A922283FF43AA923283FF4D1
:10A7500043A924283FF474A925283FF479A9262881
:10A760003FF47AA927283FF47FA928283FF48AA933
:10A7700029283FF48FA92A283FF49CA92B287FF48D
:10A78000A5A9FFF79FB900BFF8B5CB2006F008FDDB
:10A79000204B214A054603CB1368C5F803001A0C69
:10A7A000BA20C5F807102B80AA70FEF7B9FF2E4615
:10A7B000002426F80B0FA0B2FFF700F8FEF7B0FF59
:10A7C0000234BA2C26F8020FF5D16C1E05F1C6062C
:10A7D0004FF0FF3014F8013F082758400F4B40F36B
:10A7E00000017A1E0B4012F0FF0783EA5000F5D1FA
:10A7F000B442EFD1C043FEF7A5FF3A46C5F8C70003
:10A80000CB21284604F09CFE2846BDE8F84006F01F
:10A81000CFBC00BFAC3E0100A83E01002083B8EDD4
:10A82000F0B50E4B0E4C054693E8070085B0246842
:10A830002E88AD7801AB83E80700270C184600226C
:10A840000B21ADF804408DF80670ADF80C608DF862
:10A850000E5004F075FE05B0F0BD00BFB83E01001B
:10A86000A83E0100F0B5124B124D1E68124F0FCDDD
:10A8700087B06C460FC495E8030044F8040B3868B1
:10A880003B79CDF80D00320C2C2021808DF8022070
:10A890008DF81130ADF80060FEF742FF0022ADF8F0
:10A8A0000B001221684604F04BFE07B0F0BD00BF5C
:10A8B000A83E0100C43E010034330100002004F032
:10A8C000BBBE00BF02F02EBE70B5124C82B0002598
:10A8D00040230646294620460093019580232022E6
:10A8E00001F072FE20222946204602F031FA20466D
:10A8F000012102F037FA304607F0E2F9314602460C
:10A90000204602F0BFFB204602B0BDE8704001F0D7
:10A9100041BC00BF709FFF1FF0B5CA2983B075D935
:10A920000546441E00F1C6064FF0FF3014F8012F13
:10A9300008275040404A40F300017B1E0A4013F0B4
:10A94000FF0782EA5000F5D1B442EFD1C043FEF7D1
:10A95000F9FE0146D5F8C7000190019A914202D054
:10A96000B2F17F2F0BD105F10B00FEF7E1FEBA2803
:10A970000BD03248FFF7A8FF002003B0F0BD3048ED
:10A98000FFF7A2FF384603B0F0BD05F10D00FEF75A
:10A99000CFFE2C2840D1002440F6AC5613E004280A
:10A9A0001AD0062821D008281FD00A2828D00C2821
:10A9B00022D1A1F5FA7292B2B24201D8FEF7E4FEBA
:10A9C0000234BA2C0ED004F10D002844FEF7B0FE7C
:10A9D000022C0146A0B2E2D1B1F5805FEED3023481
:10A9E000BA2CF0D1012003B0F0BDA1F52F7292B2C4
:10A9F000B2F57A6FE4D8E1E7222801D0242811D1FA
:10AA0000A1F5FA7292B2B242DAD8D7E70D48FFF751
:10AA10005BFF002003B0F0BD0B48FFF755FF00209F
:10AA200003B0F0BD2A28C9D1A1F1320292B2B2F529
:10AA3000967FC5D8C2E700BF2083B8ED083F01006C
:10AA4000F43E0100DC3E01001C3F010003290CD94B
:10AA500070B5461C82B005460C46304603222A4992
:10AA600007F09CF910B102B070BD70470B2C05D9EE
:10AA700005222649281D07F091F940B12448FFF727
:10AA800023FF244802B0BDE87040FFF7C9BE05F1BE
:10AA90000901032201A807F0D1F901A803221E49E8
:10AAA00007F07CF9D8B103221C4901A807F076F918
:10AAB00008B301A803221A4907F070F9B0B9194880
:10AAC000FFF702FFA11E89B23046FFF725FF0028DD
:10AAD000C9D0154802B0BDE87040FFF7F5BE134875
:10AAE000FFF7F2FEFFF750FE1148F3E71148FFF7BA
:10AAF000EBFE1148C6E71148FFF7E6FE02B0BDE8DD
:10AB00007040FFF7AFBE00BFA83E01004C3301000C
:10AB1000343F0100483F01004C3F0100743F0100F9
:10AB20008C3F0100903F0100A43F0100503F010015
:10AB3000643F0100B83F0100CC3F0100783F0100B5
:10AB40002DE9F043174D2B6883B081460F469046A0
:10AB5000F3B1154E34880A1992B218461146328064
:10AB600006F09CFE28603A464946204402F06CFDFF
:10AB7000B8F1000F09D031882868FFF767FF28680F
:10AB800006F016FB00232B60338003B0BDE8F08392
:10AB9000054E01930846318006F002FB019B2860B8
:10ABA0001C46E0E7FC9FFF1FF89FFF1F10B51F4CDE
:10ABB0004FF4FA70FBF742FD204601F0DFF9002266
:10ABC0001146204602F0C4F82046012102F0CAF8DE
:10ABD0002046002102F0C0F80B221549204602F061
:10ABE00051FA204602F064FA0F221249204602F080
:10ABF00049FA204602F05CFA0F490722204602F08B
:10AC000041FA204602F054FA204601F0C3FA0B4BF9
:10AC10000B4A1A604FF4FA70FBF710FDFFF722FEA3
:10AC20000848BDE81040FFF74FBE00BF709FFF1FF0
:10AC3000D03F0100DC3F0100EC3F010030A2FF1FCC
:10AC400041AB0000F43F01000020704790F839202C
:10AC500090F83800101A704790F8383090F8392082
:10AC60009A4205D95A1C034480F83820187E704750
:10AC70004FF0FF30704700BF90F8383090F839201F
:10AC80009A4286BF1B18187E4FF0FF30704700BFF6
:10AC9000704700BF38B50546B0F85E0090B195F832
:10ACA0005D301446C3F1210294420CD805F13B00FB
:10ACB0001844224602F0C8FC95F85D30234485F81C
:10ACC0005D30204638BD012014462871EEE700BFF4
:10ACD000B0F85E306BB190F85D30202B07D8C21809
:10ACE000013380F85D30012082F83B10704701236A
:10ACF00003710020704700BF0023426980F838309C
:10AD000080F8393080F85C3080F85D3080F85E3053
:10AD100080F85F3006CA30B40D68046943662A4380
:10AD200083660A60A370426990F86130164914681E
:10AD300013441D7A5B7B01EBC5051B026D6803F4B0
:10AD4000E06343F064032B6090F8623013449D7C11
:10AD5000DB7D01EBC5011B02496803F4E06343F0AE
:10AD600064030B6021685368194205D003692722E8
:10AD70005A70036904229A71036920225A71036987
:10AD800080229A7030BC7047284B010043690CCB7D
:10AD900012681A420CD0094B99420AD9084B9942C1
:10ADA000036994BF1A220D225A70036904229A7112
:10ADB0007047036927225A70F7E700BF7F1A060021
:10ADC0003F420F0010B50269D378DBB2D9060446C2
:10ADD0003DD510215806D17038D503F0040303F097
:10ADE000FF02002B51D03D49626E00230B7084F8A6
:10ADF0005D30002A5BD0904794F85D30002B56D030
:10AE00002369D0229A70236994F83B201A71236930
:10AE1000012284F85C200222DA7010BD304B84F8E5
:10AE200060009C424AD02F4B9C4252D094F839107B
:10AE300013791F29DBB207D82848007820B16018A1
:10AE4000013184F8391003760223D37010BD5906FE
:10AE5000C3D4917801F0100101F0FF000029DDD08A
:10AE600013F001031ED194F85C1094F85D00884241
:10AE700081BF4B1C091984F85C3091F83B30137189
:10AE80002369D0229A702269DEE7236984F8392089
:10AE9000C0229A702369114A197901211170022286
:10AEA000DA7010BDC023937022691379CCE70122B8
:10AEB000002384F85D2084F83B30A1E7626994F8B0
:10AEC0006130094913440322187A02F043FD2269D4
:10AED000ACE7626994F861300449F3E700A0FF1F12
:10AEE0005C91FF1FC891FF1F4DAF000059AF0000DC
:10AEF0000369DB7803F0200373B190F8603001330D
:10AF0000DBB2012B80F860301AD9426990F86130C9
:10AF10001344187A02F09ABD70B5426903F0FF0538
:10AF200090F8613013440446187A02F08FFDA36E46
:10AF30005BB184F8385094F83900BDE87040184788
:10AF400090F85F30002BE0D0704770BD0148FFF7EC
:10AF5000CFBF00BF5C91FF1F0148FFF7C9BF00BF13
:10AF6000C891FF1F2DE9F047374FDFF8E0903B68AD
:10AF7000026982B006460093DDF800800021A0251A
:10AF8000D3789B065BD53B680193019BC8EB030319
:10AF90000F2BF5D949B1102BF2D0002090703369F6
:10AFA00080229A7002B0BDE8F087726996F861302D
:10AFB00013440521187A02F043FF726996F8613054
:10AFC0001344012193F812A0504602F039FF0924DE
:10AFD0000021504602F020FF2B46013BFDD101210C
:10AFE000504602F019FF2B46013BFDD1013CEFD149
:10AFF000706996F8611001444FF4A0720C7A4B7B93
:10B0000009EBC4011B02496803F4E06343F06403E5
:10B010000B6096F862300344997CDB7D09EBC1013B
:10B020001B02496803F4E06343F064030B60013AD8
:10B03000FDD13269D3789B064FF00101A3D40120E2
:10B0400002B0BDE8F08700BF28A0FF1F284B010019
:10B05000F0B503691222DA700269937803F02003D5
:10B0600085B004460D46002B5ED0B42393703C4956
:10B0700022690B680093009E05E00B680193019B19
:10B080009B1B042B42D8D37803F0200303F0FF006E
:10B09000002BF2D094F85D30002B31D04FF0000E31
:10B0A0004FF0020C04EB0E0393F83B3013710B6866
:10B0B0000393039F206907E09B060DD50B6802935D
:10B0C000029BDB1B052B28D8C378DBB203F00202FE
:10B0D00002F0FF06002AEFD080F803C02669F3785B
:10B0E000DBB2DF0632462DD49F062BD5DB0731D4E9
:10B0F0000EF1010E94F85D305FFA8EFE7345D1D8E3
:10B1000000201DBB002384F85E3004E090702369AA
:10B1100080229A70042005B0F0BD867023698022D9
:10B1200004209A7005B0F0BD03F0FF06FFF71AFF88
:10B1300010B9042005B0F0BD236984F85F60B02227
:10B140009A7094E78023B3700420DAE7266980239D
:10B15000B370D7E7BEF1000F0CBF02200320F6E763
:10B1600028A0FF1F2DE9F04106690025122780F86D
:10B17000385080F83950F770D0F810C09CF802E0D1
:10B180000EF0200E88B00446884615461E46BEF1D5
:10B19000000F49D0B4238CF80230784B21691A682B
:10B1A0000092DDF800E006E01A6801920198CEEB0B
:10B1B0000000042830D8C87800F0200000F0FF0715
:10B1C0000028F1D04FEA480242F00102D2B20A71DF
:10B1D0001A680292DDF808E0206906E01A68039216
:10B1E0000399CEEB010105292AD8C17801F00201AB
:10B1F00001F0FF070029F1D04FF0020C80F803C0E6
:10B200002269D17811F0110722D12DBB002E0CBF7D
:10B21000A0238023937003E08F70236980229A70AB
:10B22000384608B0BDE8F0810EF0FF07FFF79AFE40
:10B230000028F5D0236984F85F70B0229A70ACE7DB
:10B2400087702369802238469A7008B0BDE8F08183
:10B25000802393700027E3E7012D75D0A021917022
:10B2600021690A79BE4667464FF0A80C1A68049215
:10B27000049805E01A680592059A121A052A4AD818
:10B28000CA7802F0020202F0FF08002AF2D0CF7062
:10B290002169CA78D2B212F0100F08465AD192062C
:10B2A00058D5013DEDB2012D49D0BEF11F0F3BD95C
:10B2B0000A79012DDAD11A680692069D05E01A680E
:10B2C0000792079A521B052A46D8C27802F002025A
:10B2D00002F0FF01002AF2D00223C3702269D37862
:10B2E000DBB2D9063AD49B0634D5B023BEF11F0F8A
:10B2F00093703FD8226904EB0E0312791A760EF18F
:10B30000010E5FFA8EFE16B1236980229A7084F8CE
:10B3100039E0774684E781F80280236980229A70B9
:10B32000774684F839E07BE704EB0E0291F804805D
:10B3300082F818800EF1010E5FFA8EFEB9E781F8EF
:10B3400002C021690846B0E7A82191702069BE4675
:10B350000279B0E7774663E78170DEE71021A0232A
:10B36000D170013BFDD12269937803F0F703774652
:10B37000937055E723691B79C5E700BF28A0FF1F1D
:10B380000148FFF71FBD00BF5C91FF1F0148FFF799
:10B3900019BD00BFC891FF1F704700BF38B5144CDE
:10B3A000037801225B000546204684F83B3084F890
:10B3B0005E2084F85D20FFF78BFC20460021FFF71C
:10B3C00047FE0B4C2978012320461A46FFF7CAFE98
:10B3D0000128F6D194F8383094F839209A4205D9EA
:10B3E000E218013384F83830107E38BDFF2038BDB4
:10B3F0005C91FF1F38B51B4C037801225B000546AA
:10B40000204684F83B3084F85E2084F85D20FFF706
:10B410005FFC20460021FFF71BFE124C29782046D6
:10B4200001230222FFF79EFE0228F6D194F838206D
:10B4300094F839108A420FD2531CDBB2A0189942FB
:10B4400084F83830007E0AD9234402321B7E84F807
:10B45000382040EA032038BD4FF6FF7038BD40F475
:10B460007F4038BD5C91FF1F0C2901D90020704737
:10B470000231490001F0FE01FFF7BCBF70B50C4C72
:10B480000378164601255B00204684F83B3084F89B
:10B490005E5084F85D50FFF71BFC31462046FFF7F5
:10B4A00017FC29462046BDE87040FFF7D1BD00BF1C
:10B4B0005C91FF1FF8B505460F461646412421460C
:10B4C0003A462846FFF7DAFF611C0234C9B2324619
:10B4D0002846E4B2FFF7D2FF592CF0D1F8BD00BFE7
:10B4E00038B504460D463548FFF706FC6322802137
:10B4F00020462570FFF7C2FF012002F0C9FC20465C
:10B5000000225E21FFF7BAFF20465D21FFF746FFCC
:10B51000242801D0002038BD204606220C21FFF748
:10B52000C9FF204601222B21FFF7A8FF2046012258
:10B530002C21FFF7A3FF20460E222D21FFF79EFFAF
:10B54000204600222E21FFF799FF204601222F21BD
:10B55000FFF794FF204605223021FFF78FFF20469A
:10B5600001223121FFF78AFF204600223221FFF716
:10B5700085FF204600223321FFF780FF204600226E
:10B580003421FFF77BFF204600223521FFF776FFAD
:10B59000204600225B21FFF771FF204610225C212C
:10B5A000FFF76CFF204620225D21FFF767FF204652
:10B5B0008F225E21FFF762FF012038BD5C91FF1FE3
:10B5C00010B4047F4160022CC26002D010BC01F0B4
:10B5D000D7BB836810BC184790E80C00F0B41C6817
:10B5E00059682568164F174E29432160164D174993
:10B5F0001760D66015611160417A154A5C180A31EE
:10B6000094F8244053F8215002EBC40149680D60BE
:10B61000017A5C1803EB8101247ECD6902EBC40141
:10B6200049680D60817A581803EB810390F8300067
:10B63000596B02EBC002F0BC53681960704700BF41
:10B6400001401F00011000380110007800001F8029
:10B65000284B0100704700BFF0B50C1EBDF8146008
:10B6600034DBB0F906701919B942C4BF3B1B1BB2D9
:10B67000002BA6461CDD002A1146B8BFD11D02F0E2
:10B680000705CC10826A012007FB04E1A840012EC7
:10B690000A44C0B21ED00CD3022E09D1013B12FACB
:10B6A00083F3013A12F8011F41409A421170F9D117
:10B6B000F0BDC043013B12FA83F3C0B2013A12F865
:10B6C000011F014093421170F9D1F0BD23441BB218
:10B6D0000024C6E7013B12FA83F3013A12F8011F76
:10B6E00001439A421170F9D1F0BD00BFF8B50D1EAB
:10B6F0000EDB14461F46064601F03AFBA84207DD62
:10B70000002C05DB304601F037FBA04201DCF8BD20
:10B71000F8BD304601F02AFB022853D003284BD055
:10B72000012806D16540F3886C406540013B5D1BF4
:10B730002DB2012F03D02AD3022F14D0F8BD002C34
:10B740002246B6F90630B06AB8BFE21D42F3CF0216
:10B7500002FB035504F00704435D012101FA04F4E0
:10B760001C434455F8BD002C2246B6F90630B06A99
:10B77000B8BFE21D42F3CF0202FB035504F00704F9
:10B78000435D012101FA04F45C404455F8BD002CEE
:10B790002246B6F90630B06AB8BFE21D42F3CF02C6
:10B7A00002FB035504F00704435D012101FA04F490
:10B7B00023EA04044455F8BD3389013B591B25464F
:10B7C0000CB2B6E7F18832890139013A4D1B141BDE
:10B7D0002DB224B2ADE700BF2DE9F041079E9DF9DF
:10B7E0001880089D04461F4600F0C0FF0D4B0E4810
:10B7F0000E4984F83380FF22002F08BF1F4684F8CB
:10B800002F20002384F8302084F8312084F832205F
:10B810002060A665E565676261652362A3622046D4
:10B82000BDE8F0815C91FF1F8040010001100138EC
:10B8300010B50446806A034B236008B105F0B8FCDC
:10B84000204610BD80400100F8B5436ADBB190F896
:10B850002C200125AA4083F83B2083F85E5083F812
:10B860005D500446406A03680E461B6800219847F5
:10B87000606A036831461B6898472946606ABDE8DC
:10B88000F840FFF7E5BBC26BC56C1368046A23EA96
:10B89000050313604CB122684FF00043D36251633B
:10B8A000D36A002BFCDA936BF8BD836B466B0825DB
:10B8B000802410E03768426C3A4332601F68826C23
:10B8C0003A431A601A68876C013D22EA07024FEA80
:10B8D00054041A6007D02142ECD13268476C22EA46
:10B8E00007023260EAE7F8BD70B50446406A0D46CB
:10B8F00000282BD0A16DFFF749FA002D20460CBF80
:10B90000A621A721FFF7A0FF606A20B1E16DBDE885
:10B910007040FFF73BBA216C226D0868236A02432E
:10B920000A6093B1DA7A82B1D00703D5224A9969C5
:10B930001160DA7A910703D5204AD9691160DA7A61
:10B94000520702D51E4A1B6A136070BD236A002B82
:10B950002BD0D97A626DE1B172B6D97ACE0706D50D
:10B960001848D9680668314099610160D97A88071A
:10B9700006D51548196906683140D9610160D97A40
:10B980004E0705D5114859690668314019620160B2
:10B9900062B61B68D968914207D00D4818600D49FE
:10B9A000DA6042F0804018611960226C216D1368E2
:10B9B00023EA01031360A0E700E100E004E100E0F6
:10B9C00008E100E080E100E084E100E088E100E0DF
:10B9D00001403F0000003F80436A2DE9F0410546E9
:10B9E0000E469046002B3ED090F82C100124A1402A
:10B9F00083F83B1083F85E4083F85D40406A03683B
:10BA000000211B6808F1FF379847FFB2B8F1000F1B
:10BA100023D03744A046013E686A16F8011F036828
:10BA20001B6898470134B742E4B216D0202CF3D1FA
:10BA30000121686AFFF70CFB95F82C206B6A520015
:10BA400083F83B2083F85E8083F85D80686A036832
:10BA500000211B6898470124DEE7686A0121BDE8E0
:10BA6000F041FFF7F5BAC26BC16C136823EA01031A
:10BA700006EB080413604FF00048A6420ED02B6A74
:10BA800016F801EB63B11A68C2F82C80C2F834E0F2
:10BA9000D36A002BFCDAA642936BF0D1BDE8F081AB
:10BAA000AB6BD5F834C008208021DCF800206F6C27
:10BAB0001EEA010F14BF3A43BA43CCF800201A68BB
:10BAC000AF6C3A431A601A68AF6C013822EA070279
:10BAD0004FEA51011A60E8D1CFE700BF70B50446C4
:10BAE000406A0D46002828D0A16DFFF74FF9204687
:10BAF0002946FFF7A9FE606A20B1E16DBDE87040FC
:10BB0000FFF744B9216C226D0868236A02430A607A
:10BB100093B1DA7A82B1D00703D5234A99691160CB
:10BB2000DA7A910703D5214AD9691160DA7A520786
:10BB300002D51F4A1B6A136070BD236A002B2BD0ED
:10BB4000D97A626DE1B172B6D97ACE0706D51948B5
:10BB5000D9680668314099610160D97A880706D5AD
:10BB60001548196906683140D9610160D97A4E07D4
:10BB700005D512485969066831401962016062B6FC
:10BB80001B68D968914207D00D4818600D49DA60EA
:10BB900042F0804018611960226C216D136823EA1D
:10BBA00001031360A3E700BF00E100E004E100E04F
:10BBB00008E100E080E100E084E100E088E100E0ED
:10BBC00001403F0000003F802DE9F041044686B06F
:10BBD000806A9DF830801E460F461546B4F908303D
:10BBE000002800F04281DA1D48BF03F10E02B4F9CB
:10BBF0000630D21003FB02F2002105F0FDFDB4F97E
:10BC00000820202A00F39280B4F90610A34B0120EB
:10BC1000203A733902EBD27201EBD1714FF0200E52
:10BC2000029073208DE8014042F34F0241F34F012F
:10BC3000204600F051FE606A84F82D70002800F064
:10BC40004D81002D40F08A80B4F90830202B14BFBC
:10BC50003D253C2584F82C50B8F1000F40F085803C
:10BC600006B394F93300002818DBC0B2012102F0BA
:10BC7000E7F8012194F8330002F0CEF8012002F039
:10BC800007F9002194F8330002F0C6F80A2002F008
:10BC9000FFF8012194F8330002F0BEF8606A002832
:10BCA00000F08280A16DFFF771F804227C492046E4
:10BCB000FFF792FE217A0139C9B22046FFF7C4FD91
:10BCC000784904222046FFF787FE94F92D30012B96
:10BCD00014BF142110212046FFF7B6FD042272493B
:10BCE0002046FFF779FEB4F90630802B00F09280F1
:10BCF000602B00F0A680D9212046FFF7A5FD94F91E
:10BD00002D30012B14BFF12122212046FFF79CFD8D
:10BD1000204606226549FFF75FFE606A50B3E16D79
:10BD2000FFF734F8012006B0BDE8F081B4F9061041
:10BD30005F4B0120403A52394FF0400E029002EB27
:10BD4000D272522001EBD1718DE8014042F34F02D3
:10BD500041F34F01204600F0BFFD6CE76DB284F85F
:10BD60002C50B8F1000F3FF47BAFFEF7C5FF002E5B
:10BD700094D076E7216C226D0868236A02430A603A
:10BD800073B1DA7A62B1D00703D54A4A9969116072
:10BD9000DA7A91077CD4520702D5474A1B6A1360AE
:10BDA000012006B0BDE8F081236A002B2BD0D97AA0
:10BDB000626DE1B172B6D97ACF0706D53F48D9682E
:10BDC0000568294099610160D97A8E0706D53C48FB
:10BDD000196905682940D9610160D97A4D0705D5EF
:10BDE00038485969056829401962016062B61B68C4
:10BDF000D968914207D0344818603449DA6042F07B
:10BE0000804018611960226C216D136823EA0103D8
:10BE100013604AE7B4F90830202B00F08680402BED
:10BE20007FF469AF2A4920460322FFF7D5FD94F934
:10BE30002D30012B14BFCF219F212046FFF704FD99
:10BE400059E7B4F90830102B7FF455AF214920464B
:10BE50000322FFF7C1FD94F92D30012B14BFAF2150
:10BE600010212046FFF7F0FC45E7DA1D48BF03F13B
:10BE70000E02B4F90630D21003FB02F2104605920E
:10BE800005F08EF9A06200283FF44DAF059AB3E6A5
:10BE9000114AD9691160DA7A7DE700BFD840010004
:10BEA000B8420100BC420100C0420100C44201008E
:10BEB000CC42010000E100E008E100E080E100E0A8
:10BEC00084E100E088E100E001403F0000003F80A5
:10BED000D44001008C45010004E100E0012194F808
:10BEE0003100244F01F0ACFF94F83200012101F041
:10BEF000A7FF94F9312094F9323057F83220E263E9
:10BF000057F83330206A23640125E56425651A68F3
:10BF10002A431A6078B1B8F1000F3FF428AFFFF759
:10BF20005BFB002E3FF4BAAE9BE60422124920468A
:10BF3000FFF752FDDFE6294694F82F0001F080FF5D
:10BF4000294694F8300001F07BFF94F92F2094F9F2
:10BF5000303057F83220626357F833306564A56497
:10BF60001A68A36322F001021A60002E3FF496AE15
:10BF700077E600BF284B0100D0400100B0F908204F
:10BF8000D31D48BF02F10E03B0F90620806ADB1012
:10BF900002FB03F2002105F02FBC00BFF0B5002921
:10BFA000BDF814502EDBB0F90660B1422ADA002A3F
:10BFB00059DBB0F9087014461C44BC42C4BFBB1A1C
:10BFC0001BB2002B1EDDD2B2D408D0F828E016FB3D
:10BFD000041112F00702DBB20EEB010421D0C2F112
:10BFE0000807FAB2374F9342BF5C0CD2C3EB020C86
:10BFF000FF2646FA0CF6012D07EA06073FD005D3C7
:10C00000022D36D0F0BD012D39D030D21EF801609E
:10C0100026EA07070EF801709342F3D3B0F9061031
:10C020000C449A1AD2B2072A10D9022D36D0002D0C
:10C0300014BFFF26002613462670083BB0F90610F1
:10C04000DBB2072B0C44F7D802F00702002AD9D044
:10C050001D4B012D9B5C1DD017D3022DD2D1227810
:10C0600053402370F0BD13441BB20022A1E7022D00
:10C0700025D11EF8016077400EF80170CCE71EF85C
:10C08000016037430EF80170C6E7227822EA030305
:10C090002370F0BD227813432370F0BD114623783E
:10C0A000DB4323700839B0F90630C9B207291C44B4
:10C0B000F5D812F00702A5D0034B9B5CCFE73444C0
:10C0C000AFE700BF704001006040010070B4C47D64
:10C0D000BDF80C50022C18D0032C1FD0012C0BD013
:10C0E000002A03DBB0F90840944201DC70BC7047C1
:10C0F000039570BCFFF7B0BAC4880395013CA41A3D
:10C100000A4621B270BCFFF749BF0689C488013EC8
:10C11000641AB21AE41A12B221B2E1E70489039553
:10C12000E41A641A114622B270BCFFF737BF00BF91
:10C1300070B4C57DBDF80C60022D1AD0032D12D04D
:10C14000012D03D0039670BCFFF728BFC488E41A02
:10C15000A41A0A4621B2002A03DBB0F9084094422F
:10C1600013DC70BC70470489013C641A114622B28A
:10C17000F1E7C48805890396013CAD1AED1A621AED
:10C1800011B22AB270BCFFF709BF039670BCFFF76B
:10C1900063BA00BF2DE9F8430446406A002863D023
:10C1A000A16DFEF7F3FD052274492046FFF714FC4C
:10C1B000A1790139C9B22046FFF746FBB4F908203E
:10C1C000E588A66AD31D48BF02F10E03DB10626A40
:10C1D00015FB03F51FFA85F8002A7BD094F82C3064
:10C1E0000125AB4082F83B3082F85E5082F85D500A
:10C1F000606A036840211B6808F1FF379847BFB2A7
:10C20000B8F1000F23D03744A846013E606A16F803
:10C21000011F03681B6898470135B742EDB216D07D
:10C22000202DF3D10121606AFEF712FF94F82C2033
:10C23000636A520083F83B2083F85E8083F85D8058
:10C24000606A036840211B6898470125DEE70121E9
:10C25000606AFEF7FDFE606A002800F08D80E16DE7
:10C26000BDE8F843FEF792BD236A002B2BD0D97AA4
:10C27000626DE1B172B6D97ACE0706D54048D96869
:10C280000568294099610160D97A8D0706D53D4836
:10C29000196905682940D9610160D97A480705D52F
:10C2A00039485969056829401962016062B61B68FE
:10C2B000D968914207D0354818603549DA6042F0B4
:10C2C000804018611960226C216D136823EA010314
:10C2D000136068E7E26BE36C1168276A0B4306EBB7
:10C2E000080913604FF0004E4E450DD016F801CBF3
:10C2F0002FB33A68C2F82CE0C2F834C0D36A002BDE
:10C30000FCDA4E45936BF1D1226C236D11680B431F
:10C31000136097B1FB7A83B1D90703D51D4BBA6976
:10C320001A60FB7A9A0703D51B4BFA691A60FB7AED
:10C330005B0702D5194B3A6A1A60BDE8F883A36B14
:10C34000D4F8348008208021D8F80020656C1CEADD
:10C35000010F14BF2A43AA43C8F800201A68A56C2D
:10C360002A431A601A68A56C013822EA05024FEACE
:10C3700051011A60E8D1B7E7276AC5E768400100B4
:10C3800080E100E084E100E088E100E001403F005E
:10C3900000003F8000E100E004E100E008E100E08F
:10C3A0002DE9F04F85B09946BDF93870BDF83CA035
:10C3B000BB1AC1EB090B002BB8BF5B42BBF1000FEE
:10C3C000B8BFCBF1000B5B450D4616460093804687
:10C3D00048DC4D453A4633464CDC194613460A467E
:10C3E000C5EB09019B1A89B2002B0CB2B8BF5B42A6
:10C3F00004EBD474BE42ACBF4FF0FF3201224D4576
:10C40000039102924FEA640429DC9BB201930DE090
:10C41000D8F80070BF69B847019BE41AA3B21CB2F8
:10C420000135002C2DB211DBA94518DB009B5B45C3
:10C430002A46534631464046EADCD8F800205346A7
:10C440009769294632464046B847E5E7029A1644BE
:10C45000039AA94502EB030436B224B2E6DA05B02A
:10C46000BDE8F08F4A462B46B94635464D4517463E
:10C470001E46B2DD304629463E464D4607468946B1
:10C48000AEE700BF10B404682469A44610BC60473E
:10C4900030B40468BDF808500295A46BA44630BCC3
:10C4A000604700BF30B40468BDF808500295E46BE3
:10C4B000A44630BC604700BF70B40468BDF90C608E
:10C4C000BDF8105003960495246CA44670BC6047D8
:10C4D000704700BF10B582B0B0F90C20019101681F
:10C4E000009200220C6CB0F90A301146A04702B04D
:10C4F00010BD00BF704700BF01F003010129C175E5
:10C5000006D0032904D0C288038942818381704701
:10C510000289C38842818381704700BF2DE9F041C1
:10C520000568134E6F6986B0B7420446BDF8308087
:10C5300010D1013B13441BB20093CDF804800B468D
:10C54000AD6A2046A8472368DB6AB3420AD106B029
:10C55000BDE8F081059304920391B84703A92568CB
:10C560000EC9E6E7204606B0BDE8F041184700BF17
:10C57000D1C400002DE9F0410568124E6F6986B004
:10C58000B7420446BDF830800FD1013BCDF804809E
:10C590000B4400921BB2AD6A2046A8472368DB6AB1
:10C5A000B3420AD106B0BDE8F0810593049203912D
:10C5B000B84703A925680EC9E7E7204606B0BDE8DD
:10C5C000F0411847D1C400002DE9F04F0568DFF8AD
:10C5D00058B06F6985B05F450646BDF93890BDF823
:10C5E0003CA00C46904615D11F19BC420CDACDF880
:10C5F00000A0214601342D6A4B464246304624B203
:10C60000A847BC423568F2DBEB6A5B4507D105B051
:10C61000BDE8F08F0393B8473568039BE4E73046E5
:10C6200005B0BDE8F04F1847D1C400002DE9F04334
:10C6300087B099420546BDF93840BDF83C6025D029
:10C64000A24212D00768DFF88080D7F81490C14565
:10C6500032D18DE850002846BC6AA0472B68DB6ABF
:10C66000434524D107B0BDE8F083994202DD084676
:10C670001946034628680E96C46B01335B1A1BB239
:10C680002846A44607B0BDE8F0436047A24202DD59
:10C69000134622461C4628680E96631C846B9B1A20
:10C6A0001BB22846A44607B0BDE8F04360472846C1
:10C6B00007B0BDE8F0431847059304920391C847BB
:10C6C00003A92F680EC9C4E7D1C400002DE9F04FBB
:10C6D000D0F800E0DFF89090DEF814B083B0CB45DE
:10C6E0000446BDF93080BDF834A00D4617461E46FD
:10C6F00031D1CDF800A0DEF824B0294633463A46C1
:10C700002046D8472368CDF800A008F1FF323A440C
:10C71000D3F824B0294612B233462046D8472368BE
:10C72000CDF800A02946D3F820B03A46434620462B
:10C73000D8472068CDF800A0711E29444346056AF9
:10C7400009B23A462046A8472368DB6A4B4506D122
:10C7500003B0BDE8F08FD847D4F800E0C9E7204621
:10C7600003B0BDE8F04F1847D1C40000F0B4002476
:10C7700001264FF6FF75094F07600471C475C48127
:10C7800004824476C4618675067685824582C180BE
:10C79000028141818281F0BC704700BF9845010051
:10C7A0002DE9F04F85B00668BDF84450BDF93880DA
:10C7B000CDF8008004460195D6F848B00392BDF943
:10C7C0003C60BDF9407089469A46D8472368019578
:10C7D000009742465146D3F8488020463346C0472A
:10C7E0002068039B0E930F95856C4B463A46314665
:10C7F0002046AC4605B0BDE8F04F60472DE9F04F4C
:10C8000087B01746BDF9404000912546E91D0593C4
:10C8100044BF2B4603F10E010268BDF8486053691E
:10C820000294C91003912B49BDF9444001968B42F3
:10C83000824645D1002C3CDD029B3C445E1EB6B2D4
:10C840004FF0000923B2049301364D46029B002BA2
:10C8500028DD059B002403EB090806E0EDB22B065A
:10C8600004F1010411D4A6421CD0A1B211F0070FAB
:10C8700023B24FEA4505F1D1002BB8BF0733DB10D7
:10C88000013418F803502B06EDD5009BD2F818B0F0
:10C8900019443A4609B2019B5046D847A642DAF8F5
:10C8A0000020E2D1039B01379944049B3FB2BB4275
:10C8B000CCD1D36A074A934206D107B0BDE8F08FC6
:10C8C0009847DAF80020B5E7504607B0BDE8F04FCA
:10C8D000184700BFD1C4000070B4BDF90C60BDF9A9
:10C8E0001050BDF8144003960495059470BCFFF7F2
:10C8F00085BF00BF2DE9F04F93B090460591C16907
:10C900001090BDF870000790BDF874909DF878A065
:10C910000493002900F0CD800A7A0AC98946049957
:10C920008A1AD2B203EBC203BAF1010FDA780B9282
:10C9300093F905201E8893F802B00F9293F90640F0
:10C9400079D913B2099323B20C93109B1A68A94B9F
:10C950001193194653698B4240F0A6800B9B002B24
:10C9600055D01FFA88F300210D93C8462344DDF803
:10C97000409006910E930F460C46BBF1000F3FD03E
:10C98000BDF818100C9B03971FFA8AF0CB1813FB05
:10C9900000F304900E9801440D98034409B21BB2B1
:10C9A0000A910893002505E00135EBB264009B4530
:10C9B000E4B222D9039B2B44590703D1731C18F806
:10C9C00006409EB22306EFD5099BBDF81000E9187A
:10C9D00011FB00F10598BAF1010F0FFA8AF3014437
:10C9E0001CD0079801900093D26909B217464846B7
:10C9F000089AB847D9F80020D6E7039F5F44FFB2F2
:10CA0000069B0B9901330693DBB29942B5D8D36AE2
:10CA1000119A934243D113B0BDE8F08F0F9B1918C0
:10CA200093690A9A29441F4609B2079B4846B847AA
:10CA3000D9F80020B8E700230C93099385E70A9AF8
:10CA40000D9B0132013B52B213F0FF030A920D938A
:10CA50006FD1DDF81890079BDDF83C80DDF820A051
:10CA60004B4517D0BAF1010F00F0C8800B9A109D0A
:10CA7000CDF804900BEB8B014FEACB030A440093F3
:10CA80001146DEF81C405346424609B22846A047EC
:10CA9000D5F800E0DEF82C30119A9342BBD0109804
:10CAA00013B0BDE8F04F1847109D284698472A68F4
:10CAB00054E7109A0598B2F90A308342ABDDB2F917
:10CAC0000C304345A7DD062313FB0A03002BA2DD30
:10CAD00008EBCA03002B9EDD537E2BB9049BAF2BC2
:10CAE00002D90133DBB20493109BD3F800E0414B31
:10CAF00011931A46DEF81430934240F08E801FFAEC
:10CB000088F30E9308339BB2BDF8142005930523D8
:10CB10000D9300230A93CDF83C800FFA8AF3DDF8D9
:10CB20004080CDF818900B921FFA8AFBCDF820A018
:10CB300099460A9ABDF810000B9C0E9D05231946D4
:10CB400011FB00232C481146C75C039702FB0B42E4
:10CB500014FA81F312B21BB209920C932C462E46A2
:10CB60001CE0089B0999012B2AB24B4640462DD068
:10CB7000079F0197CDF80090DEF81CA0D047D8F8A9
:10CB800000E0039B5B0801340393059BA4B25D4462
:10CB90005E44A342ADB2B6B23FF451AF039BD80797
:10CBA000DFD4079B069A9342EBD0089B012B16D04B
:10CBB000069B0193CDF80090DEF81CA009994B4626
:10CBC00032B24046D047D8F800E0DAE7DEF818A0E5
:10CBD000079B0C9922B2D047D8F800E0D1E7DEF8E5
:10CBE00018A00C991346404622B2D047D8F800E06E
:10CBF000C7E700BFD1C40000E84501000B99109DB4
:10CC0000CDF800900531DEF8204009B242460823F5
:10CC10002846A047D5F800E03CE7109C20469847FE
:10CC2000D4F800E06BE700BFF0B5C36985B00446F7
:10CC30002BB30A2968D00D294AD01A7A914247D3DA
:10CC4000587A884244D35D688A1A05EBC205AA78EF
:10CC5000002A50D0E87800284DD0207E00283AD015
:10CC600095F905E0B4F90E00A67DB4F90A70724496
:10CC700006FB0202BA4262DCB4F9102030E00A2955
:10CC800056D00D2924D0027E002A4BD0B0F90E00D8
:10CC9000A57DB4F90A60062212FB0502B2423EDD10
:10CCA000228AE38102EBC50212B218462282A78AC9
:10CCB000668A02950B468DE8C00001462046FFF7C4
:10CCC00019FEA37DE28903EB430302EB4303E381F7
:10CCD000012005B0F0BDA67DB4F90E00B4F9102016
:10CCE000B4F814E0678A02960B468DE8804001464E
:10CCF0002046FFF7FFFD2979E389A27D012001FB92
:10CD00000233E38105B0F0BD0022C2819A7A817DB1
:10CD1000038A01FB02330382012005B0F0BDB4F9A0
:10CD20001020C4E7857DB4F91020B0F90E00BEE7ED
:10CD3000028A817DC38102EBC1030382C8E7002020
:10CD4000E0819B7A228A03FB062212B22282C7E785
:10CD5000C1810282704700BF002908BF012181758F
:10CD6000704700BF81824182704700BFC07D70471D
:10CD7000B0F90A00704700BFB0F90C00704700BF5F
:10CD800010B4EFF3108272B6437F33B9017F0129EB
:10CD900007D003290FD00123437702B962B610BC34
:10CDA0007047124C2168A1B1114943610B6883613E
:10CDB00008605861EFE70F4C216881B10E4943616B
:10CDC0000B688361086058610C4B4FF0805119600B
:10CDD000E1E7074B4161816120601860DBE7064BAA
:10CDE0004161816120601860EEE700BF14A0FF1F61
:10CDF00010A0FF1F04A0FF1F08A0FF1F04ED00E00C
:10CE000070B5EFF3108272B60C4C206880B10C4EF6
:10CE100000254369236073B19D6102B962B645770D
:10CE200083689847EFF3108272B620680028F0D12B
:10CE300002B962B670BD3360EFE700BF04A0FF1F08
:10CE400008A0FF1FFFF7DCBF184A30B41468002C9D
:10CE500027D0036821688B420ED2CB1A0021846050
:10CE6000C1602360E06010600223037530BC70472E
:10CE700011688B42144608D3A2685B1A0360002A2B
:10CE8000F6D18260C460A060EEE7D268C2608460C0
:10CE9000E060C568CB1A0222A8602360027530BC2E
:10CEA00070478460C4601060DEE700BF0CA0FF1F05
:10CEB000F8B5224E34682CB32368002B3AD1204FAA
:10CEC0001D4604E03468ECB12368002B32D1A3681E
:10CED00003B1DD6020693360036825751B68BB42C0
:10CEE00021D1037F4560022BC46020D0FFF748FFAB
:10CEF0006368002BE6D023602046FFF7A5FF346867
:10CF0000002CE1D1EFF3108372B60E4A00211068B5
:10CF1000116003B962B628B18468FFF795FF204617
:10CF20000028F9D1F8BD224600219847E0E7836840
:10CF30009847DDE7013B2360E4E700BF0CA0FF1F3B
:10CF4000C1B500001CA0FF1F024A13680133136023
:10CF5000FFF7AEBF28A0FF1F704700BF0368F0B403
:10CF6000FBB1002501249D60DC601B4C1A601C4451
:10CF7000241104F144056A11032692009E60174FA4
:10CF80000679174B47F8241002F1604202F561421E
:10CF900005F01F05012000FA05F5E6541560F0BC08
:10CFA0007047104C236843F40003236000BF0E4B0E
:10CFB0000E4DA4F58734A4F59E7401261E60234609
:10CFC00004609C68002CD0D01033AB420360F8D1D1
:10CFD000002303601846E2E7008FFCBF3492FF1F76
:10CFE00044E400E03C800440007003404071034092
:10CFF0000168A9B10B4BF0B40B441B110A4E0B4F47
:10D000000B4D46F8237003F1440202F01F04012384
:10D010005211A340002445F822308C600460F0BC1B
:10D02000704700BF008FFCBF3492FF1F59CF000034
:10D0300080E100E0024A034B012111601B681847A0
:10D040000C7103403492FF1F024A034B012111600F
:10D050005B6818471C7103403492FF1F024A034B60
:10D06000012111609B6818472C7103403492FF1F07
:10D07000024A034B01211160DB6818473C710340F1
:10D080003492FF1FF8B50E4671B17AB107461446C7
:10D0900000253B6816F8011B1B6838469847013C81
:10D0A0000544F6D12846F8BD0846F8BD1046F8BD3F
:10D0B00000B5064A036812885B6883B001A9ADF821
:10D0C00004200222984703B05DF804FBE84A0100FF
:10D0D000F0B507468BB0002A33D0012A08BF0A22D8
:10D0E00051B3212400E0F4B2B1FBF2F502FB1511BB
:10D0F000C8B2092900F1300198BFC8B20AA988BF97
:10D100003730214488BFC0B201F8240C661E29467E
:10D11000002DE8D133B1013CE4B20AAB23442D2207
:10D1200003F8242C3B6801AA11195B683846C4F146
:10D13000220298470BB0F0BD30228DF82520212423
:10D14000E8E70368C9B21B6898470BB0F0BD00BFA1
:10D150000029BABF49422D2300230A22FFF7B8BF96
:10D16000374A384913681B06FCD40B6813F0800358
:10D17000F8D172B634490A78002A5FD0334A34486D
:10D18000F0B4344C176806682568D4680C303E4407
:10D19000143200681268304F35442C442044024455
:10D1A000C2F34E022D4E2E482E4D2F4C42F400421B
:10D1B0003A60376806682D682C4A24680C303E4473
:10D1C000006812682A4F35442C4420440244C2F3BC
:10D1D0004E02284E2848294D294C42F400423A601C
:10D1E000376806682D68274A24680C303E4400687A
:10D1F0001268254F35442C4420440244C2F34E02A9
:10D20000224E2348234D244C42F400423A603768B2
:10D2100006682D68214A24680C303E440068126874
:10D2200035442C4420440244C2F34E021C4842F4CC
:10D23000004202600B7062B6F0BC704762B6704785
:10D2400024B0034024B00B4021A0FF1F38B003409E
:10D250003CB0034040B003402CB0034058B0034002
:10D260005CB0034060B0034064B003406CB0034066
:10D2700030B0034038B00B403CB00B4040B00B40E6
:10D2800044B00B404CB00B402CB00B4058B00B409E
:10D290005CB00B4060B00B4064B00B406CB00B4016
:10D2A00030B00B4030B42948294A2A4B2A4D60241B
:10D2B000E121047011701B78284C082B30D00A2B08
:10D2C0002748284937D00C2B0CBF35223D2212238A
:10D2D0002A60236002600B60234B24491B78244A98
:10D2E000BBB101230B601360224B23491B78234AF7
:10D2F000012B26D9042B0FD9082B1ED9102B94BF34
:10D30000862387230B6013601D4B01221A7030BCEB
:10D3100070470B601360E7E784230B601360F3E74B
:10D3200000F58E200F490830012213232A60236064
:10D3300002600B60D0E73922F7E785230B601360AA
:10D34000E2E780230B601360DEE700BF0040074088
:10D35000014007404492FF1F08B003400CB0034057
:10D3600008B00B400CB00B4024A0FF1F20B00340BE
:10D3700020B00B404592FF1F24B0034024B00B4067
:10D3800021A0FF1F0C2830B417D91023984228BFC2
:10D3900018461C46104A114D1178181A8C422870F4
:10D3A00018D00F4913700B7823B10E490E4A002391
:10D3B0000B60136030BCFFF775BF0A2802D90C233D
:10D3C0001C46E7E7082802D90A231C46E2E708239F
:10D3D0001C46DFE730BC70474492FF1F20A0FF1FB0
:10D3E00021A0FF1F24B0034024B00B4028282FD8D1
:10D3F000334B2DE9F0411E5CFF2E2BD0314B1B78B7
:10D40000002B2AD132062CD472B62F4D2F4C2F462A
:10D41000012326602B7062B672B623681B060CD4FB
:10D420003B781BB9F4E72B78002BF1D062B602F001
:10D4300073FB72B623681806F5D5254B1B680022CE
:10D440002A7062B6234A107843FA00F0BDE8F081F2
:10D45000002070470020BDE8F081FFF781FE320612
:10D46000D2D572B61C4DDFF87C801C4C06F040070C
:10D47000FFB206F03F06D8F80030DFB123F010030A
:10D48000C8F8003001232660134A2B7062B672B6CA
:10D49000236819060CD413781BB9ECE72B78002B02
:10D4A000E9D062B602F038FB72B623681B06F5D5E8
:10D4B0000B4BC3E743F01003C8F80030E2E700BFAE
:10D4C000EC4A010021A0FF1F23A0FF1F00B0034072
:10D4D00010B0034020A0FF1F22A0FF1F00B00B4090
:10D4E00010B00B400CB00B400A4A0B49136843F4D0
:10D4F000805313600B7843B9084BC0221A70084B55
:10D5000080F30C0000B218807047044B80221A7020
:10D51000F5E700BF2C80044024A0FF1F21C00C4071
:10D5200000C00C40F0B51B4B1B4E596818689A6838
:10D53000DB6885B06C460FC4337899071DD5174A50
:10D54000174C1378174913F0700318BF1370164A5D
:10D55000164B8027177000263320032226706D4655
:10D5600008701A7072B6043C45F001052046A847C1
:10D5700062B6237813F0700309D10D4B064901E020
:10D58000013B02D00A78D207FAD505B0F0BD23706E
:10D5900005B0F0BD184B0100010002400000024040
:10D5A000040002400B000240070002400A00024053
:10D5B000410D0300B0F5006F0AD210B5094B1B787E
:10D5C000DB07044606D504F1A0500078C0B210BDB8
:10D5D00000207047FFF7A6FF04F1A0500078C0B20A
:10D5E00010BD00BF01000240B0F5006F17D238B582
:10D5F0000F4B1B78DA070D46044611D504F1A050F5
:10D600000378AB420AD00B4A137813F0700318BFAB
:10D610001370074A05701378DB07FCD538BD7047D7
:10D62000FFF780FF04F1A0500378AB42EBD1F5E7A0
:10D63000010002400000024008B5F4F703FBF4F7D4
:10D640006BFF02F069FAFAE7844641EA000313F03F
:10D6500003036DD1403A41D351F8043B40F8043BF9
:10D6600051F8043B40F8043B51F8043B40F8043BBC
:10D6700051F8043B40F8043B51F8043B40F8043BAC
:10D6800051F8043B40F8043B51F8043B40F8043B9C
:10D6900051F8043B40F8043B51F8043B40F8043B8C
:10D6A00051F8043B40F8043B51F8043B40F8043B7C
:10D6B00051F8043B40F8043B51F8043B40F8043B6C
:10D6C00051F8043B40F8043B51F8043B40F8043B5C
:10D6D00051F8043B40F8043B403ABDD2303211D3FC
:10D6E00051F8043B40F8043B51F8043B40F8043B3C
:10D6F00051F8043B40F8043B51F8043B40F8043B2C
:10D70000103AEDD20C3205D351F8043B40F8043BFB
:10D71000043AF9D2043208D0D2071CBF11F8013BF9
:10D7200000F8013B01D30B8803806046704700BFBF
:10D73000082A13D38B078DD010F003038AD0C3F1CE
:10D740000403D21ADB071CBF11F8013B00F8013BB0
:10D7500080D331F8023B20F8023B7BE7043AD9D36F
:10D76000013A11F8013B00F8013BF9D20B78037044
:10D770004B7843708B7883706046704708B5104CC7
:10D7800008E0236859050DD423681A050FD42368CF
:10D79000DB0411D423685803F3D501F065F823683E
:10D7A0005905F1D502F01CFA23681A05EFD500F0EF
:10D7B0007FFD2368DB04EDD500F0C8FEEAE700BF7B
:10D7C0003480044008B5FFF7D9FF00BF014B102299
:10D7D0001A80704700200540704700BF094908B50E
:10D7E0000B6830B16A461844A2F58052904202D2CA
:10D7F0000860184608BD03F0A5FC0C2303604FF039
:10D80000FF3008BD4892FF1FFEE700BFEFF3138013
:10D8100070B9EFF310836BB9EFF305825AB94FF487
:10D820008070EFF311832BB1984228BF18467047E0
:10D830004FF0FF3070470F2A01D81846F1E7014B2F
:10D84000D05CEEE7F0E300E0F0B44D1E2E4600247D
:10D8500000E00134B0FBF2F302FB1300092800F1F1
:10D8600030078ABF3730F8B2C0B206F8010F184649
:10D87000002BEED10A1953704CB1107815F8016FD6
:10D8800028700133E01A834202F80169F5DB08468B
:10D89000F0BC7047704700BF10B40F4B53F83020F6
:10D8A00092F880422CB1012369B182F8803010BC1B
:10D8B000704703EBC0035B681A6841B922F00202AB
:10D8C0001A6010BC704782F8003110BC704742F0FB
:10D8D00003021A6010BC7047284B01001C4A02EB7F
:10D8E000C00301295B6811D004291BD052F8300015
:10D8F000002280F8802229B1022920D0032922D0D9
:10D900001A6070474FF480721A60704752F8300006
:10D910004FF4A27280F880121A601A6822F0200276
:10D920001A60704752F830104FF4A272012081F84B
:10D9300080021A601A6842F020021A60704740F2B2
:10D9400003121A6070474FF481721A60704700BF6B
:10D95000284B0100212848D8F8B5042A44D8DFE82C
:10D9600002F0484B4E0345004FF410262B4B03EBBF
:10D97000C0030D465C68216811F4E06148D0284B73
:10D98000284A2949C3F89C2104F140422748C3F89A
:10D99000A411A2F59221264FC3F8A0017C292548A5
:10D9A000C3F8A871C3F8AC012CD9A2F594237C2B41
:10D9B0002AD9A2F596237C2B28D9A2F598237C2B73
:10D9C00029D9A2F59A227C2A27D81B4872B6236847
:10D9D00023F4702343F08072C4F384011643236060
:10D9E00040F82150266062B6F8BD70474FF43026EB
:10D9F000BCE74FF40026B9E74FF44026B6E74FF4F2
:10DA00002026B3E70D48E1E70D48DFE70D48DDE7E5
:10DA1000FFF764FFB3E70C48D8E7F8BD284B0100D7
:10DA20000082FF1FF188FF1F9988FF1FC588FF1F15
:10DA30006D88FF1F4188FF1F2493FF1F4C92FF1F1B
:10DA40008492FF1FD492FF1F0493FF1F1A4B03EB16
:10DA5000C00010B4426802F14043A3F592217C2932
:10DA600023D9A3F594217C290DD9A3F596217C29EE
:10DA70001FD9A3F598217C2919D9A3F59A237C2BCA
:10DA800011D80E4C00E00E4C72B613680D4823F00E
:10DA90008773C2F3840123F4803343F080731360EF
:10DAA00044F8210062B610BC7047074CECE7074C05
:10DAB000EAE7074CE8E700BF284B01002493FF1F6B
:10DAC0008492FF1F95D800004C92FF1F0493FF1F04
:10DAD000D492FF1F30B4054B054D064C0022102197
:10DAE0001A602A602060196030BC704714D003406F
:10DAF00004D0034000D00340282838B52ED0002998
:10DB000004464FDD5F4B1B78012505FA03F28A427C
:10DB100002D8212837D938BD0338C2B2012A3AD9F0
:10DB2000202C4AD0192C48D0574A126802FB011207
:10DB300022FA03F31D2800F29B80DFE800F0928BAD
:10DB4000847D9999766F99999999999999999968F4
:10DB5000615A53994C99999999999945494B1B78D0
:10DB60000B2B08D90C2B1CBF0C3B19410846BDE8F8
:10DB70003840FFF7B9BCC3F10C0399400846BDE833
:10DB80003840FFF7B1BC2946FFF786FE2946BDE8BD
:10DB90003840FFF7A3BE3D4A126802FB011222FA89
:10DBA00003F3C7E72128B6D80021FFF775FE20460A
:10DBB0000121BDE83840FFF791BE354A126802FBEB
:10DBC000011222FA03F3B5E73249334A0B604FF4EE
:10DBD0005173136038BD3149314A0B604FF45173B2
:10DBE000136038BD2F49304A0B6040F24443136044
:10DBF00038BD2E492E4A0B6040F24443136038BDB5
:10DC00002C492D4A0B6040F24443136038BD2B4928
:10DC10002B4A0B6040F24443136038BD29492A4A1D
:10DC20000B6040F24443136038BD2849284A0B601A
:10DC300040F24443136038BD2649274A0B6040F246
:10DC40004443136038BD2549254A0B6040F24443E4
:10DC5000136038BD2349244A0B604FF4517313609D
:10DC600038BD2249224A0B604FF45173136038BD0E
:10DC7000212C3FF650AF7F29D4BF0021012120463F
:10DC800093E700BF2C93FF1F0880034008900340D8
:10DC900008800B4010800B4048A0044018800B40C7
:10DCA0004CA004401880034008B00440108003409A
:10DCB00004B004404080034018C004403880034052
:10DCC00014C004402880034010B00440208003406A
:10DCD0000CB004403080034010C004404880034032
:10DCE0001CC004401890034034900440109003403E
:10DCF0003090044038B1102828BF1020044AC3B225
:10DD0000107813707047024A01231078137070471F
:10DD10002C93FF1F2DE9F8430E4680463249334DC0
:10DD2000304603F095F947F6122300281ABF1D4626
:10DD30004FF002094FF00109002425FA04F002F027
:10DD400091FF4FF05E51074602F0E4FF0146304676
:10DD500003F092F930B90134072CEED1E80902F052
:10DD600081FF07463146384603F088F84FF07C5172
:10DD700002F0C6FE03F0BAF94FF6FF729042A8F126
:10DD8000030328BF1046012B29D9B8F1170F17D864
:10DD9000174B23FA08F303F0010383F0010223B9C0
:10DDA000B8F1190F0FD0BDE8F883124B124D13498B
:10DDB0001A6044EAC9042A6008601C60BDE8F88360
:10DDC000B8F1200FECD10E4B0E4D0F49002244EA62
:10DDD000C9041A602A6008601C60BDE8F8830B4B18
:10DDE0000B4D0C49F2E700BF001BB740006CDC0292
:10DDF0006006F00000800340048003400880034078
:10DE000000800B4004800B4008800B4000900340D2
:10DE10000490034008900340212801D8FFF73CBD3F
:10DE2000704700BF212806D8044B53F8303093F8D0
:10DE30000002C0B270470020704700BF284B0100AD
:10DE4000212801D8FFF74ABD704700BF72B60C49C0
:10DE50000C4B0D4A1B680868126862B6520102D565
:10DE6000322B88BF01300949C3F5BB334FF47A72B6
:10DE7000FF33A1FB031302FB00F000EB931070478C
:10DE800028A0FF1F18E000E004ED00E0ABAAAAAA5A
:10DE90002DE9F843054672B6204F214B214A1B68F5
:10DEA0003C68126862B6520102D5322B88BF013439
:10DEB00095B3C3F5BB331C4EDFF86490DFF8648084
:10DEC000FF334FF47A72A6FB031302FB04F404EB56
:10DED000931472B6D9F800103A68D8F800E062B628
:10DEE000C1F5BB33FF33A6FB03031EF0806FC4EB09
:10DEF00093134FF47A7002D0322988BF013200FBAD
:10DF00000233B3F57A7F04D3013D05D004F57A746A
:10DF1000DFE701F001FEDCE7BDE8F88328A0FF1F82
:10DF200018E000E004ED00E0ABAAAAAAF8B52D4B7A
:10DF30002D49DFF8D0E0DFF8D0C02C4E2C4D2D4C11
:10DF40002D4A2E4F4FF4000018604FF0807018607B
:10DF50004FF0007018604FF0806018604FF0006064
:10DF600018600020086028234BF6FF71CCF80010E1
:10DF7000CEF80030336013602B6023603B60B362E7
:10DF80009362092245F8242CC4F8D80F05F57F6563
:10DF9000C7F8D41F07F5FF2707F5FA67C6F8F83F5B
:10DFA0002B6006F5FF26C4F8D42F05F5FD2504F5F2
:10DFB000FF24386006F2F4761148316005F5FF65FC
:10DFC00004F5FD642B6023600260FFF76BF91920F4
:10DFD000FFF75EFF01F08EF940F21310BDE8F84044
:10DFE000FFF756BF08E100E00480034014800340BF
:10DFF000248003402C8003401C8003403480034075
:10E0000000800B400C800340088003402B4A2C49C1
:10E010001368F0B543F4006313600A78294F2A4E61
:10E020002A4D2B4C2B490023092A3B7033702B704F
:10E0300023700B703DD01A2A21D0274B1B780A2B56
:10E0400025D01F2B30D01F2827D8002002460125BD
:10E05000224B234C1A7023495D7004224FF0020EAC
:10E0600088273C26402598729A704FF4004083F828
:10E0700013E05A751F74DE7025700860F0BD1A4BEE
:10E0800040F213321A60144B1B780A2BD9D1174B6C
:10E090004FF451721F281A60D7D9C0F34432C0F32D
:10E0A000471500F01F00D3E7114B4FF451721A606F
:10E0B000C9E7104B40F213321A60BEE734800440C7
:10E0C0002D93FF1F9CA0FF1F31A0FF1FA4A0FF1FC7
:10E0D0009DA0FF1F30A0FF1F2E93FF1F00B0064022
:10E0E0002FE400E004E100E004D0044010B004405C
:10E0F00000D004400CB0044009B140F08000174A41
:10E100001378984216D010B4154C246824050FD506
:10E1100003F07F030A2B1CD01F2B11D0002900F025
:10E120007F0114BF602344230A290DD01F2902D088
:10E13000107010BC70470B4943F440730B60F7E755
:10E14000084B00241C60E9E7074943F440730B6067
:10E15000EEE7054B00241C60E0E700BF2E93FF1F95
:10E160003480044000D0044010B00440124B1A78B0
:10E1700082420CD011490968090507D5092A16D031
:10E180001A2A0AD009280DD01A2801D01870704711
:10E190000B4A40F213311160F8E7094A00210928BF
:10E1A0001160F1D1074A40F213311160EEE7054AE0
:10E1B00000211160E6E700BF2D93FF1F348004406B
:10E1C00004D004400CB004402DE9F84F234B1B68E9
:10E1D0001A053BD5224B1B680BB101221A70DFF8E0
:10E1E0009090204D99F80040DFF888801E4E013451
:10E1F000272C8ABF4FF0000A5FFA84FA544607467C
:10E20000AB462B789C4216D1FFF700FB40281FDC61
:10E2100033791B06F5D59BF800300133272B86BFD9
:10E2200000221346DAB218F80330DBB2F3712A7019
:10E230002B789C42E8D00D490B4BFFB20120BC2249
:10E2400008F80470087089F800A0DA70BDE8F88F4B
:10E25000FF28D6DD01F060FCD3E700BF3480044026
:10E26000A0A0FF1F9DA0FF1F00B0064030A0FF1F11
:10E27000A4A0FF1F34A0FF1F10B5044C237823B1C6
:10E2800001F04AFC2378002BFAD110BD30A0FF1F0B
:10E29000054A064B10781B78C0B2DBB2984238BFF3
:10E2A0004030C01A704700BF9CA0FF1F31A0FF1F65
:10E2B000F0B4384B1A7912F0300F2CD072B6997D29
:10E2C00001F0FF0200293DD062B6334F3349387860
:10E2D0000D78334E1C46C0B2EDB2431C402BE179A1
:10E2E00028BF0023AB4202F1FF32C9B21CBFF15478
:10E2F000184612F0FF02F0D12A4B1B68C2B23A70E6
:10E300004BB1A84236BFC5F14005401B4019272834
:10E31000C4BF01221A701F49CA78D2B2150616D49A
:10E3200052060DD51B4B1B795B0609D51E4B1F49A9
:10E330001B6800220A7003B11A70164B3C22DA7077
:10E34000F0BC70474022D9795A7462B6E3E70B7982
:10E350001C06E5D5164B174E1C783378E4B2DBB2B9
:10E360009C420ED0144D01E0A3420AD00133282B69
:10E3700028BF00230879E85CC0B2C871087D07286F
:10E38000F2D9DBB2034933700B79180644BF7C2302
:10E39000CB70C5E700B006409CA0FF1F31A0FF1F57
:10E3A0005CA0FF1F2CA0FF1FA0A0FF1F30A0FF1F1D
:10E3B000A4A0FF1F9DA0FF1F34A0FF1F2DE9F84F51
:10E3C000214B1B6807460BB101221A70DFF88890B9
:10E3D0001E4D99F80040DFF884801D4E0134272C33
:10E3E0008ABF4FF0000A5FFA84FA5446AB462B7896
:10E3F000A34216D1FFF70AFA40281FDC33791B0627
:10E40000F5D59BF800300133272B86BF0022134639
:10E41000DAB218F80330DBB2F3712A702B78A3421A
:10E42000E8D00C490A4BFFB208F804700120AC2276
:10E43000087089F800A0DA70BDE8F88FFF28D6DDF3
:10E4400001F06AFBD3E700BF1CA1FF1F19A1FF1F4A
:10E4500000C0064018A1FF1F20A1FF1FB0A0FF1F92
:10E460001C4BDFF894C01A681B49F0B542F4805287
:10E470001A4D1A60DFF884E0194F1A4E1A4C002327
:10E480008CF800304FF451722B701F2840F2133576
:10E490008EF800303B70337025600A6012D8194640
:10E4A0000124124A124D11701248547000212C2779
:10E4B000402693724FF4003491701174D7702E700F
:10E4C0000460F0BDC0F34431C0F3471400F01F03F3
:10E4D000E7E700BF348004400CC00440ADA0FF1F3C
:10E4E00019A1FF1F18A1FF1F08C0044000C006406B
:10E4F00031E400E004E100E0ACA0FF1F20A1FF1F19
:10E50000034B1B68DB0401D5FFF758BF704700BF02
:10E510003480044010B5044C237823B101F0FCFA98
:10E520002378002BFAD110BD18A1FF1F054A064B16
:10E5300010781B78C0B2DBB2984238BF4030C01AA6
:10E54000704700BFACA0FF1FADA0FF1F30B42B4B26
:10E550001A7994061FD52A48DA79037829490133B4
:10E560003F2B0978C8BF00238B42D2B203D0264C80
:10E57000D9B2E2540170254A116861B1244A127877
:10E58000D2B2934236BFC2F140029B1A9B18272B8E
:10E59000C4BF01230B70194AD378DBB2180611D41B
:10E5A0005A060DD5154B1B795B0609D5194B1A492F
:10E5B0001B6800220A7003B11A70104B2C22DA700B
:10E5C00030BC704711790906EAD5144910480C7817
:10E5D0000178C9B28C420DD04A1C272A84BF002181
:10E5E0000A460F4D054C98BFD1B2AA5CD2B2E27177
:10E5F0000170D5E76C21D170D2E700BF00C00640A2
:10E60000ACA0FF1FADA0FF1FD8A0FF1FA8A0FF1F39
:10E6100019A1FF1F1CA1FF1F18A1FF1F20A1FF1F91
:10E62000B0A0FF1F21282FD8184B195CFF292BD031
:10E63000174B184ADFF870C003EBC000F0B5436811
:10E64000DFF868E0144F154D154E00241C60DEF80D
:10E650000030012043F020038840CEF800301460E1
:10E660004FF4A07338602E60C2F800C0013BFDD1AA
:10E6700013689B05FCD42023013BFDD1094B09B253
:10E6800033F8110080B2F0BD00207047384C010013
:10E69000284B01000050044008500440045004403E
:10E6A000000002030051044080014A003880044009
:10E6B000431E032B14D872B60A4951F8230068B1DF
:10E6C00070B4094C058834F81320466841F823607B
:10E6D000521B24F8132062B670BC704762B67047B4
:10E6E000002070477CA1FF1F44A3FF1F01380328AF
:10E6F0000BD872B6074B53F8203043B100205B684B
:10E700000130002BFBD162B67047002070471846DD
:10E71000F9E700BFD0A1FF1F30B472B62B4A1378BF
:10E720001D0706D52A4B196A002936D0996A002997
:10E7300041D053781C0706D5254B196C00293ED0D3
:10E74000996C002939D09378190705D5204B196E9B
:10E75000002936D0996E89B1D3781B0707D51C4B99
:10E76000D3F880207AB3D3F8882011213AB162B669
:10E77000184B00221A7030BC00F04ABE0D21154C17
:10E78000154D227843F8315003EBC1030830013AAC
:10E790005860227062B630BC704704220D4C0F4D99
:10E7A000217843F8325003EBC20308304A1E586008
:10E7B000227062B6EFE70521E1E70921DFE70822D1
:10E7C000ECE70C22EAE71022E8E700BF5C4C01000E
:10E7D0000080FF1FF9A1FF1FC80040008800400013
:10E7E000431E032B1DD81B4A400140F0100030B4DB
:10E7F000104472B6184CE25C032A1BD8DFE802F022
:10E800000212151703220D88E25410F0080F14BFEE
:10E81000C823882343EA054308310360416062B698
:10E8200030BC704708300222EDE70522EBE70830E4
:10E830000422E8E7094A52F8230038B1084A52F89E
:10E840002300416042F8231062B6E9E742F8231042
:10E85000034AF7E70080FF1F08A2FF1FD0A1FF1F98
:10E86000E0A1FF1F00BE70472DE9F04FDFF818B39D
:10E87000DFF818A387B044E0AD4F4FEA930807EBE9
:10E88000C809013ED9F8042003F00803F6B2A2F14A
:10E89000080003F0FF04002B40F0018157F83830E6
:10E8A0001B0C99B222F8081C002B00F0EF80A14B42
:10E8B00022F8064C42F8044C53F82620002A00F0B7
:10E8C000CF819D4D55F8263058609C4C45F8260068
:10E8D00034F81630194424F8161000F079FD002899
:10E8E00000F0C281964A974B19F0080F00F108001A
:10E8F00018BF1346C9F8040047F8383008238BF8CE
:10E9000000309BF80040E4B265071CD58E4B1B78A5
:10E91000B3B18E490A7802F0FF0322B1013BDBB2AA
:10E920000B7003B900BE8A490A7802F0FF032AB1CE
:10E93000013BDBB20B70002B00F0688100F066FE3B
:10E9400004238BF8003004F0080303F0FF02002BCF
:10E9500000F0C9809AF80030DBB21E098CD19A0809
:10E96000DFF8CC9159F8321009EBC200C1F38301F2
:10E97000013940680C2900F28580DFE801F07A7ADD
:10E980008383838383834683838307000168714D78
:10E990004068714F714E6860296088B240F28161B1
:10E9A0000024674B49F832304FF0010E88423C603A
:10E9B000C9F81040C9F8184086F800E05C4A00F237
:10E9C000E780B0F5D06F80F01B82B0F5817F00F05A
:10E9D000D98100F26981802800F02A82822840F0E3
:10E9E000D781A98801F07F01042900F2D1815C4818
:10E9F0005C4A890008441470547001788C0740F117
:10EA0000608382F800E0022173E1534F3A682AB331
:10EA1000554B524E554819883478057840298E4612
:10EA200045F0020828BF4FF0400E002C84F001048E
:10EA30003470CEEB01010CBF8824C82409EBC80652
:10EA400089B285F0010544EA0E447260198049F8E4
:10EA5000384072440570002965D03A603D4B1A88F1
:10EA6000B2F5A06F0ED100219A785970404B1A7000
:10EA700008E038493F4C0D68A54200F098803049C5
:10EA800049F832103C4A0123137037E72C4A2D4BCA
:10EA900019F0080F18BF134647F838302EE700F07A
:10EAA000B7FC364A364952F82630002B00F0E38096
:10EAB00058688C5D42F8260003F10802C9F804206A
:10EAC000032C05D8DFE804F02C02292602228A55FF
:10EAD0001A8819F0080F0CBF8823C82343EA0243A1
:10EAE00047F838300AE7E00700F19380210600F18B
:10EAF000D180A20706D5234A234913780220DBB22E
:10EB000013700870E30602D51F4B10221A7007B06D
:10EB1000BDE8F08F04228A55DAE705228A55D7E747
:10EB200003228A55D4E7BEF1400F18BF002294E7B4
:10EB30000080FF1F7CA1FF1F28A1FF1F44A3FF1F10
:10EB4000C80040008800400004A2FF1F8DA1FF1FE5
:10EB500078A2FF1FF0A1FF1F24A1FF1F8CA1FF1FA0
:10EB6000C0200740FCA1FF1F38A1FF1FF8A1FF1F15
:10EB7000982007402109000394200740D0A1FF1FDF
:10EB800008A2FF1F882007408020074090200740F0
:10EB9000B0F5106F00F07C8140F2A38040F62112A6
:10EBA000904240F07B82A54A012313706AE74C68CB
:10EBB000A3498C427FF463AF0178A9297FF45FAF4A
:10EBC000417845297FF45BAF8178C2297FF457AF44
:10EBD000C1786B297FF453AF9A489B4E0178347803
:10EBE00081F00105002C41F0020105700CBF882066
:10EBF000C82084F0010449F8310009EBC1019348B1
:10EC00003470002505244D60047038E700F064FF7F
:10EC100094E68F4B89488B491A614FF0020E80F8B9
:10EC200000E08C4F0A708C49196099608B4E8C4DB6
:10EC30008C4C9A610D213970FF213170DFF84CE264
:10EC400029702270884D894A8EF800109F27012470
:10EC500006F8047C5D600470DA6007B0BDE8F08FF0
:10EC600043F82600824D30E6824A47F83800137890
:10EC70000133137042E68B5D032B00F2BA8001A2D0
:10EC800052F823F0FDE80000FDE80000DDEC000094
:10EC9000D7EC00006F49724B80220D2008701A706B
:10ECA000A2077FF52FAF26E740F20232904240F0F4
:10ECB000ED81AA8802F07F02042A69D86D88002DB0
:10ECC00066D16449CDF804E0920011440A7842F01C
:10ECD00002020A70C1E101238B550FE600238B5518
:10ECE0000CE6B0F5086F53D16349644A0978117096
:10ECF0007146ED888D4280F0E88252480478402DBC
:10ED0000AE4644F0020C28BF4FF0400E02EB0E035B
:10ED100009EBCC01029301234A604FEA0E48CEEB87
:10ED2000050101930025C82242EA080384F001028C
:10ED300049F83C3035700270DFF814C1424BDFF8FF
:10ED4000048149BBBEF1400F7FF42DAF42F0020CAD
:10ED500009EBCC03029ADFF8F8E05A608DBB0D0492
:10ED600045F088059DF804304EF83C500A44337055
:10ED70000470134640297FF416AF0021404A3B60DF
:10ED8000118010E7AA8802F07F02042A40F28B81EA
:10ED9000304A0F23137006E74029D7D942F0020208
:10EDA0000CEBC200029E4660BDB19DF80450354890
:10EDB0001D703346403988F8004040334CF832002B
:10EDC000DCE79DF8043033700D04029B047045F0BD
:10EDD000C8050B444EF83C50CCE79DF804501D701C
:10EDE000029B1D4888F80040403940334CF83200FF
:10EDF000C4E719F0080F0CBF022303238B557DE5F0
:10EE000021494A68002AC3D06C88B5F804E003E0C1
:10EE10000C314A68002ABBD00B88A342F8D14B883A
:10EE20007345F5D1240A032C0CBF1178098960E7DA
:10EE3000124A0221147054705BE700BF942007400F
:10EE400001000400F8A1FF1F8CA1FF1F8DA1FF1F6F
:10EE50000080FF1FC0200740880040008820074036
:10EE600080200740982007403CA1FF1F90A1FF1F72
:10EE700028A1FF1FF9A1FF1F04A2FF1FFCA1FF1F74
:10EE800038A1FF1FC8004000604C01008C200740E3
:10EE9000B248116AAC7804700C0600F19881D9F878
:10EEA0002820AF49100600F1DB81D9F83020AC49A9
:10EEB000120600F1D081D9F83820A949130600F1D3
:10EEC000C581D9F84020A649150600F1BA81D9F8C4
:10EED0004820A349140600F1AF81D9F85020A04979
:10EEE000100600F1A481D9F858209D49120600F1BE
:10EEF0009981D9F860209A49130600F18E81D9F8DA
:10EF000068209749150600F18381D9F8702094494B
:10EF1000140600F17881D9F878209149100600F1A3
:10EF20006D81D9F880208E49120600F16181D9F8EF
:10EF300088208B49130600F15581D9F89020884923
:10EF4000150600F14981D9F898208549140600F189
:10EF5000FF808448844A854901908548854D864CC8
:10EF6000049700230596029580460F4616461D46D7
:10EF70000394306828B1446800F04AFA2046002C17
:10EF8000F9D100233360029B38681A46002342F807
:10EF9000253028B1446800F03BFA2046002CF9D116
:10EFA00000223A60019A98F800301146002241F898
:10EFB000042B039A0191023B4FF0000122F8151037
:10EFC000032B07D8DFE803F05D025D024FF0010379
:10EFD00088F800300135042D06F1040607F1040716
:10EFE00008F10108C5D1654C654D2278654B049F39
:10EFF000059E0021100729701A7000F19280624965
:10F0000062780A700021C9F83010C9F83810110769
:10F01000DFF84C816ED4A2785C49DFF844810A7035
:10F0200000211207C9F85010C9F858104BD4E278E3
:10F0300057494B4C0A7013074FF00001C9F8701084
:10F04000C9F8781000F1AE8033780193002283F084
:10F050000105C9F89020C9F898200021029188463E
:10F060008E460A464B48047844F0020C09EBCC0368
:10F070000393019B002B039B5A600CBF8822C8227C
:10F0800052E64FF0000388F80030A3E7B0F5A06F18
:10F090007FF47EAE012300250193DEE740F62122B6
:10F0A0009042F7D074E66D88002D7FF471AE3A4936
:10F0B000CDF804E0920011440A7822F002020A70AE
:10F0C000CBE7022115E600F083F9002800F0EB8081
:10F0D0000830324AC8F86400C8F8602000F078F9B7
:10F0E000002800F0DA8008302D4AC9F86C00C9F811
:10F0F00068209CE700F06CF9002800F0E080083000
:10F10000264AC8F84400C8F8402000F061F90028F9
:10F1100000F0CF800830224AC9F84C00C9F84820D6
:10F1200079E700F055F9002800F0A58008301B4A67
:10F13000C9F82400C9F8202000F04AF9002800F09E
:10F1400094800830164AC9F82C00C9F8282056E7E0
:10F15000D1F89C00083800F05BF9FAE604A2FF1F22
:10F160000080FF1FE0A1FF1F7CA1FF1FD0A1FF1F98
:10F1700008A2FF1F28A1FF1F44A3FF1F5C4C010032
:10F18000F9A1FF1FC4200740C8200740CC2007403A
:10F19000D0200740F8A1FF1FC02007408800400092
:10F1A000C800400000F014F9002870D008304F4A21
:10F1B000C4F88400C4F8802000F00AF9002860D068
:10F1C00008304B4AC9F88C00C9F888203CE7506ADF
:10F1D000083800F01DF962E6D1F89400083800F014
:10F1E00017F9B0E6D1F88C00083800F011F9A4E660
:10F1F000D1F88400083800F00BF998E6C86F083899
:10F2000000F006F98DE6486F083800F001F982E653
:10F21000C86E083800F0FCF877E6486E083800F051
:10F22000F7F86CE6C86D083800F0F2F861E6486D52
:10F23000083800F0EDF856E6C86C083800F0E8F839
:10F240004BE6486C083800F0E3F840E6C86B083835
:10F2500000F0DEF835E6486B083800F0D9F82AE609
:10F26000C86A083800F0D4F81FE62A78C9F82800E0
:10F2700001322A70C3E62A78C9F8200001322A70C8
:10F280005AE72A78C9F8880001322A70DCE62A7821
:10F29000C4F8800001322A708EE72A78C9F8680025
:10F2A00001322A70C3E62A78C8F8600001322A7059
:10F2B00014E72A78C9F8480001322A70ABE62A78A8
:10F2C000C8F8400001322A701FE740298E4628BF47
:10F2D0004FF0400E02EB0E0302930123CEEB01012F
:10F2E0004FEA0E4800250193BCE600BF88004000AD
:10F2F000C8004000F8B500F0F9FC294B29482A4C19
:10F300002A4F2B4DDFF8BCC0DFF8BCE0294E0022AD
:10F310001A605A609A60DA601A615A619A61DA6119
:10F320001A625A629A62DA621A635A639A63DA63F9
:10F330001A645A649A64DA641A655A659A65DA65D9
:10F340001A665A669A66DA661A675A679A67DA67B9
:10F35000C3F880200168C3F8842041F48021016053
:10F36000C3F307212170C3F30740134938701B0E04
:10F370002B70FF238CF80030104D8EF800301048B1
:10F380000B700123337084F8642070264FF40074EE
:10F39000102207F82C3C2E70046081F8F820F8BD8C
:10F3A0000080FF1F348004409C200740B0200740AD
:10F3B000B4200740942007401020074049E400E0B3
:10F3C00008E100E08020074088200740704700BF28
:10F3D00072B60D480268B2FA82F30F2B10DC4FF0C0
:10F3E0000041D94022EA0102026062B6074803EBFD
:10F3F000C303DB00C2180021C150104651607047A2
:10F4000062B60020704700BF3093FF1FBC83FF1F10
:10F410000D4B0E4AC31AA2FB03231B090F2B0CD85A
:10F420000B4A127852B972B60A484FF0004102688E
:10F4300021FA03F31A43026062B67047064A127853
:10F44000002AF0D0FFF768B9BC83FF1F398EE3387C
:10F45000F9A1FF1F3093FF1F04A2FF1F38B50E4B09
:10F460000E4C1B68218805468BB1B1F5917F05D202
:10F470000B4A4B1C55549BB2238038BD00220848D0
:10F4800098470021064A55540123238038BDB1F521
:10F49000917FEDD338BD00BF30A2FF1F4EA3FF1FE9
:10F4A00054A3FF1F2DE9F843214E224F3168012359
:10F4B00080463B70B1B1204D4B8801EB8302013394
:10F4C00000240F2BC2F808802C7004D84B80002336
:10F4D0003B70BDE8F88340230B800320FFF780F9E1
:10F4E0003460F4E7DFF8549099F80030002BF0D046
:10F4F000114D45F6215408E0013C12D02B7883B918
:10F5000000F00AFB99F800307BB10320FFF7EEF81A
:10F510000528F1D8FFF75CFF014630600028EBD0EA
:10F52000CAE701232B70BDE8F883BDE8F88300BF6C
:10F530004CA2FF1F20A2FF1F50A2FF1F04A2FF1F0B
:10F540001201F8B5D5B2A1B3012943D043780446DE
:10F5500000781B0643EA004040F4704045F0040682
:10F560008F1E3043FFF79EFF022F04F1020314D9D0
:10F57000053414F8023C14F8032C14F8010C1B0495
:10F5800043EA0223334343EA0060033FFFF78AFF65
:10F59000022F234604F10304EBD8022F23D0012FBE
:10F5A0000DD045F4774040F00500BDE8F840FFF786
:10F5B00079BF14482843BDE8F840FFF773BF1878B7
:10F5C00045F4770545F0060545EA0020BDE8F8401A
:10F5D000FFF768BF03780C4845EA03452843BDE8B8
:10F5E000F840FFF75FBF1A78587845F0774545F047
:10F5F000070545EA022545EA0040BDE8F840FFF767
:10F6000051BF00BF06F0F70007F000F738B5084B10
:10F610001C7824B9074D296809B14B8803B938BD56
:10F620009B000B800320FFF7DBF82C6038BD00BF88
:10F6300020A2FF1F4CA2FF1F2DE9F041AD4E336801
:10F640000746002B00F092801D885A88910803EB32
:10F6500081010432AA428C6842D25A8004F00F061B
:10F660004FEA1428A449A6F1080208F00F00C4F3D9
:10F670000313062A00F101050B701AD9B31E012BE2
:10F680005FFA88F04ED9052E48D0042E00F0A481F0
:10F69000731F022B7FD90F2E0ED1F72842D8F028E6
:10F6A00002D0964B1B883BB1FFF7D8FE0020BDE887
:10F6B000F08127B1BD4202D00020BDE8F081082EC4
:10F6C000C4F3033300F08780092E11D00A2E40F0D6
:10F6D00094800A2BF0D18A4B8A4A1B68A02181E0D2
:10F6E0001846FFF795FE0420FEF7E2FF3060B5E70D
:10F6F000092BE1D1270E00F07B81834B814A1B68E7
:10F700009021C4F307461170EDB2FCB2002B00F05B
:10F710009D80224631462846984797E0F02843D9F5
:10F72000F72841D0F1380E28C6D801A353F820F0AD
:10F73000E7F80000CBF80000B9F80000B9F60000C7
:10F74000B9F60000ABF80000B9F600008BF9000034
:10F75000B9F6000055F900006FF9000093F80000B9
:10F76000B9F600007BF800005FF80000674B1B78DB
:10F77000002BA1D00420FEF79BFF03463060002839
:10F780009AD00588002D7FF460AFFFF741FE356009
:10F790002846BDE8F081FFF761FEC4F30740FFF79C
:10F7A0005DFE072E02D1200EFFF758FE534B584A3C
:10F7B000198858481468584D524A017000270E0A9B
:10F7C000F0201F802E7010700CB301225348A04708
:10F7D0000120BDE8F081082B7FF46EAF504B494A01
:10F7E0001B688021C4F307461170EDB2240E6BB381
:10F7F000284622463146984728E00B2E11D10B2B84
:10F800007FF45AAF474B3F4A1B68B021EAE7464BAB
:10F810001B68002B00F0FB80404898470120BDE8A2
:10F82000F0810C2E40F000810C2B7FF445AF3F4B54
:10F83000344A1B68C0211170EDB2C4F30746002B97
:10F8400000F0C88028463146240E98473849314A8E
:10F85000314B0D7016701C700120BDE8F081354BE6
:10F860001B68002B00F0D6809847C4F30746254B51
:10F87000EDB2240E83F80080E8E72F4B1B68002BC5
:10F88000F2D12E4B1B68A3B1FE209847C4F3074664
:10F89000EDE72B4B1B68002BE6D1284B1B6843B1CF
:10F8A000FC209847C4F30746E1E7264B1B68002B72
:10F8B000DAD1C4F30746DAE7234B1B68C4F30746E3
:10F8C000002BD4D030469847D1E7204B1A68002A45
:10F8D000EFD0260C630C06F07F0003F47E53184330
:10F8E000F6B29047C3E71A4B1B68C4F30746002BD8
:10F8F000E8D1BCE758A2FF1F52A3FF1F4EA3FF1F72
:10F9000034A2FF1F4CA3FF1F68A2FF1F04A2FF1F0A
:10F9100030A2FF1F50A3FF1F51A3FF1F54A3FF1FBF
:10F9200060A2FF1F64A2FF1F48A2FF1F24A2FF1FA7
:10F9300053A3FF1F10A2FF1F14A2FF1F18A2FF1F37
:10F9400054A2FF1F44A2FF1F5CA2FF1F2CA2FF1F97
:10F9500040A2FF1F3F4B1B68002B85D13E4B1B680D
:10F96000002BA6D0FA209847C4F307467FE73B4B0D
:10F970001B68002B7FF478AF374B1B68002B98D0A7
:10F98000FB209847C4F3074671E7354B1B68002BF3
:10F990007FF46AAF304B1B68002B8AD0F820984761
:10F9A000C4F3074663E70E2B7FF486AE2D4A2E4B39
:10F9B0001268E0211970002A47D0260C610C06F06D
:10F9C0007F0301F47E511943EDB2A1F500512846A1
:10F9D0009047F6B2240E39E7FFF740FDC4F3074025
:10F9E000FFF73CFD200EFFF739FD0020BDE8F08158
:10F9F0001E4B1D4A1B6880211170EDB2C4F30746EF
:10FA000083B1314628463A4698473C461EE70120D6
:10FA1000BDE8F081104B1B68002B3FF44AAFFF207C
:10FA2000984746E71C4611E70D2EBCD10D2B7FF4FD
:10FA300043AE0F4B0C4A1B68D0211170EDB2C4F3DA
:10FA40000746002B7FF4FEAEC4E7C4F30746EDB2D1
:10FA5000240EFBE63CA2FF1F18A2FF1F1CA2FF1FE3
:10FA60000CA2FF1F28A2FF1F4CA3FF1F60A2FF1FB5
:10FA700038A2FF1F38B5164D2868E0B101884488C8
:10FA8000A14213DD03191B7A83B104F10803C218E4
:10FA90000C1B002302E012F8011F21B10133A34225
:10FAA000F9D1204638BD1C46204638BDFFF7B0FCD2
:10FAB0000020286038BD074B1B780BB9002038BDEB
:10FAC0000220FEF7F5FD28600028D7D1F6E700BF39
:10FAD00074A2FF1F04A2FF1F0D4B1B78BBB910B50A
:10FAE0000C4C216803F0FF024B883F2B07DC0733E7
:10FAF0000B4401F1470003F8012F8342FBD140235F
:10FB00000B800120FEF76CFE0023236010BD7047C0
:10FB10006CA2FF1F70A2FF1F38B5224C237803B1DF
:10FB200038BD01232370FFF7A5FF70BB00F048F834
:10FB300040BBFEF7ADFB10BBFEF7F8FCE0B90023BD
:10FB40002370EFF30583002BEAD1EFF3108172B637
:10FB5000154B1868E0B1154C2278CAB945691D608B
:10FB600001232370C5B1AA6101B962B600254577AA
:10FB7000836898472570D3E700F020F8DFE700F0AE
:10FB80001BF8D9E700F016F8D3E7FFF71FFCCDE725
:10FB90000029C5D162B638BD054B1D600029E5D1ED
:10FBA000E3E700BF79A2FF1F14A0FF1F18A0FF1FEB
:10FBB00010A0FF1F704700BF704700BF704700BF15
:10FBC000054A064B10781B78C0B2DBB2984238BFAA
:10FBD0004030C01A704700BF80A2FF1F81A2FF1FE4
:10FBE000F0B4384B1A7912F0300F2CD072B6997DE0
:10FBF00001F0FF0200293DD062B6334F3349387817
:10FC00000D78334E1C46C0B2EDB2431C402BE17957
:10FC100028BF0023AB4202F1FF32C9B21CBFF1542E
:10FC2000184612F0FF02F0D12A4B1B68C2B23A709C
:10FC30004BB1A84236BFC5F14005401B40192728EB
:10FC4000C4BF01221A701F49CA78D2B2150616D451
:10FC500052060DD51B4B1B795B0609D51E4B1F4960
:10FC60001B6800220A7003B11A70164B3C22DA702E
:10FC7000F0BC70474022D9795A7462B6E3E70B7939
:10FC80001C06E5D5164B174E1C783378E4B2DBB270
:10FC90009C420ED0144D01E0A3420AD00133402B08
:10FCA00028BF00230879E85CC0B2C871087D072826
:10FCB000F2D9DBB2034933700B79180644BF7C23B9
:10FCC000CB70C5E700A0064080A2FF1F81A2FF1FE6
:10FCD000C4A2FF1F7CA2FF1F08A3FF1F04A3FF1FD6
:10FCE0000CA3FF1F05A3FF1F84A2FF1F70B584B0E4
:10FCF00072B6194B194D1A48702241260F248021E3
:10FD00001A702E701A460470197013781B06FCD5F1
:10FD1000144B186862B6144B144C984298BF00EB11
:10FD2000800001A998BF40000A22FDF78DFD01A9BE
:10FD30002046002311F8012B01333AB10A2B20F899
:10FD4000022FF7D11623237004B070BD5B00DBB225
:10FD5000237004B070BD00BF0000024007000240E5
:10FD600006000240080002407F969800FC93FF1FA7
:10FD70002DE9F043DFF8EC808BB006460F4600F02B
:10FD800073F898F90030013304460D4637D03046F9
:10FD9000394600F0DFF9002831D02BA3D3E9002346
:10FDA0003046394600F026FE814668BB28A3D3E9D9
:10FDB00000233046394600F0FFFD00B398F90030CB
:10FDC000254ACDF82090042400200021022BCDE903
:10FDD0000467CDE9026700940192CDE906012CD0B9
:10FDE000684600F0BDF940B3089B1BB101F0AAF9C9
:10FDF000089B0360DDE906010BB0BDE8F0832046F7
:10FE000029460BB0BDE8F083134A98F900300192FF
:10FE100003210022CDE90467CDE902670091089231
:10FE20002BB90E4B4FF06042CDE90623D8E70C49C1
:10FE30000020022BCDE90601D2D101F083F9222363
:10FE40000360D1E7AFF30080EF39FAFE422E86401F
:10FE500051302DD5104987C0CC4C0100FFFFEF4732
:10FE60000000F07F1294FF1F2DE9F04FB04F21F0FA
:10FE70000042BA4283B00C464FEAD17605460DD90E
:10FE8000AC4FBA4225D9C1F31303034340F0EF80CE
:10FE90000EB10020014603B0BDE8F08FA64B9A4298
:10FEA00000F2CC80A54B9A4200F2DE808AA3D3E90F
:10FEB000002300F05DF90022A14B00F09BFD00281B
:10FEC00000F005812846214600229D4B00F050F9A4
:10FED000E1E783A3D3E9002300F08CFD002840F084
:10FEE000CB802846214680A3D3E9002300F064FD9F
:10FEF0000028CED1934B284603EBC60821467CA3AD
:10FF0000D3E9002300F0E6FAD8E9002300F030F945
:10FF100000F07AFD804600F077FA77A3D3E900235A
:10FF200006460F4600F0D6FA02460B462846214602
:10FF300000F01CF972A3D3E90023CDE9000130469B
:10FF4000394600F0C7FA82468B4652465B46DDE9E9
:10FF5000000100F00BF905460C462A4623462846C8
:10FF6000214600F0B7FA68A3D3E9002306460F46FE
:10FF700000F0B0FA66A3D3E9002300F0F7F83246A8
:10FF80003B4600F0A7FA64A3D3E9002300F0F0F8A1
:10FF900032463B4600F09EFA61A3D3E9002300F00D
:10FFA000E5F832463B4600F095FA5FA3D3E900231B
:10FFB00000F0DEF832463B4600F08CFA02460B4673
:10FFC0002846214600F0D2F806460F46284621462C
:10FFD00032463B46B8F1000F56D000F07BFA32466D
:10FFE00004460D463B4600204FF0804100F0BEF82D
:10FFF00002460B462046294600F096FB02460B4679
:020000021000EC
:100000005046594600F0B2F8DDE9002300F0AEF8A2
:100010000B4602464A49002000F0A8F86FF47F73AF
:1000200098454FDA08F57A7801EB085100224FF035
:10003000B87300F04FFA03B0BDE8F08F424B9A421C
:100040003FF658AF414BF4002344D3E9002300F0BE
:100050008DF83F4BC6F101081C44CDE90001D4E9FD
:1000600000ABC6EB080870E74FF0000875E70246E2
:100070000B4600F07DF80EE717A3D3E900231046E6
:10008000194600F027FA06E700F024FA002280461D
:1000900089464FF080433046394600F067F8024603
:1000A0000B464046494600F03FFB2A46234600F0F7
:1000B0005DF802460B460020214900F057F803B0D6
:1000C000BDE8F08F01EB085103B0BDE8F08F80462A
:1000D00043E700BFAFF300809C7500883CE4377EA7
:1000E000EF39FAFE422E864051302DD5104987C097
:1000F000FE822B654715F73F0000E0FE422EE63FEB
:10010000763C7935EF39EA3DD0A4BE726937663E58
:10011000F16BD2C541BDBB3E2CDE25AF6A56113F07
:1001200093BDBE166CC1663F3E5555555555C53FEE
:10013000412E8640FFFFEF7F422ED63FFFFF2F3E2E
:100140000000F03FD04C0100B1A2F03FF04C0100A4
:10015000E04C010041F0004101F58010C00F7047F4
:100160000020704781F0004102E000BF83F00043AF
:1001700030B54FEA41044FEA430594EA050F08BF42
:1001800090EA020F1FBF54EA000C55EA020C7FEA06
:10019000645C7FEA655C00F0E2804FEA5454D4EB83
:1001A0005555B8BF6D420CDD2C4480EA020281EA4D
:1001B000030382EA000083EA010180EA020281EA85
:1001C0000303362D88BF30BD11F0004F4FEA0131D7
:1001D0004FF4801C4CEA113102D0404261EB4101E6
:1001E00013F0004F4FEA03334CEA133302D052426C
:1001F00063EB430394EA050F00F0A780A4F1010428
:10020000D5F1200E0DDB02FA0EFC22FA05F2801861
:1002100041F1000103FA0EF2801843FA05F3594147
:100220000EE0A5F120050EF1200E012A03FA0EFCC6
:1002300028BF4CF0020C43FA05F3C01851EBE371F0
:1002400001F0004507D54FF0000EDCF1000C7EEB0D
:1002500000006EEB0101B1F5801F1BD3B1F5001F4B
:100260000CD349085FEA30004FEA3C0C04F101046A
:100270004FEA445212F5800F80F09A80BCF1004F93
:1002800008BF5FEA500C50F1000041EB045141EA15
:10029000050130BD5FEA4C0C404141EB010111F416
:1002A000801FA4F10104E9D191F0000F04BF0146C1
:1002B0000020B1FA81F308BF2033A3F10B03B3F19F
:1002C00020020CDA0C3208DD02F1140CC2F10C022F
:1002D00001FA0CF021FA02F10CE002F11402D8BF8D
:1002E000C2F1200C01FA02F120FA0CFCDCBF41EA59
:1002F0000C019040E41AA2BF01EB0451294330BD28
:100300006FEA04041F3C1CDA0C340EDC04F1140404
:10031000C4F1200220FA04F001FA02F340EA0300DB
:1003200021FA04F345EA030130BDC4F10C04C4F121
:10033000200220FA02F001FA04F340EA0300294601
:1003400030BD21FA04F0294630BD94F0000F83F44B
:10035000801306BF81F480110134013D4EE77FEA2E
:10036000645C18BF7FEA655C29D094EA050F08BF7A
:1003700090EA020F05D054EA000C04BF194610465B
:1003800030BD91EA030F1EBF0021002030BD5FEA9F
:10039000545C05D14000494128BF41F0004130BDC7
:1003A00014F580043CBF01F5801130BD01F000451B
:1003B00045F0FE4141F470014FF0000030BD7FEA8E
:1003C000645C1ABF194610467FEA655C1CBF0B4689
:1003D000024650EA013406BF52EA033591EA030FA0
:1003E00041F4002130BD00BF90F0000F04BF002198
:1003F000704730B54FF4806404F132044FF00005CB
:100400004FF0000150E700BF90F0000F04BF002143
:10041000704730B54FF4806404F1320410F00045A9
:1004200048BF40424FF000013EE700BF42004FEAA4
:10043000E2014FEA31014FEA02701FBF12F07F4321
:1004400093F07F4F81F06051704792F0000F14BF1E
:1004500093F07F4F704730B54FF4607401F0004562
:1004600021F0004120E700BF50EA010208BF7047B9
:1004700030B54FF000050AE050EA010208BF7047AE
:1004800030B511F0004502D5404261EB41014FF417
:10049000806404F132045FEA915C3FF4DCAE4FF01B
:1004A00003025FEADC0C18BF03325FEADC0C18BF02
:1004B000033202EBDC02C2F1200300FA03FC20FA53
:1004C00002F001FA03FE40EA0E0021FA02F11444A0
:1004D000C1E600BF70B54FF0FF0C4CF4E06C1CEAB5
:1004E00011541DBF1CEA135594EA0C0F95EA0C0F2A
:1004F00000F0DEF82C4481EA030621EA4C5123EA9D
:100500004C5350EA013518BF52EA033541F48011CB
:1005100043F4801338D0A0FB02CE4FF00005E1FB7E
:1005200002E506F00042E0FB03E54FF00006E1FBC8
:1005300003569CF0000F18BF4EF0010EA4F1FF040B
:10054000B6F5007F64F5407404D25FEA4E0E6D414B
:1005500046EB060642EAC62141EA55514FEAC5205C
:1005600040EA5E504FEACE2EB4F1FD0C88BFBCF5D8
:10057000E06F1ED8BEF1004F08BF5FEA500E50F189
:10058000000041EB045170BD06F0004646EA01014F
:1005900040EA020081EA0301B4EB5C04C2BFD4EB81
:1005A0000C0541EA045170BD41F480114FF0000E7A
:1005B000013C00F3AB8014F1360FDEBF002001F0E8
:1005C000004170BDC4F10004203C35DA0C341BDC62
:1005D00004F11404C4F1200500FA05F320FA04F034
:1005E00001FA05F240EA020001F0004221F0004168
:1005F00010EBD37021FA04F642EB06015EEA430EDB
:1006000008BF20EAD37070BDC4F10C04C4F120050A
:1006100000FA04F320FA05F001FA04F240EA0200BD
:1006200001F0004110EBD37041F100015EEA430E8E
:1006300008BF20EAD37070BDC4F1200500FA05F2AE
:100640004EEA020E20FA04F301FA05F243EA02032D
:1006500021FA04F001F0004121FA04F220EA02003C
:1006600000EBD3705EEA430E08BF20EAD37070BD82
:1006700094F0000F0FD101F00046400041EB010162
:1006800011F4801F08BF013CF7D041EA060195F044
:10069000000F18BF704703F00046520043EB0303FE
:1006A00013F4801F08BF013DF7D043EA06037047EB
:1006B00094EA0C0F0CEA135518BF95EA0C0F0CD0F6
:1006C00050EA410618BF52EA4306D1D181EA03013C
:1006D00001F000414FF0000070BD50EA410606BF36
:1006E0001046194652EA430619D094EA0C0F02D17B
:1006F00050EA013613D195EA0C0F05D152EA0336C0
:100700001CBF104619460AD181EA030101F00041DD
:1007100041F0FE4141F470014FF0000070BD41F026
:10072000FE4141F4780170BD70B54FF0FF0C4CF400
:10073000E06C1CEA11541DBF1CEA135594EA0C0F1F
:1007400095EA0C0F00F0A7F8A4EB050481EA030E6C
:1007500052EA03354FEA013100F088804FEA033353
:100760004FF0805545EA131343EA12634FEA022221
:1007700045EA111545EA10654FEA00260EF00041E2
:100780009D4208BF964244F1FD0404F5407402D234
:100790005B084FEA3202B61A65EB03055B084FEAC5
:1007A00032024FF480104FF4002CB6EB020E75EBC2
:1007B000030E22BFB61A754640EA0C005B084FEAEA
:1007C0003202B6EB020E75EB030E22BFB61A754667
:1007D00040EA5C005B084FEA3202B6EB020E75EBB2
:1007E000030E22BFB61A754640EA9C005B084FEA2A
:1007F0003202B6EB020E75EB030E22BFB61A754637
:1008000040EADC0055EA060E18D04FEA051545EA25
:1008100016754FEA06164FEAC30343EA52734FEACE
:10082000C2025FEA1C1CC0D111F4801F0BD141EA47
:1008300000014FF000004FF0004CB6E711F4801FAC
:1008400004BF01430020B4F1FD0C88BFBCF5E06F8C
:100850003FF6AFAEB5EB030C04BFB6EB020C5FEA9C
:10086000500C50F1000041EB045170BD0EF0004EF1
:100870004EEA113114EB5C04C2BFD4EB0C0541EA23
:10088000045170BD41F480114FF0000E013C90E620
:1008900045EA060E8DE60CEA135594EA0C0F08BFE4
:1008A00095EA0C0F3FF43BAF94EA0C0F0AD150EAE3
:1008B00001347FF434AF95EA0C0F7FF425AF104676
:1008C00019462CE795EA0C0F06D152EA03353FF49E
:1008D000FDAE1046194622E750EA410618BF52EA1B
:1008E00043067FF4C5AE50EA41047FF40DAF52EAEF
:1008F00043057FF4EBAE12E74FF0FF3C06E000BF8C
:100900004FF0010C02E000BF4FF0010C4DF804CD98
:100910004FEA410C7FEA6C5C4FEA430C18BF7FEA58
:100920006C5C1BD001B050EA410C0CBF52EA430C86
:1009300091EA030F02BF90EA020F0020704710F106
:10094000000F91EA030F58BF994208BF90422CBF95
:10095000D8176FEAE37040F0010070474FEA410C8E
:100960007FEA6C5C02D150EA013C07D14FEA430CAC
:100970007FEA6C5CD6D152EA033CD3D05DF8040B1D
:10098000704700BF8446104662468C46194663464F
:1009900000E000BF01B5FFF7B7FF002848BF10F126
:1009A000000F01BD4DF808EDFFF7F4FF0CBF01206B
:1009B00000205DF808FB00BF4DF808EDFFF7EAFFE7
:1009C00034BF012000205DF808FB00BF4DF808EDA2
:1009D000FFF7E0FF94BF012000205DF808FB00BF97
:1009E0004DF808EDFFF7CEFF94BF012000205DF821
:1009F00008FB00BF4DF808EDFFF7C4FF34BF01202E
:100A000000205DF808FB00BF4FEA410212F500121A
:100A100015D211D56FF47873B3EB625212D94FEA45
:100A2000C12343F0004343EA505311F0004F23FA2F
:100A300002F018BF404270474FF00000704750EA84
:100A4000013005D111F0004008BF6FF00040704741
:100A50004FF00000704700BF4FEA4102B2F1E0439F
:100A600024BFB3F5001CDCF1FE5C0DD901F0004C95
:100A70004FEAC0024CEA5070B2F1004F40EB8300E5
:100A800008BF20F00100704711F0804F21D113F111
:100A90003872BCBF01F00040704741F480114FEA4A
:100AA0005252C2F11802C2F1200C10FA0CF320FAD3
:100AB00002F018BF40F001004FEAC1234FEAD323F0
:100AC00003FA0CFC40EA0C0023FA02F34FEA43035A
:100AD000CCE77FEA625307D150EA01331EBF4FF0E3
:100AE000FE4040F44000704701F0004040F0FE40FE
:100AF00040F40000704700BF80F0004002E000BFFB
:100B000081F0004142001FBF5FEA410392EA030FF8
:100B10007FEA226C7FEA236C6AD04FEA1262D2EB42
:100B20001363C1BFD218414048404140B8BF5B4247
:100B3000192B88BF704710F0004F40F4000020F0E0
:100B40007F4018BF404211F0004F41F4000121F0F6
:100B50007F4118BF494292EA030F3FD0A2F1010240
:100B600041FA03FC10EB0C00C3F1200301FA03F17E
:100B700000F0004302D5494260EB4000B0F5000FA1
:100B800013D3B0F1807F06D340084FEA310102F160
:100B90000102FE2A51D2B1F1004F40EBC25008BF12
:100BA00020F0010040EA03007047490040EB0000DC
:100BB00010F4000FA2F10102EDD1B0FA80FCACF10B
:100BC000080CB2EB0C0200FA0CF0AABF00EBC2500A
:100BD00052421843BCBFD0401843704792F0000FF8
:100BE00081F4000106BF80F400000132013BB5E74B
:100BF0004FEA41037FEA226C18BF7FEA236C21D0C1
:100C000092EA030F04D092F0000F08BF0846704725
:100C100090EA010F1CBF0020704712F07F4F04D1F3
:100C2000400028BF40F00040704712F100723CBF06
:100C300000F50000704700F0004343F0FE4040F430
:100C4000000070477FEA226216BF08467FEA2363EE
:100C50000146420206BF5FEA412390EA010F40F4D9
:100C6000800070474FF0000304E000BF10F0004325
:100C700048BF40425FEA000C08BF704743F096430C
:100C800001464FF000001CE050EA010208BF704727
:100C90004FF000030AE000BF50EA010208BF7047AE
:100CA00011F0004302D5404261EB41015FEA010CC3
:100CB00002BF84460146002043F0B64308BFA3F1BB
:100CC0008053A3F50003BCFA8CF2083AA3EBC2539D
:100CD00010DB01FA02FC634400FA02FCC2F12002BC
:100CE000BCF1004F20FA02F243EB020008BF20F0F3
:100CF0000100704702F1200201FA02FCC2F1200259
:100D000050EA4C0021FA02F243EB020008BF20EA4D
:100D1000DC7070474FF0FF0C1CEAD0521EBF1CEA7B
:100D2000D15392EA0C0F93EA0C0F6FD01A4480EA69
:100D3000010C400218BF5FEA41211ED04FF0006352
:100D400043EA501043EA5111A0FB01310CF000407E
:100D5000B1F5000F3EBF490041EAD3715B0040EAA4
:100D6000010062F17F02FD2A1DD8B3F1004F40EB74
:100D7000C25008BF20F00100704790F0000F0CF047
:100D8000004C08BF49024CEA502040EA51207F3A0B
:100D9000C2BFD2F1FF0340EAC250704740F40000E6
:100DA0004FF00003013A5DDC12F1190FDCBF00F0D7
:100DB00000407047C2F10002410021FA02F1C2F185
:100DC000200200FA02FC5FEA310040F1000053EA21
:100DD0004C0308BF20EADC70704792F0000F00F06F
:100DE000004C02BF400010F4000F013AF9D040EA75
:100DF0000C0093F0000F01F0004C02BF490011F409
:100E0000000F013BF9D041EA0C018FE70CEAD15306
:100E100092EA0C0F18BF93EA0C0F0AD030F0004C86
:100E200018BF31F0004CD8D180EA010000F000403A
:100E3000704790F0000F17BF90F0004F084691F0F8
:100E4000000F91F0004F14D092EA0C0F01D1420232
:100E50000FD193EA0C0F03D14B0218BF084608D1FB
:100E600080EA010000F0004040F0FE4040F4000045
:100E7000704740F0FE4040F4400070474FF0FF0CD8
:100E80001CEAD0521EBF1CEAD15392EA0C0F93EA1F
:100E90000C0F69D0A2EB030280EA010C49024FEA71
:100EA000402037D04FF0805343EA111143EA10132A
:100EB0000CF000408B4238BF5B0042F17D024FF4E2
:100EC000000C8B4224BF5B1A40EA0C00B3EB510FBD
:100ED00024BFA3EB510340EA5C00B3EB910F24BFA6
:100EE000A3EB910340EA9C00B3EBD10F24BFA3EB2B
:100EF000D10340EADC001B0118BF5FEA1C1CE0D1F3
:100F0000FD2A3FF650AF8B4240EBC25008BF20F0A5
:100F1000010070470CF0004C4CEA50207F32C2BFF9
:100F2000D2F1FF0340EAC250704740F400004FF096
:100F30000003013A37E792F0000F00F0004C02BFC7
:100F4000400010F4000F013AF9D040EA0C0093F091
:100F5000000F01F0004C02BF490011F4000F013BEB
:100F6000F9D041EA0C0195E70CEAD15392EA0C0F53
:100F700008D142027FF47DAF93EA0C0F7FF470AF8B
:100F8000084676E793EA0C0F04D14B023FF44CAFCE
:100F900008466EE730F0004C18BF31F0004CCAD163
:100FA00030F000427FF45CAF31F000437FF43CAF9F
:100FB0005FE700BF4FF0FF3C06E000BF4FF0010CC1
:100FC00002E000BF4FF0010C4DF804CD4FEA4002A3
:100FD0004FEA41037FEA226C18BF7FEA236C11D0ED
:100FE00001B052EA530C18BF90EA010F58BFB2EBA0
:100FF000030088BFC81738BF6FEAE17018BF40F020
:10100000010070477FEA226C02D15FEA402C05D1D3
:101010007FEA236CE4D15FEA412CE1D05DF8040B58
:10102000704700BF844608466146FFE70FB5FFF7EB
:10103000C9FF002848BF10F1000F0FBD4DF808EDA3
:10104000FFF7F4FF0CBF012000205DF808FB00BF94
:101050004DF808EDFFF7EAFF34BF012000205DF8EE
:1010600008FB00BF4DF808EDFFF7E0FF94BF01203B
:1010700000205DF808FB00BF4DF808EDFFF7D2FF38
:1010800094BF012000205DF808FB00BF4DF808ED7B
:10109000FFF7C8FF34BF012000205DF808FB00BF48
:1010A0004FEA4002B2F1FE4F0FD34FF09E03B3EB75
:1010B00012620DD94FEA002343F0004310F0004FB5
:1010C00023FA02F018BF404270474FF0000070470B
:1010D00012F1610F01D1420205D110F0004008BFAA
:1010E0006FF0004070474FF00000704742000ED292
:1010F000B2F1FE4F0BD34FF09E03B3EB126209D453
:101100004FEA002343F0004323FA02F070474FF008
:101110000000704712F1610F01D1420202D14FF07D
:10112000FF3070474FF00000704700BF0B4601468C
:10113000184600F001B800BF13460A4601460220D7
:1011400000F0B0BE014B1868704700BF4098FF1F09
:1011500070B50F4E0F4D761BB61018BF002405D08A
:10116000013455F8043B9847A642F9D10A4E0B4D7D
:10117000761B03F0C7FDB61018BF002406D001345B
:1011800055F8043B9847A642F9D170BD70BD00BF29
:10119000104D0100104D0100244D0100104D0100C3
:1011A000024B0146186800F00BB800BF4098FF1FC3
:1011B000024B0146186800F039BF00BF4098FF1F7E
:1011C0002DE9F04F01F10B05162D83B0064640F2D4
:1011D0009F8035F0070500F1BF80A94200F2BC8076
:1011E00000F058FBB5F5FC7FC0F09C826B0A00F064
:1011F000BA80042B00F28381A80900F1390E4FEA6E
:101200004E033830C44F07EB8303A3F108015C6839
:10121000A14207D1ACE0002A80F2AC80E468A14290
:1012200000F0A680636823F003035A1B0F2AF2DD47
:10123000B9493C6901F1080E744500F0B381636857
:1012400023F003035A1B0F2A00F39981002AC1F8E7
:1012500014E0C1F810E080F29E80B3F5007F80F0CA
:101260006781DB0803F1010C01229B1002FA03F3F2
:101270004A6851F83C80C4F8088001EBCC091A4355
:10128000A9F10803E3604A6041F83C40C8F80C400B
:10129000831001249C40944200F28A80144206D1BB
:1012A00020F003006400144200F10400FAD007EBC0
:1012B000C009CC468046DCF80C108C4507D173E1A0
:1012C000002A80F28181C9688C4500F06D814B68ED
:1012D00023F003035A1B0F2AF2DD0C46D1F80CC091
:1012E00054F8088F4B1945F001054D6042F001019B
:1012F000C8F80CC03046CCF808807B613B61C3F86D
:101300000CE0C3F808E059609A5000F0C5FA1FE0FD
:10131000102921D800F0BEFA1025062302207E4FA6
:1013200007EB8303A3F108025C68944200F0458157
:101330006368E168A56823F00303234430465A68D4
:10134000E96042F001028D605A6000F0A5FA0834AD
:10135000204603B0BDE8F08F00240C232046336004
:1013600003B0BDE8F08F80234FF0400E3F2049E7E7
:1013700070465DE72344E1685A68A56842F00102BF
:10138000E96030468D605A6000F086FA08342046E5
:1013900003B0BDE8F08F234430465A6842F00102A2
:1013A0005A6000F079FA0834204603B0BDE8F08FA7
:1013B000BC68636823F00308A84504D3C5EB0803A1
:1013C0000F2B00F38C80554BDFF860911A68D9F829
:1013D000003001332A4404EB080A00F0608102F572
:1013E00080520F3222F47F6222F00F021146304603
:1013F000019200F04BFCB0F1FF3F8346019A00F0F0
:101400005881824500F2FC80454B1968DA45114449
:10141000196000F05381D9F80000DFF810E10130C5
:101420001BBFCAEB0B0A5144CEF800B019601BF089
:10143000070100F01781C1F10800C1F58051834414
:1014400008315A44C2F30B02C2EB01094946304647
:10145000019300F01BFC431C019B00F03F81CBEB90
:1014600000024A4442F001021968C7F808B0494432
:10147000BC42CBF804201960DFF8A49016D0B8F174
:101480000F0F40F2FD806268A8F10C0323F0070300
:10149000E01802F001024FF0050E1A430F2B6260B4
:1014A000C0F804E0C0F808E000F21C811D4BBC68E5
:1014B0001A68914288BF19601B4B1A689142626892
:1014C00088BF196022F003029542A2EB050301D800
:1014D0000F2B04DC304600F0DFF9002438E76219F6
:1014E00043F0010345F0010565603046BA60536082
:1014F00000F0D2F90834204603B0BDE8F08F142B79
:1015000071D9542B00F2A480280B00F16F0E4FEA22
:101510004E036E3076E600BF4498FF1F18A3FF1FEE
:101520001CA3FF1F14A3FF1F10A3FF1F509CFF1F2E
:101530005A0A042A5ED9142A00F2B38002F15C012F
:1015400049005B3207EB810C57F82110DFF8DC8192
:10155000ACF1080C8C4500F088804A6822F0030248
:10156000934202D289688C45F7D1D1F80CC07A68D1
:10157000C4F80CC0A160CCF80840CC6088E66319C0
:1015800042F0010745F00105656030464B610B6193
:10159000C3F80CE0C3F808E05F609A50083400F02C
:1015A0007BF9D5E64A6873E608F1010818F0030FE5
:1015B0000CF1080C7FF47FAE30E0DC68A34208BF7A
:1015C00002303FF435AEB3E60B440C465A68C968A6
:1015D00054F8085F42F001025A603046E9608D60BD
:1015E00000F05AF9B4E603F15C0E03F15B004FEA38
:1015F0004E0307E69A0902F1390149003832A1E7A2
:10160000BC424A4B3FF400AF9C68626822F0030280
:101610005AE759F80839994540F0828010F0030FD5
:1016200000F1FF30F5D17B6823EA04037B6064009E
:101630009C423FF6BDAE002C3FF4BAAE1C42404681
:101640007FF435AE64001C4200F10400FAD02EE6AF
:10165000B3F5AA7F18D8E80B00F1780E4FEA4E03D5
:101660007730CFE54FF48051EBE60121D8F8043014
:10167000921001FA02F21A43C8F80420614677E793
:101680000123CBF8043025E740F25452934220D88E
:10169000A80C00F17D0E4FEA4E037C30B2E510320B
:1016A000A4E6542A26D81A0B02F16F0149006E32C3
:1016B00048E7BC68626822F0030205E7CAF30B0042
:1016C00000287FF4A8AE4244BB6842F001025A6091
:1016D000ECE6FE234FF07F0E7E2093E501224FF0D3
:1016E0000009C1E604F10801304600F09FFCD9F87A
:1016F0000010DBE6B2F5AA7F05D8DA0B02F178011B
:10170000490077321EE740F254518A4205D89A0CBC
:1017100002F17D0149007C3214E7FE217E2211E7AF
:101720007B6884E7E808431C5B00F8E54498FF1FEA
:101730008842F0B50DD98B1898420AD28118002A38
:1017400051D09A1A13F8014D01F8014D9342F9D185
:10175000F0BD0F2A48D941EA00039B0746D100F1AA
:10176000100401F11003154653F8106C44F8106C86
:1017700053F80C6C44F80C6C53F8086C44F8086C83
:10178000103D53F8046C44F8046C0F2D03F1100362
:1017900004F11004E8D8A2F1100323F00F0302F0C3
:1017A0000F0E1033BEF1030F1944034421D91E1F3D
:1017B0000D467446043C55F8047B46F8047F032C20
:1017C000F8D8AEF1040424F0030404342344214483
:1017D00002F0030262B1013B0A4411F8014B03F825
:1017E000014F8A42F9D1F0BD0346F3E70346F2E721
:1017F000F0BD7246EEE700BF70B4840746D0541EB9
:10180000002A41D0CDB2034602E0621EE4B3144682
:1018100003F8015B9A07F8D1032C2ED9CDB245EA23
:1018200005250F2C45EA054519D903F11002264676
:10183000103E0F2E42F8105C42F80C5C42F8085C37
:1018400042F8045C02F11002F2D8A4F1100222F076
:101850000F0204F00F041032032C13440DD91E465E
:101860002246043A032A46F8045BFAD8221F22F0E3
:1018700003020432134404F003042CB1C9B21C4423
:1018800003F8011BA342FBD170BC7047144603460A
:10189000C2E700BF704700BF704700BF024B0A4657
:1018A0000146186800F002B84098FF1F2DE9F04F7C
:1018B000174683B0002900F0C1800E46814607F12B
:1018C0000B05FFF7E7FF56F804EC162D2EF0030486
:1018D000A6F1080840D810221546AF4241D89442DC
:1018E00075DAC94B996808EB04008842416800F03A
:1018F000D98021F0010303445B68DB077DD51EF02E
:10190000010F35D039464846FFF75AFC0746E0B18B
:1019100056F8043C23F001034344A0F108029A4224
:1019200000F04481221F242A00F23181132A00F2A0
:101930000481034632461168196051685960926803
:101940009A603146484600F071FB4846FFF7A4FF15
:10195000384603B0BDE8F08F25F00705002D2A4674
:10196000BBDA0C230020C9F8003003B0BDE8F08FCB
:1019700056F8083CC3EB080ADAF8043023F0030CED
:1019800004EB0C039342BDDB5746DAF80C1057F812
:10199000080F221F242AC160886000F21781132AD1
:1019A00040F212813168CAF808107168CAF80C1048
:1019B0001B2A00F22B8108360AF1100231681160EF
:1019C00071685160B16891603E461C46D046631B09
:1019D0000F2B1DD8D8F8043003F0010323434444EF
:1019E000C8F80430636843F0010363604846FFF7BA
:1019F00053FF304603B0BDE8F08F21F003012144CE
:101A0000914221DBC36882680C46D3609A60DEE7AE
:101A1000D8F8042008EB050102F00102154343F059
:101A200001020B44C8F804504A605A6842F00102AF
:101A300008315A60484600F0F9FAD7E7114603B07A
:101A4000BDE8F04FFFF7BCBB1EF0010F7FF45AAFAB
:101A500056F8083CC3EB080ADAF8043023F0030C0C
:101A600001EB0C0E96458BDBC36882685746D3604A
:101A70009A6057F8081FDAF80C30CB60221F242A2E
:101A8000996000F29980132A62D93368CAF8083045
:101A90007368CAF80C301B2A00F2A08008360AF1DD
:101AA000100356E021F0030BA34405F11000834519
:101AB00059DA1EF0010F7FF425AF56F8081CC1EB70
:101AC000080ADAF8041021F0030CE34458453FF704
:101AD00057AF5746DAF80C1057F8080F221F242A80
:101AE000C160886000F2B480132A40F2A58031689A
:101AF000CAF808107168CAF80C101B2A00F2AF80EF
:101B000008360AF110023168116071685160B168DD
:101B100091600AEB0501C5EB0B0242F001029960EE
:101B20004A60DAF8043003F001031D434846CAF85E
:101B30000450FFF7B1FE38465CE733680360736812
:101B400043601B2A27D800F1080306F10802F2E6D9
:101B50003B4632681A6072685A60B2689A603E46C4
:101B60007446D04633E708EB0501C5EB0B0B4BF091
:101B7000010299604A6056F8043C03F001031D43DA
:101B8000484646F8045CFFF787FE304632E73146A8
:101B9000FFF7CEFDD5E6B3688360F368C360242AFF
:101BA00028D000F1100306F11002C4E650F8043CFE
:101BB00023F003031C440AE7314638467446D046F6
:101BC000FFF7B6FD3E4602E73A46F7E631463846AD
:101BD0001C46D046FFF7ACFD3E46F8E6B368CAF8AF
:101BE0001030F368CAF81430242A1BD010360AF1DA
:101BF0001803AEE7336903617369436106F11802A4
:101C000000F1180397E600BF4498FF1FB168CAF8B7
